:100000000C9476070C94A7070C94A7070C94A707E9
:100010000C94A7070C94A7070C94A7070C94A707A8
:100020000C94A7070C94A7070C94A7070C94A70798
:100030000C94A7070C94C68A0C94A7070C94A707E6
:100040000C94A7070C94C1880C94A7070C94A707DD
:100050000C94A7070C94A7070C94A7070C94ED87A2
:100060000C94A7070C9444800C941A800C94A70756
:100070000C94A7070C94A7070C94A7070C94A70748
:100080000C9493880C94A7070C94A7070C94A707CB
:100090000C94A7070C94A7070C94A7070C943D8D0C
:1000A0000C94A7070C94A7070C9465880C94A707D9
:1000B0000C94A7070C94A7070C94A7070C943788F7
:1000C0000C94A7070C94A7070C94A7070C94A707F8
:1000D0000C94A7070C94A7070C94E47F0C94BA7FA8
:1000E0000C94A7070C944D920C9493110C942F1917
:1000F0000C94B4760C941E080C9492080C949F7483
:100100000C941D120C9474140C9485190C94FF74A7
:100110000C943C130C94AE070C9414760C9464125B
:100120000C9481200C9407760C94AC1E0C947F08E0
:100130000C94CE070C9439760C945B130C942676B1
:100140000C94A1760C943E760C94186D0C94D811F6
:100150000C9403760C94D9150C9441750C94187674
:100160000C94DC270C94EE150C940E760C94340849
:100170000C942C760C94E1130C94F1740C948E086E
:100180000C949E740C9485130C942C120C94D80827
:100190000C94DE990C94A0740C94CE740C941E767E
:1001A0000C946F080C94A9080C948E750C94FF188D
:1001B0000C94BA170C94A2080C94D30D0C94027FE3
:1001C0000C94FB130C94BB760C948A080C947E154B
:1001D0000C945D140C94AC080C94F9750C947D0887
:1001E0000C94FF750C94AE110C9482080C94B08C96
:1001F0000C9489170C9431170C94A1740C940B7601
:100200000C94DD0D0C9434760C944F170C943076CE
:100210000C9433110C94AE730C941C140C94DD7478
:100220000C9492760C949D740C9459080C948299B9
:100230000C94F5080C945A190C9473080C944E08FD
:100240000C94A0150C943A760C9422760C942715F5
:100250000C9438080C94E8764E414E494E49545956
:10026000494E46CDCCCC3D0AD7233C17B7D1387781
:10027000CC2B329595E6241FB14F0A000020410097
:1002800000C84200401C4620BCBE4CCA1B0E5AAEE1
:10029000C59D7400407A10F35A00A0724E180900F0
:1002A00010A5D4E80000E87648170000E40B5402DB
:1002B0000000CA9A3B000000E1F505000080969816
:1002C00000000040420F000000A086010000001066
:1002D0002700000000E803000000006400000000A8
:1002E000000A00000000000100000000002C76D889
:1002F00088DC674F0823DFC1DFAE59E1B1B796E56F
:10030000E3E453C63AE651997696E8E6C28426EBD2
:10031000898C9B62ED407C6FFCEFBC9C9F40F2BAE5
:10032000A56FA5F490055A2AF75C936B6CF9676D7D
:10033000C11BFCE0E40D47FEF520E6B500D0ED90D2
:100340002E0300943577050080841E080000204E9F
:100350000A000000C80C333333330F986E12831138
:1003600041EF8D2114893BE65516CFFEE6DB18D10F
:10037000844B381BF77C1D901DA4BBE424203284E1
:10038000725E228100C9F124ECA1E53D27436F6E26
:1003900074656E742D547970653A20746578742F85
:1003A00068746D6C0D0A0D0A3C68313E4550494336
:1003B000204641494C3C2F68313E00485454502F50
:1003C000312E302034303020426164205265717506
:1003D0006573740D0A004163636573732D436F6E1B
:1003E00074726F6C2D416C6C6F772D4F72696769F9
:1003F0006E3A202A0D0A436F6E74656E742D54791F
:1004000070653A20005365727665723A20576562CE
:100410006475696E6F2F312E370D0A0048545450A1
:100420002F312E3020323030204F4B0D0A00436FD9
:100430006E6E656374696F6E3A20636C6F73650DE1
:100440000A436F6E74656E742D547970653A20613D
:1004500070706C69636174696F6E2F782D77777730
:100460002D666F726D2D75726C656E636F64656459
:1004700000506F7374206661696C65640055706C20
:100480006F6164204661696C65643A2000234E6F99
:100490002073656E736F7220666F722074656D7065
:1004A00020262068756D696469747921004E6F207B
:1004B00053656E736F72210020666F722074656DD4
:1004C0007020262068756D69646974792100235352
:1004D000656E736F72204572726F72200053656E85
:1004E000736F72204572726F7221002357726F6EA4
:1004F000672073656E736F7220666F722074656D0E
:100500007020262068756D696469747921005772BE
:100510006F6E672053656E736F7221004320483DF4
:1005200000543D00202020202020202020202020BA
:1005300020202020002020202020202020202020DB
:1005400020202020200020202020202020202020CB
:1005500020202020202000202020202020202020BB
:1005600020202020202000202020202020202020AB
:100570002020202020200054696D657374616D7007
:100580002075706C6F6164206661696C65640053EE
:10059000657474696E6720636C6F636B2074696D3A
:1005A0006500236572726F72202D20004950206112
:1005B0006464726573733A2000416E676C65400035
:1005C000496E76616C696420534D20737465707355
:1005D0002070657220616E676C653D00534D20731D
:1005E000746570732070657220616E676C653D0084
:1005F0003C703E54696D653A20003C2F68333E0ADA
:10060000003C62723E4254206E616D653D003C626A
:10061000723E506174683D003C68333E5379737498
:10062000656D3A2056657273696F6E3D0050617258
:10063000616D657465727320726573657420646F93
:100640006E6521002F6F652F736D6C69676874701C
:100650006F2F73332F00616E676C6520646972655C
:100660006374696F6E3A200043757272656E742010
:10067000534D206973202300534D3A5461626C65D9
:100680002073746570732070657220616E676C658D
:100690003D00534D3A506F6C6172697A65722073F8
:1006A000746570732070657220616E676C653D00C3
:1006B0002344485450494E3D00234448543D0023B0
:1006C0006E65743D424C4500236E65743D57694626
:1006D0006900236E65743D42540023667470207572
:1006E0007365726E616D653A003A0023486F7374EA
:1006F0002073657276657220495020616E642050C7
:100700006F72743A002354696D6520736572766563
:10071000722049503A002352656C617920646576F5
:10072000696365733A002352656C61792073746163
:10073000747573206C6162656C733A200023526596
:100740006C6179207374617465733A002352656C2F
:1007500061792070696E733A00234E6F2E206F66A8
:1007600020636F6E74726F6C2072656C6179733D7B
:1007700000234E6F2E206F662072656C6179733D89
:1007800000234C6F67676572204E616D653A2000EB
:1007900046696E64696E6720576946692049500052
:1007A0004E45543D426C7565746F6F7468204C45BE
:1007B000004E45543D426C7565746F6F7468004E11
:1007C00045543D57694669005344206F70656E205B
:1007D0006661696C004E6577206461746120636FA7
:1007E0006C6C656374696F6E207374617274656498
:1007F0000043757272656E742073657474696E67F8
:10080000733A0053797374656D2072657365742053
:100810006174200023445320546865726D6F6D65C8
:100820007465722063616C696272617465642066CC
:100830006F72202300496E76616C696420616E6777
:100840006C6520666F722000207374657073207071
:10085000657220616E676C653D002073746570730E
:100860002070657220616E676C653D005461626C3A
:100870006520536574203000235475726E74616274
:100880006C6520536574203000506F6C6172697A1A
:1008900065722053657420300023506F6C6172695B
:1008A0007A6572205365742030005461626C652053
:1008B000536574203000235475726E7461626C65E8
:1008C00020536574203000506F6C6172697A6572D4
:1008D0002053657420300023506F6C6172697A6513
:1008E0007220536574203000576946692049503A98
:1008F00000234C6F67676572204E616D653A20007A
:100900004C4F474745520056455253494F4E0052AF
:1009100065626F6F74696E672E2E2E005245424FCE
:100920004F540053657276657220506F7274207553
:100930007064617465640053504F52543D004950D7
:100940002075706461746564005349503D00235400
:10095000696D652053657276657220495020757007
:10096000646174656400545349503D004352454CE2
:1009700041590044485450494E3D0074696D65200A
:10098000696E74657276616C3D0054494D455354EF
:10099000414D503D0054494D455354414D50002365
:1009A00077656273657276657220626567696E73DA
:1009B0000053657474696E67204950005365747400
:1009C000696E6720446576696365204950202E2E44
:1009D0002E005461626C65205365742030002354EE
:1009E00075726E7461626C652053657420300050BE
:1009F0006F6C6172697A65722053657420300023D0
:100A0000506F6C6172697A65722053657420300092
:100A100054657374204C616D70732F46616E730062
:100A20006572726F72206F70656E696E672066699D
:100A30006C653A20004C616D70204D6F746F7200D0
:100A40002354696D65202020202020446174652096
:100A5000202020205365636F6E647320506F6C619B
:100A600072697A6572205461626C652054286F4304
:100A7000292048282529202000696E69742E2064C9
:100A80006F6E652E00534420696E69742E20666176
:100A9000696C65642100696E69742E206661696CF9
:100AA000656421002323204F452057656C636F6DDB
:100AB0006520232300496E697469616C697A696EE7
:100AC0006720534420636172642E2E2E0075706C73
:100AD0006F616420627920465450206661696C65BC
:100AE00064210075706C6F616420627920465450F7
:100AF000204F4B210053797374656D2073746172BC
:100B000074696E672E2E2E003C703E4C616D702015
:100B1000616E64204D6F746F7220447269766572E5
:100B20007320537461747573EFBC9A3C2F703E0050
:100B30003C21646F63747970652068746D6C3E3C11
:100B400068746D6C3E3C686561643E3C6D657461C3
:100B500020636861727365743D227574662D382256
:100B60003E3C7469746C653E4F6E6C696E652065C1
:100B700078706572696D656E74202D20506F6C61A0
:100B800072697A6174696F6E2065666665637473F5
:100B9000206F66206C696768743C2F7469746C659B
:100BA0003E3C2F686561643E3C626F64793E3C6800
:100BB000313E4F6E6C696E65206578706572696D47
:100BC000656E74202D20506F6C6172697A61746952
:100BD0006F6E2065666665637473206F66206C694E
:100BE0006768743C2F68313E003C68343E436F7048
:100BF000797269676874284329323032302D323077
:100C000032322E50726F662E205945554E4720596C
:100C10006175205975656E3C2F68343E3C2F626FBC
:100C200064793E3C2F68746D6C3E003C68313E43F5
:100C3000616E6E6F74206765742073656E736F727A
:100C40002072656164696E6773213C2F68313E00D4
:100C50007C3C3E5E2B3D3F2F5B5D3B2C2A225C00A3
:100C6000000020002300260029002C002F00320065
:100C70000001000003010601090100000A0B02093E
:100C80000C0D0E0807030401000000000000000026
:100C90000000000000000000000000000000000054
:100CA0000000000000001211100000000000000011
:100CB0000000000000000000000000000000000034
:100CC00053797374656D20726573746172746564B1
:100CD00021002053797374656D207265737461729D
:100CE00074656421004E6574776F726B206D616965
:100CF0006E7461696E656420617420002323436F04
:100D00006D6D616E64400000002200250028002BFC
:100D1000002E003100340002010000050108010B23
:100D20000100002100240027002A002D003000339C
:100D30000001010000040107010A01010210202046
:100D4000080810204010204080020102010804021F
:100D50000101020408102040808040201008040295
:100D600001800402018040201008040201080402EE
:100D700001010204081020408001020408102040F4
:100D80008005050505070508080808020202020A91
:100D90000A0808040404040101010101010101031E
:100DA00003030303030303040707070C0C0C0C0CD9
:100DB0000C0C0C0202020206060606060606060BCC
:100DC0000B0B0B0B0B0B0B417070656E64206D658C
:100DD00061732E200053696E676C65206D656173C9
:100DE0002E200053617665206D65617375726520F4
:100DF000746F3A0020202020202020202020202056
:100E0000202020200000000100010010100200013D
:100E1000000100B0000000160000002800000010D3
:100E200000000020000000010001000000000000A0
:100E300000000000000000000000000000000000B2
:100E400000000000000000FF000000FFFF0000FFA6
:100E5000FF0000FFFF0000CFBF0000C7BF0000C3BE
:100E6000BF0000C1BF0000C0BF000000000000C004
:100E7000BF0000C1BF0000C3BF0000C7BF0000CF5C
:100E8000BF0000FFFF0000FFFF00000000000000A7
:100E90000000000000000000000000000000000052
:100EA0000000000000000000000000000000000042
:100EB0000000000000000000000000000000000032
:100EC0000000000000000000000000557365722D56
:100ED0006167656E743A202A0D0A446973616C6C0F
:100EE0006F773A202F0D0A00DE99829911241FBED8
:100EF000CFEFD1E2DEBFCDBF00E00CBF19E0A0E034
:100F0000B2E0ECEFFBE601E00BBF02C007900D92F0
:100F1000AE3CB107D9F725E1AEECB9E001C01D92B6
:100F2000AC3EB207E1F717E0C5E7D7E000E006C046
:100F300021970109802FFE010E9405B3C437D10714
:100F400080E00807A9F70E94969D0C94ECB50C94DC
:100F500000008EBD0DB407FEFDCF0895DC0159964B
:100F6000ED91FC913097B9F083899489A589B68970
:100F70004285538564857585841B950BA60BB70B3D
:100F8000811520E89207A105B10538F08FEF9FE7A2
:100F9000A0E0B0E0089590E080E00895CF93DF9363
:100FA0001F92CDB7DEB76983DC01ED91FC91028021
:100FB000F381E02D41E050E0BE016F5F7F4F199556
:100FC0000F90DF91CF910895FC0120812EBD9B01F0
:100FD0002150310941F051810DB407FEFDCF4EB5CE
:100FE0005EBD4193F5CF61507109860F971F0DB417
:100FF00007FEFDCF2EB5FC0120830895E091480C3B
:10100000F091490C90818091470C809589238083D1
:1010100008958EBD00000DB407FEFDCF8EB5089576
:1010200090E020914A0C233339F40C96982F990FB5
:10103000990F990F80E008954896F8CFCF93DF93EA
:101040001F92CDB7DEB76983DC01ED91FC91028080
:10105000F381E02D41E050E0BE016F5F7F4F1995B5
:101060000F90DF91CF910895FC01818D928D0895AD
:10107000CF93DF931F92CDB7DEB76983DC01ED918B
:10108000FC910280F381E02D41E050E0BE016F5FF2
:101090007F4F19950F90DF91CF910895FC019485B2
:1010A000FB018485981303C081E0983008F080E04C
:1010B0000895CF93DF931F92CDB7DEB76983DC012C
:1010C000ED91FC910280F381E02D41E050E0BE0102
:1010D0006F5F7F4F19950F90DF91CF910895FC01BD
:1010E000768765870895DC01ED91FC91068CF78D7C
:1010F000E02D199591E089270895862F089581E0C4
:101100008627089521E0FC018485883008F020E0DE
:10111000822F0895FC01848595850895FC018489BA
:101120009589089522E134E0FC0131832083FB019D
:101130004089518962897389FC01428353836483A6
:1011400075830895DC01ED91FC91048CF58DE02D03
:10115000199490E080E00895FC01818D928D0097B4
:1011600011F00C94EF8F089561E0FC0184810C94E0
:101170007A80CF93DF93EC018FEF8EBD2FEF8F81BD
:101180009885AC014F5F5F4F58874F838130924005
:1011900028F40DB407FEFDCF2EBDF1CF0DB407FE30
:1011A000FDCFCE010E94B4081E82DF91CF91089539
:1011B000CF93DF93EC01E98DFA8D309749F481E00C
:1011C00090E09B838A8390E080E0DF91CF91089547
:1011D00013821282898D9A8D0E94BE90E98DFA8DBC
:1011E00022813381232B59F7F0CFCF92DF92EF92F8
:1011F000FF920F931F93CF93DF93CDB7DEB7AF97D7
:101200000FB6F894DEBF0FBECDBF7C016A0102E1CC
:1012100014E01A8309831C861B8688EE93E0A0E005
:10122000B0E08D879E87AF87B88B8CE993E09A8773
:101230008987188F0F8B198E1A8E1B8E1C8E88E053
:1012400089A31BA70AA71CA61DA61EA61FA68091E0
:10125000190E90911A0EA0911B0EB0911C0E8EA328
:101260009FA3A8A7B9A78B839C83AD83BE83188651
:101270001F82AE01465D5F4FCE0101960E948D85B3
:1012800081309105B1F4D701ED91FC910488F58985
:10129000E02D1DA30CA38CA59DA5AEA5BFA58EA377
:1012A0009FA3A8A7B9A7A601BE016C5D7F4FC70188
:1012B0001995AF960FB6F894DEBF0FBECDBFDF9184
:1012C000CF911F910F91FF90EF90DF90CF900895F5
:1012D0009F92AF92BF92CF92DF92EF92FF920F93C5
:1012E0001F93CF93DF935C017B018B01D0E0C0E0C3
:1012F000F80191908F016501CC0EDD1EC6010E94A0
:101300003DB1981621F0692DC6010E9445B1219684
:10131000C233F1E0DF0761F7C701DF91CF911F9181
:101320000F91FF90EF90DF90CF90BF90AF909F9084
:101330000895FF920F931F93CF93DF93F82ECAEA7D
:10134000DBE08E0161E0D80112968C910E949781BA
:101350006091690BF80182810E947A8064EF71E0EC
:1013600080E090E00E94ED810E5F1F4FFBE0003BAC
:101370001F0741F7FF2009F447C060916B0B8A817A
:101380000E947A8068EE73E080E090E00E94ED8138
:1013900060916B0B8C810E947A8068EE73E080E034
:1013A00090E00E94ED816091690B8A810E947A80B1
:1013B00068EE73E080E090E00E94ED8122968BE081
:1013C000CE3AD807D1F668EE73E080E090E00E9454
:1013D000ED81C1EDD2E00CEA1BE0E991F991D80171
:1013E0008C910E5F1F4FEE0FFF1FE759F44F608186
:1013F0000E947A8068EC70E080E090E00E94ED81CD
:10140000B2E0C73DDB0749F7DF91CF911F910F9104
:10141000FF90089581E08093EF028091F00288238D
:1014200041F088E08093DF1160E084ED91E10C945D
:10143000838C08958091F0028823F9F08091EF0267
:101440008823D9F081E00E94C78C8BE39FE101974C
:10145000F1F760E080E00E94D88C67E675E084EDEB
:1014600091E10E948A7F61E080E00E94D88C67E56C
:1014700075E084ED91E10C948A7F08950F931F939A
:10148000CF93DF932091F002222309F45CC02091D6
:10149000EF02222309F457C0EA018C016F3F7F4F0E
:1014A000F1F461E080E00E94D88CB80184ED91E114
:1014B0000E94687F66E475E084ED91E10E948A7F76
:1014C00061E0F80184810E94D88CBE01DD0F880B99
:1014D000990BDF91CF911F910F910C94ED810E9498
:1014E000BC84AB01BC0180919B0A90919C0AA091A5
:1014F0009D0AB0919E0A8C599F4FAF4FBF4F8417E2
:101500009507A607B707F8F461E080E00E94D88C41
:10151000B80184ED91E10E94687F65E375E084ED98
:1015200091E10E948A7F61E0F80184810E94D88C59
:101530000E94BC8460939B0A70939C0A80939D0ACE
:1015400090939E0AC2CFDF91CF911F910F91089582
:10155000CF93DF93EC010E94EF8F882311F01D825F
:1015600081E0DF91CF9108953F924F925F926F9209
:101570007F928F929F92AF92BF92CF92DF92EF9223
:10158000FF920F931F93CF93DF93CDB7DEB72C97C6
:101590000FB6F894DEBF0FBECDBF5C01DC015B96D9
:1015A0008D909C905C9716964D905D906D907C9080
:1015B0001997411451046104710409F468C0BFEF24
:1015C0004B1A5B0A6B0A7B0A312CF40181859285E8
:1015D000A385B4859C01AD012F5F3F4F4F4F5F4FF7
:1015E00029873A874B875C87730162011D821E82BF
:1015F0001F821886F40181859285A385B4852D818B
:101600003E814F815885281739074A075B0708F044
:1016100056C089859A85AB85BC858C159D05AE0520
:10162000BF0550F482E0C82ED12CE12CF12C92E0C1
:10163000492E512C612C712C9E012F5F3F4FB70119
:10164000A601C4010E94038F8823C9F189819A8170
:10165000AB81BC81892B8A2B8B2B09F126013701A9
:101660009FEF491A590A690A790A2D813E814F81F3
:1016700058852F5F3F4F4F4F5F4F2D833E834F83E2
:1016800058873FEFC31AD30AE30AF30AB3CFF40132
:1016900040805180628073803324339496CFC41489
:1016A000D504E604F70409F70FEF1FEF2FEF3FE033
:1016B000B701A601C4010E94618E811119C080E0AA
:1016C0002C960FB6F894DEBF0FBECDBFDF91CF9141
:1016D0001F910F91FF90EF90DF90CF90BF90AF9050
:1016E0009F908F907F906F905F904F903F90089564
:1016F000F501468157816085718541155105610568
:10170000710539F097018601C4010E94618E88231A
:10171000B1F2D5011696CD92DD92ED92FC92199719
:10172000332051F0D701C6010196A11DB11DF4016E
:1017300080839183A283B383F5018789908DA18DE6
:10174000B28D892B8A2B8B2B39F4C78AD08EE18EF0
:10175000F28E84818068848381E0B2CF8FEF0E9413
:10176000A9078EB508958F929F92AF92BF92FF9274
:101770000F931F93CF93DF93EC01F62E49015A018B
:101780008E81882319F0CE010E94B90860E08C8117
:101790000E947A808CE291E00E9472858F2D806495
:1017A0000E94A90708E110E0D501C401002E04C081
:1017B000B695A795979587950A94D2F70E94A907A1
:1017C00008501109083F8FEF180771F785E9FF20CE
:1017D00021F088E0F8120DC087E80E94A90710E008
:1017E0000E94AE0B8A8787FF06C01F3F21F01F5F54
:1017F000F7CF8FEFF2CFDF91CF911F910F91FF9035
:10180000BF90AF909F908F900895AF92BF92CF926C
:10181000DF92EF92FF920F931F93CF93DF93EC0130
:101820006901C801820F931F8130924050F58E816B
:10183000882379F088819981AA81BB8184179507D3
:10184000A607B70731F48F819885C816D90608F026
:1018500042C0488359836A837B838B85833039F008
:1018600089E0440F551F661F771F8A95D1F79A01AB
:10187000AB0161E1CE010E94B30B882389F083E0C4
:101880008D83CE010E94B40880E0DF91CF911F913B
:101890000F91FF90EF90DF90CF90BF90AF900895A1
:1018A0000E94BC845B010E94AE0B8A878F3F69F463
:1018B0000E94BC846A197B096D327140A0F38FE0ED
:1018C0008D83CE010E94B408DCCF8E3FB1F4188620
:1018D0001F8281E08E838FEF8EBD2FEF8F819885E1
:1018E0008C159D0560F40DB407FEFDCF2EBD8F81D4
:1018F0009885019698878F83F1CF8DE0E1CFC8015D
:101900000197F7012FEFAF014E195F0948175907EB
:1019100038F40DB407FEFDCF3EB531932EBDF3CFA5
:101920000DB407FEFDCF2EB5E80EF91EF70120839A
:101930008F819885080F191F18870F838985882341
:1019400019F00115124030F08E81882319F0CE0174
:101950000E94B90881E099CF0F931F93CF93DF9333
:10196000EC01890182E1411551056105710599F08C
:101970008B85833039F089E0440F551F661F771F30
:101980008A95D1F79A01AB0168E1CE010E94B30BB1
:10199000882319F084E08D8338C08EEF8EBDF80166
:1019A000C8019E5F0DB407FEFDCF20812EBD0DB492
:1019B00007FEFDCF21812EBD3296E817F90791F77A
:1019C0000DB407FEFDCF8FEF0E94A9078FEF0E9495
:1019D000A9070E94AE0B8A878F71853089F488E54C
:1019E00092E00E9472858823A9F020E030E0A901EE
:1019F0006DE0CE010E94B30B882371F084E1CBCF60
:101A000081E18D83CE010E94B408CE010E94B4080A
:101A100080E00AC085E1BFCF0E94AE0B8111EECFFE
:101A2000CE010E94B40881E0DF91CF911F910F9108
:101A30000895FC01DB0112968D919C91139793837D
:101A4000828384E793E09183808314968C9114972A
:101A5000848315968C911597858316964D915D918B
:101A60006D917C91199746835783608771871A9689
:101A70004D915D916D917C911D974287538764874D
:101A800075871E964D915D916D917C91519746871A
:101A90005787608B718B52968C915297828B53969D
:101AA0004D915D916D917C915697438B548B658BD5
:101AB000768B57964D915D916D917C915A97478B9E
:101AC000508F618F728F5B968D919C91948F838FD5
:101AD0000895DC015996ED91FC91309721F081E059
:101AE0009581911101C080E00895CF93DF93EC01BF
:101AF000898D9A8D009741F00E94A80A898D9A8D50
:101B00000E94C4B31A8E198EDF91CF910895EF927F
:101B1000FF920F931F93CF93DF93EC017B018A0118
:101B20001B821A8288EE93E0A0E0B0E08C839D8354
:101B3000AE83BF8384EF93E0998388838DE190E047
:101B40000E9428B39A8F898F009779F02DE1F701D1
:101B5000DC0101900D922A95E1F74CE050E0B801CC
:101B6000CE010C960E9493B5188EDF91CF911F91F4
:101B70000F91FF90EF900895CF93DF931F92CDB711
:101B8000DEB741E050E0BE016F5F7F4F0E94CA9216
:101B9000019731F4898190E00F90DF91CF91089502
:101BA0008FEF9FEFF9CFFC01818D928D009711F09F
:101BB0000C94BC0D8FEF9FEF08950F931F93CF935D
:101BC000DF93EC01898D9A8D10E000E0009799F089
:101BD0000E94BC0D8C010F3F100769F0898D9A8D12
:101BE000FC01428553856485758541505109610921
:101BF00071090E942A90C801DF91CF911F910F9126
:101C00000895E091480CF091490C80819091470C27
:101C1000892B80830895AF92BF92CF92DF92EF928B
:101C2000FF920F931F93CF93DF9300D01F92CDB7F6
:101C3000DEB78C016B017A0180914A0C8333E9F4A1
:101C40005B016801C40ED51EC016D106A9F10E9421
:101C5000FE078FE00E940908812F0E940908802F4B
:101C60000E9409080F5F1F4F80E00E940908F501DC
:101C700081935F010E94010EE7CF843369F50E94D2
:101C8000FE0719830A838F2D8F778B83EC8264E0A4
:101C900070E0CE0101960E94E407A70170E060E0C9
:101CA000C6010E9463B5E114F10421F0B701C60139
:101CB0000E94E4070E94010EC7010F900F900F9041
:101CC0000F90DF91CF911F910F91FF90EF90DF90D8
:101CD000CF90BF90AF9008950E94FE070F3F11056F
:101CE00009F030F419820A831B8263E070E0D1CFDF
:101CF00017FD0BC019820A8333E0169507953A95B4
:101D0000E1F7007E08600B83F0CFC80126E09695CE
:101D100087952A95E1F7807E19830A830115104C77
:101D200018F480618B83E1CF8861FCCFCF93DF9380
:101D30001F92CDB7DEB720914B0C30E0322F222717
:101D4000260F371F90E0982F882741E050E0BE0112
:101D50006F5F7F4F820F931F0E940B0E89810F9040
:101D6000DF91CF910895AF92BF92CF92DF92EF9221
:101D7000FF920F931F93CF93DF9300D000D01F9259
:101D80001F92CDB7DEB78C017B016A0180914A0CAE
:101D90008333E1F45801A40EB51EA016B10609F470
:101DA0006FC00E94FE0780EF0E940908812F0E94E9
:101DB0000908802F0E9409080F5F1F4FF7018191CA
:101DC0007F010E9409080E94010EE7CF5B01A40E6B
:101DD000B51E8433C1F40E94FE0719830A838D2D3A
:101DE00080688B83CC8264E070E0CE0101960E9413
:101DF000E407AE14BF0409F441C0F70181917F01EB
:101E00000E940908F6CF0E94FE070F3F110509F056
:101E100028F419820A8384E08B830CC017FD17C055
:101E200019820A8333E0169507953A95E1F7007E0B
:101E30000C600B8386E0C816D104A0F5F701DE0123
:101E40001496EA15FB0599F081918D93FACFC8019C
:101E500026E0969587952A95E1F7807E19830A8377
:101E60000115104C10F48461D7CF8C61D5CFB60129
:101E70006D5F7F4FCE0101960E94E4070E94010E24
:101E8000C60128960FB6F894DEBF0FBECDBFDF9116
:101E9000CF911F910F91FF90EF90DF90CF90BF9067
:101EA000AF90089563E070E0CE0101960E94E407D0
:101EB000F70181917F010E940908AE14BF04C1F7A8
:101EC000DDCFCF93DF931F92CDB7DEB741E050E077
:101ED000BE016F5F7F4F90E080E00E940B0E898112
:101EE0000F90DF91CF910895CF93DF93C4E1D0E0BD
:101EF0000E94610F882361F061E070E080E090E073
:101F00000E94ED812197A1F780E0DF91CF910895A4
:101F100081E0FBCFCF93DF931F92CDB7DEB78983EC
:101F200041E050E0BE016F5F7F4F90E080E00E9493
:101F3000B30E0F90DF91CF91089563E070E00C94A1
:101F4000960EDA01E0914B0CF0E0FE2FEE27E60F43
:101F5000F71F90E0982F8827A901BD018E0F9F1FC2
:101F60000C94B30ECF93DF931F921F92CDB7DEB7C1
:101F700079836A8322E030E0AE014F5F5F4F60E11A
:101F800070E00E94A10F0F900F90DF91CF91089504
:101F9000CF93DF931F921F92CDB7DEB779836A8309
:101FA00022E030E0AE014F5F5F4F64E070E00E94DE
:101FB000A10F0F900F90DF91CF910895CF93DF93F2
:101FC0001F92CDB7DEB720914B0C30E0322F222785
:101FD000260F371F90E0982F8827498341E050E073
:101FE000BE016F5F7F4F820F931F0E94B30E0F9051
:101FF000DF91CF910895CF93C82F462F61E070E015
:102000000E94DE0F61E070E08C2F0E94960E81111D
:10201000F9CFCF910895DA01E0914B0CF0E0FE2F5B
:10202000EE27E60FF71F90E0982F8827A901BD0142
:102030008E0F9F1F0C940B0E6F927F929F92AF9208
:10204000BF92CF92DF92EF92FF920F931F93CF93A5
:10205000DF931F921F92CDB7DEB7982E8B013A0106
:10206000690122E030E0AE014F5F5F4F64E270E053
:102070000E940B10E980FA80FE24EF24FE24E00E7B
:10208000F11E9701377040914A0C092D10E0C801EC
:10209000433309F04CC00896982F8827990F990F61
:1020A000990F820F931F473309F446C0A9014C0DC5
:1020B0005D1D4130584008F43FC060E078E05B01AE
:1020C000A21AB30AA501B3010E94B30EA6014A19D0
:1020D0005B09B3016A0D7B1D80914A0C833349F57E
:1020E000085F1F4F000F000F000F80E0902F0E942D
:1020F000B30EEC0CFD1CF982EA8222E030E0AE0166
:102100004F5F5F4F64E270E0892D0E94A10F0F9036
:102110000F90DF91CF911F910F91FF90EF90DF9083
:10212000CF90BF90AF909F907F906F900895409612
:10213000B3CF005F1F4FD6CFA601B301D8CFEF9228
:10214000FF921F93CF93DF931F921F92CDB7DEB7FD
:10215000182F22E030E0AE014F5F5F4F60E270E089
:102160000E940B10E980FA80FE24EF24FE2422E076
:1021700030E0AE014F5F5F4F60E270E0812F0E9460
:102180000B1089819A81982789279827E816F906E4
:1021900089F487E0189FF0011124E350F44FF58291
:1021A000E482C7010F900F90DF91CF911F91FF90B4
:1021B000EF9008957C01DBCFFF920F931F93CF9395
:1021C000DF931F921F92CDB7DEB7F82E22E030E0EA
:1021D000AE014F5F5F4F66E270E00E940B10098115
:1021E0001A8110270127102722E030E0AE014F5F4F
:1021F0005F4F66E270E08F2D0E940B1089819A81FB
:102200009827892798270817190749F4C8010F90BC
:102210000F90DF91CF911F910F91FF9008958C0146
:10222000E3CF44E050E0BC018FE090E00C94B30EAB
:1022300008951F93CF93DF93182F80E591E00E94BC
:102240002478812F0E949F10EC01812F0E949D0F06
:10225000873121F08C3111F0D0E0C0E0CE01DF9168
:10226000CF911F910895FC018485883010F40C945F
:10227000191190E080E00895CF92DF92EF92FF92E3
:102280001F93CF93DF93182F7B01EA014130584011
:1022900010F0C0E0D8E080E591E00E942478812F22
:1022A0000E949F106C01812F0E949D0F873111F0B9
:1022B0008C3121F5CC16DD0670F380E591E00E94AB
:1022C00024789E01A70170E060E0812F0E941C101D
:1022D00060E270E0812F0E94FB0F62E070E0812FCE
:1022E0000E94960E84FD0DC0812F0E949D0F8823B1
:1022F000B9F080E591E00E942478EFCFD0E0C0E013
:10230000DCCF40E162E070E0812F0E94DE0FCE0161
:10231000DF91CF911F91FF90EF90DF90CF900895C4
:10232000D0E0C0E0F4CF0F931F93CF93DF938C01E5
:10233000EA01FC018485883048F40E943C11892B15
:1023400039F481E090E0F80193838283D0E0C0E02B
:10235000CE01DF91CF911F910F910895CF92DF921F
:10236000EF92FF920F931F93CF93DF938B017A012C
:102370006C0129EBC20ED11CF6014081EC012A96BA
:10238000442349F050E0BC0167567F4FCE010E94C4
:102390009311F6011082A701B801CE01DF91CF9110
:1023A0001F910F91FF90EF90DF90CF900C949311BD
:1023B000CF93DF93EC01C754DF4FE88121E02E0F6C
:1023C0002883E80FF92FF11DE756FF4F6083203275
:1023D00049F4BC0167567F4F40E250E00A960E94E4
:1023E0009311188281E090E0DF91CF9108951F93BF
:1023F000CF93DF931F92CDB7DEB7182F80E591E022
:102400000E942478812F0E94100827E0129FF0017B
:102410001124E350F44F22813381377041E050E0C2
:10242000BE016F5F7F4F820F931F0E940B0E898149
:102430000F90DF91CF911F910895FC01808D88301E
:1024400040F4218D328D232B21F00E94F71190E072
:1024500008958FEF9FEF0895CF93DF93FC012485BC
:10246000283028F08FEF9FEFDF91CF910895EC0196
:102470000190F081E02D0084F185E02D1995892BE4
:1024800089F38C850E94F71190E0EECF1F93CF93D4
:10249000DF93182F87E0189FE0011124C350D44F19
:1024A00088819981009761F480E591E00E94247809
:1024B000812F0E94DC102E81821B910999838883D1
:1024C000DF91CF911F910895FC018485883010F42D
:1024D0000C94461290E080E008954F925F927F92B4
:1024E0008F929F92AF92BF92CF92DF92EF92FF9224
:1024F0000F931F93CF93DF931F921F92CDB7DEB739
:10250000782E6B014A01A82EB12C27E0829FC001D2
:102510001124FC01E350F44F7F010081118180E51B
:1025200091E00E9424780815190554F4872D0E9423
:10253000DC10F70126818C01021B11091183008335
:102540000115110519F5872D0E949D0F843159F051
:10255000882349F001E010E08C3111F410E000E034
:10256000119501951109C8010F900F90DF91CF913E
:102570001F910F91FF90EF90DF90CF90BF90AF90A1
:102580009F908F907F905F904F9008958016910656
:102590000CF4840187E08A9DF0018B9DF00D1124DD
:1025A000E350F44FE280F380C114D10451F12701CC
:1025B000F7E05F22872D0E941008840D951D209161
:1025C0004A0C273309F453C09801240D351D2130DE
:1025D000384008F44CC020E038E0490184189508E0
:1025E000A401B6010E940B0E2601480C591C68017B
:1025F000C818D908872D0E941008A601B2010E94B0
:102600000B0EE00EF11E87E08A9DF0018B9DF00D10
:102610001124E350F44FF382E28220813181201BA8
:10262000310B318320838681800F912F911D8A3F4A
:10263000910510F4232BF1F487E08A9DF0018B9D26
:10264000F00D1124E350F44F1682F982EA8222E061
:1026500030E0AE014F5F5F4F68E270E0872D0E946F
:10266000A10F60E470E0872D0E94FB0F7CCFA801D2
:10267000B601C5CF868377CFCF93DF93FC01218D41
:10268000328D2115310529F48FEF9FEFDF91CF9126
:102690000895EC01808D4217530708F0A9010E94AC
:1026A0006D121816190684F7298D3A8D281B390BDF
:1026B0003A8F298FEBCF0F931F93CF93DF931F9206
:1026C000CDB7DEB7FC01218D328D232B41F48FEF86
:1026D0009FEF0F90DF91CF911F910F9108958C0183
:1026E00041E050E0BE016F5F7F4FFC01808D0E9492
:1026F0006D12181619065CF7F801818D928D0197FD
:10270000928F818F898190E0E4CF0F931F93CF93B5
:10271000DF9300D000D01F921F92CDB7DEB78C019F
:10272000D80159964D915C915A974115510551F038
:10273000ED91FC91048CF58DE02D70E060E0C80116
:102740001995EECFF801808D0E944612892BB1F1C8
:1027500048E050E0BE016F5F7F4FD80158968C91E2
:102760000E946D1218161906F4F4D801509684E0F0
:10277000FE01319601900D928A95E1F78D8190E0EE
:10278000982F88272E81820F911DF801958B848BBD
:102790008F81282F30E0322F22278885820F932FB8
:1027A000911D928F818F28960FB6F894DEBF0FBED1
:1027B000CDBFDF91CF911F910F91089590E080E000
:1027C000F2CFCF93DF931F92CDB7DEB741E050E059
:1027D000BE016F5F7F4FFC0184850E946D12181649
:1027E000190634F4898190E00F90DF91CF9108951C
:1027F0008FEF9FEFF9CFFC018485883010F40C94A3
:102800006D1290E080E00895CF93C82F80E591E0AD
:102810000E94247868E070E08C2FCF910C94FB0F1D
:10282000CF93C82F80E591E00E94247860E170E0AA
:102830008C2FCF910C94FB0FCF92DF92EF92FF92EF
:102840000F931F93CF93DF9300D000D0CDB7DEB7A7
:102850008C016B017A01FC01808D883010F40E949C
:10286000101482E194E09A838983F6018281938136
:10287000A481B5818B839C83AD83BE83B701CE01D8
:1028800001960E94A47AF801808F8830A0F4F58622
:10289000E486128E118E81E026960FB6F894DEBF84
:1028A0000FBECDBFDF91CF911F910F91FF90EF90A1
:1028B000DF90CF90089580E0EFCFCF93DF93EC01CE
:1028C000888D883020F40E94101488E0888FDF9172
:1028D000CF910895CF93C82F80E591E00E9424788E
:1028E0008C2FCF910C949D0FEF92FF920F931F931B
:1028F000CF93DF937C0180914A0CD4E0833309F0BD
:10290000D8E005E31CE0C0E0F801219131918F018E
:10291000F701848195812817390729F0CF5FDC13EF
:10292000F3CF80E006C08C2F0E946A148431B1F787
:1029300081E0DF91CF911F910F91FF90EF9008956B
:102940009F92AF92BF92CF92DF92EF92FF920F933E
:102950001F93CF93DF93EC017B0180914A0C81118F
:1029600021C01B821A8288EE93E0A0E0B0E08C8345
:102970009D83AE83BF8386EC93E09983888388E050
:102980008C8788EE93E09E878D87CE01DF91CF9173
:102990001F910F91FF90EF90DF90CF90BF90AF907D
:1029A0009F90089534E0932E833311F028E0922E07
:1029B00085E3C82E8CE0D82E10E098E0B92EA12C2B
:1029C000D6012D913D916D01F701848195812817E4
:1029D000390791F4812F0E946A14082F873111F072
:1029E0008C3139F5812F0E944612892B59F50C3113
:1029F00019F4812F0E9404141F5F9112E1CFA110DE
:102A000008C0D701ED91FC910084F185E02DC7014C
:102A100019951B821A8288EE93E0A0E0B0E08C83C7
:102A20009D83AE83BF8386EC93E099838883BC86C5
:102A3000A8CF843149F08111DFCFF601329711829E
:102A40001082DACFB12ED8CFAA24A394D5CF8F92FB
:102A50009F92AF92BF92CF92DF92EF92FF920F932D
:102A60001F93CF93DF93CDB7DEB72F970FB6F894B0
:102A7000DEBF0FBECDBF5C014B017A0180914A0CD5
:102A80008823C9F104E0833309F008E0B501CE01E1
:102A900001960E94A01485E3C82E8CE0D82E10E089
:102AA000F601219131916F01F501848195812817FB
:102AB000390751F4812F0E946A14873129F4A70144
:102AC000B401812F0E943C111F5F0113E9CFC701A0
:102AD0002F960FB6F894DEBF0FBECDBFDF91CF911A
:102AE0001F910F91FF90EF90DF90CF90BF90AF902C
:102AF0009F908F900895F12CE12CE9CFCF93DF9335
:102B0000EC018C858830D0F40E946A14843189F0FD
:102B1000882379F0883169F021E08C3159F4E8811B
:102B2000F9810084F185E02DCE01199521E0892BF2
:102B300009F420E0822FDF91CF91089580E0FBCF50
:102B4000CF92DF92EF92FF92CF93DF93EC018C85CF
:102B5000883068F40E9404140E94BC846B017C01DC
:102B60008C850E946A14811109C088E08C87DF91EE
:102B7000CF91FF90EF90DF90CF90089561E070E0EB
:102B800080E090E00E94ED810E94BC84AB01BC011A
:102B90004C195D096E097F098D859E85B0E0A0E026
:102BA000481759076A077B07D8F28C850E941014D2
:102BB000DCCFCF93DF93EC018C85883060F40E94EA
:102BC0006A14873111F08C3131F48C850E9419110F
:102BD0008115984088F3DF91CF910895CF92DF92CD
:102BE000EF92FF920F931F93CF93DF93CDB7DEB792
:102BF000AF970FB6F894DEBF0FBECDBF8C016B014F
:102C00007A0182E194E09A8389831B821C821D826F
:102C10001E821C861B8648EE53E060E070E04D8704
:102C20005E876F87788B2CE933E03A872987988F06
:102C30008F8B198E1A8E1B8E1C8E28E029A39BA7C2
:102C40008AA71CA61DA61EA61FA6D8011C968C919D
:102C5000883060F40E946A14882321F0F80184858A
:102C60000E94041488E0D8011C968C938091190E60
:102C700090911A0EA0911B0EB0911C0E8EA39FA3D3
:102C8000A8A7B9A78B839C83AD83BE8318861F82B8
:102C9000AE01465D5F4FB601CE0101960E948D8563
:102CA0000097C1F0D801ED91FC910684F785E02DE5
:102CB00082E194E09DA38CA38CA59DA5AEA5BFA5A4
:102CC0008EA39FA3A8A7B9A7A701BE016C5D7F4FE4
:102CD000C8011995AF960FB6F894DEBF0FBECDBFF1
:102CE000DF91CF911F910F91FF90EF90DF90CF90E8
:102CF00008958F929F92AF92BF92CF92DF92EF9200
:102D0000FF920F931F93CF93DF9300D000D000D09A
:102D10001F92CDB7DEB790914A0C911115C018E003
:102D2000812F2A960FB6F894DEBF0FBECDBFDF917C
:102D3000CF911F910F91FF90EF90DF90CF90BF90B8
:102D4000AF909F908F90089528E0F22E933311F466
:102D500094E0F92E6B01082F80E591E00E94247821
:102D60009E012F5F3F4F5901490110E0812F0E94C2
:102D70009D0FF40181934F018823C1F01F5FF11271
:102D8000F5CFF12CF50191915F019D3149F098311A
:102D900039F09A51923020F0F3941F11F3CFBFCF46
:102DA00060E170E08F2D0E94FB0F1F2DE12EF12CB2
:102DB000F701EE0FFF1FEB5CF34F1182108283EEE1
:102DC00093E00197F1F7402F70E060E0812F0E94BF
:102DD000DE0F4FEF62E070E0812F0E94DE0FB60140
:102DE000CD2889F4809190029091910201968115ED
:102DF000F0EC9F0798F1909391028093900260917C
:102E0000900270919102812F0E94C80F61E070E0E2
:102E1000812F0E94FB0F27E02E9DC0012F9D900D5A
:102E200011249C012350344F7901F9011182108241
:102E300022E030E0AE01475F5F4F68E270E0812F33
:102E40000E940B1089859A85982789279827F70172
:102E50009383828316821582148262CF80E090EC85
:102E6000CACF0F931F93CF93DF93EC018B01888D13
:102E7000883010F40E941014B80182E00E94791684
:102E8000888F883050F41D870C871A8E198E81E048
:102E9000DF91CF911F910F91089580E0F9CF9F921C
:102EA000AF92BF92CF92DF92EF92FF920F931F9358
:102EB000CF93DF938C015B01942EE52EFC01C68835
:102EC000D788F08C80E591E00E9424788F2D0E94B5
:102ED0009F10C92DDE2D8C179D0708F4EC019E0173
:102EE000A501B6018F2D0E941C10F80186899789D3
:102EF0008C0F9D1F978B868BCE01DF91CF911F91F9
:102F00000F91FF90EF90DF90CF90BF90AF909F9088
:102F10000895CF93FC01C08D80E591E00E94247854
:102F200060E270E08C2F0E94FB0F62E070E08C2F5B
:102F30000E94960E84FD16C062E070E08C2F0E9405
:102F4000960E83FF0AC048E162E070E08C2F0E9479
:102F5000DE0F80E090E0CF91089580E591E00E943F
:102F60002478E3CF40E162E070E08C2F0E94DE0F16
:102F700081E0F0CFFF920F931F93CF93DF93EB018C
:102F8000FC01178A168A2A81211109C02B8121117F
:102F900006C02C81211103C02D81222301F141158E
:102FA0005105E9F08A01FC01F08C80E591E00E9476
:102FB0002478AE014E5F5F4F24E030E06CE070E0BB
:102FC0008F2D0E94A10FB8018F2D0E94B20F81E0BA
:102FD00090E0DF91CF911F910F91FF90089580E0D5
:102FE000F7CF7F928F929F92AF92BF92CF92DF9254
:102FF000EF92FF920F931F93CF93DF93CDB7DEB77E
:10300000A6970FB6F894DEBF0FBECDBF8C01762E0B
:10301000942E852E20E2A22ECE0101967C01DC01A9
:10302000EA2D1D92EA95E9F76801F3E4CF0ED11C71
:1030300082E194E09AA389A38FEF8BA38CA38DA345
:103040008EA343E450E0BE016F5D7F4FC6010E9436
:10305000BA17019609F4BFC081E089838A8386E0AC
:10306000B82EBB821C82D80114966D917D918D91F2
:103070009C9117970E940DB36D837E838F839887F1
:1030800089869A8680E890E09C878B874CE150E0A7
:10309000B701C6010E944F17FE0137968AE1DF0192
:1030A0001D928A95E9F74801B8E08B0E911CF40156
:1030B000D70101900D92BA94E1F740E150E0B701D9
:1030C000C6010E944F17F7011192AA94E9F796E002
:1030D000A92EB12C40E250E0B701C6010E944F1763
:1030E000F1E0AF1AB108B1F783E6898392E89A83D9
:1030F00093E59B838C8385E38D8381E08E837F8240
:103100009DE3988797E099878A8786E0F401DE013E
:103110001B9601900D928A95E1F78CE0898B8A8B42
:1031200064E174E0CE0143960E947EB5D8011B96FF
:103130006C91CE0149960E946979F8016485CE01AF
:103140004B960E946979D8011D966C91CE014D96DF
:103150000E9469794EE150E0B701C6010E944F1705
:10316000B3E07B121EC082E3898384E08A83F80186
:1031700096859B8397859C8390899D8391899E8367
:1031800096E39F838887828D8987838D8A87848D44
:103190008B87858D8C874CE050E0B701C6010E947B
:1031A0004F1787E3898386E08A8391E09B8393E0CE
:1031B0009C838D838FE08E838AE38F838BE3888764
:1031C0008FEF898749E050E0B701C6010E944F1791
:1031D000C6010E948917A6960FB6F894DEBF0FBEEF
:1031E000CDBFDF91CF911F910F91FF90EF90DF90B6
:1031F000CF90BF90AF909F908F907F9008950F9346
:103200001F93CF938C01FC016481758181E20E9440
:103210007916C82F8830F8F480E591E00E94247870
:103220008C2F0E949D0F833131F08C2FCF911F91F5
:103230000F910C94041462E070E08C2F0E94FB0F3D
:10324000F80184819581EC2FF0E0EE0FFF1FEB5C1D
:10325000F34F91838083CF911F910F9108950F9326
:103260001F93CF93DF931F921F92CDB7DEB7FC0160
:1032700024852830E0F48C0180E591E00E942478D8
:1032800022E030E0AE014F5F5F4F60E170E0F80197
:1032900084850E940B1089819A8198278927982715
:1032A0000F900F90DF91CF911F910F91089590E0B3
:1032B00080E0F6CF0F931F93CF93DF931F921F925F
:1032C000CDB7DEB7FC0124852830E0F48C0180E521
:1032D00091E00E94247822E030E0AE014F5F5F4F22
:1032E00064E070E0F80184850E940B1089819A8166
:1032F0009827892798270F900F90DF91CF911F91E2
:103300000F91089590E080E0F6CFCF92DF92EF9298
:10331000FF921F93CF93DF93EC017B016A018C85B1
:10332000883048F40E946A14882319F08C850E9422
:10333000041488E08C87F70182819381A481B58190
:103340000097A105B10551F490E080E0DF91CF91A5
:103350001F91FF90EF90DF90CF9008958F3F9F4F88
:10336000AF4FBF4F89F370E060E081E20E947916B1
:10337000182F8C87883040F780E591E00E942478F0
:10338000A7014E5F5F4F24E030E06CE070E0812FDA
:103390000E94A10FB601812F0E94B20F64E070E07D
:1033A000812F0E94FB0F0E94BC846B017C018C85E5
:1033B0000E946A14873111F18C3101F1882321F2C6
:1033C0000E94BC84AB01BC014C195D096E097F09E8
:1033D0008D859E85B0E0A0E084179507A607B70706
:1033E00038F061E070E080E090E00E94ED81DFCF96
:1033F0008C850E94101488E08C87A6CF81E090E035
:10340000A5CFCF93DF93EC0182E194E09983888389
:103410001A821B821C821D8280E591E00E94247822
:10342000BE016E5F7F4F44E050E08FE090E00E946D
:103430000B0ECE01DF91CF9108954F925F926F9264
:103440007F928F929F92AF92BF92CF92DF92EF9234
:10345000FF920F931F93CF93DF93EC011816190679
:103460001CF44C0104972CF0C1E0D0E063E0862E00
:10347000912C8E01000F111F7E01EE0CFF1CEE0C33
:10348000FF1C8C169D060CF4B3C097012C5B3D4FBE
:103490005901F90180819181A281B3819701215263
:1034A0003D4F6901181619061A061B063CF50E94C5
:1034B0001489F60140805180628073806419750917
:1034C00086099709F5014080518062807380461615
:1034D00057066806790658F4108211821282138208
:1034E0000E941489F60160837183828393832196FD
:1034F0000E5F1F4FF4E0EF0EF11CC3CF980129526D
:103500003D4F3901F90180819181980121533D4F4F
:103510005901F9012081318182179307C1F0880F89
:10352000991FFC01E759F44F6081F801E655F44F0B
:1035300080810E947A80F30180819181F5019183DD
:1035400080836CE271E080E090E00E94ED81F60102
:1035500080819181A281B381181619061A061B0673
:1035600034F60E941489F601208131814281538111
:10357000621B730B840B950BF701E154FD4F208107
:10358000318142815381261737074807590708F0D0
:10359000AECFF601108211821282138298012C5A4A
:1035A0003D4F6901F90180819181F50120813181CF
:1035B0008217930709F49BCF880F991FFC01E759E5
:1035C000F44F6081F801E655F44F80810E947A80C3
:1035D000F60180819181F50191838083F3019183CC
:1035E00080836CE271E080E090E00E94ED817FCF0B
:1035F000DF91CF911F910F91FF90EF90DF90CF90CF
:10360000BF90AF909F908F907F906F905F904F9002
:103610000895CF93DF93FC0124813581232B69F03A
:10362000EC01BC0185E29DE00E94767FBE0188E846
:103630009CE0DF91CF910C94767FDF91CF9108953C
:10364000CF93DF93FC0124813581232B69F0EC01BA
:10365000BC0185E29DE00E94687FBE0188E89CE095
:10366000DF91CF910C94687FDF91CF9108958F9275
:103670009F92AF92BF92CF92DF92EF92FF920F9301
:103680001F93CF93DF938C01862F0B30110509F028
:103690009FC090915D11992309F0F89462E10E9416
:1036A0002082EC0180915D11882309F078942097A5
:1036B00001F180E090ECA9E7B4EC80935011909375
:1036C0005111A0935211B0935311809354119093C0
:1036D0005511A0935611B0935711CE3F8FEFD807D5
:1036E00009F4A9C0CF3FDC0709F462C0CCEFDFEFDB
:1036F00030C1C0915811E09059116E2D70E090E0EA
:1037000080E00E9420B02DEC3CEC4CEC5DE30E948C
:103710007FB04B015C016C2F70E090E080E00E9474
:1037200020B09B01AC01C501B4010E94C7B16093F8
:103730005011709351118093521190935311D09165
:103740005A11F0905B116D2F6F7770E090E080E080
:103750000E9420B04B015C016F2D70E090E080E092
:103760000E9420B02DEC3CEC4CEC5DE30E947FB05D
:103770009B01AC01C501B4010E94C7B1D7FD26C0B1
:103780006093541170935511809356119093571173
:10379000CE0DCD0FCF0D81E090E020915C11C213D2
:1037A00002C090E080E0892B09F493C0CFEFDFEFF7
:1037B000CE01DF91CF911F910F91FF90EF90DF909D
:1037C000CF90BF90AF909F908F9008959058D8CF92
:1037D000CFEFDFEF0631110509F0BBC090915D110D
:1037E000992309F0F89461E00E942082EC01809115
:1037F0005D11882309F07894209701F180E090EC26
:10380000A9E7B4EC8093501190935111A0935211F9
:10381000B09353118093541190935511A093561166
:10382000B0935711CF3FDC0719F2209709F451C02C
:10383000229609F05BCFCEEFDFEF8BC0C09159111C
:10384000D0915811609158117091591176276727BE
:10385000762790E080E00E941EB02DEC3CEC4CEC12
:103860005DE30E947FB0609350117093511180937B
:10387000521190935311E0905B11F0905A116F2DFB
:103880006F77762F6E2D90E080E00E941EB02DECB9
:103890003CEC4CEC5DE30E947FB0F7FC18C06093F9
:1038A00054117093551180935611909357118C2F8A
:1038B0008D0F8E0D8F0DC1E0D0E090915C118913BA
:1038C00002C0D0E0C0E0D195C195D109ABCF9058EE
:1038D000E6CFC0905011D0905111E0905211F0906D
:1038E000531120E030E048EC52E4C701B6010E94D9
:1038F000DBB2D0E0C0E0181614F4CBEFDFEF20E02D
:1039000030E0A901C701B6010E9419B087FF02C0CB
:10391000CAEFDFEFC0905411D0905511E0905611CE
:10392000F090571120E030E048EC52ECC701B601AE
:103930000E9419B087FF02C0C9EFDFEF20E030E03E
:1039400040EF52E4C701B6010E94DBB218160CF436
:1039500083C00C30110509F02BCF81E08093830CDC
:103960008CE58093850C1092840C1092860C60E09C
:1039700082EC9DE00E94E87681E00E94938B0E9499
:10398000C8816B017C0180917D0C811168C081E050
:1039900080937D0C80937C0C9FEF90937B0C109216
:1039A0007A0C94E09093790C8093580C8091580C89
:1039B000886B8093580C8091570C813009F028C196
:1039C0001092570C0E94C8816B017C018091580CA9
:1039D0008093BB0080917F0C9091800CA091810C12
:1039E000B091820C892B8A2B8B2BA1F00E94C8816D
:1039F00000917F0C1091800C2091810C3091820CF1
:103A00006C197D098E099F090617170728073907C2
:103A100008F446C08091BC0083FDD8CF85EC80932C
:103A2000BC000E94C8816B017C0180917D0C8130BB
:103A300009F4F0C080917A0C853008F00DC18091B6
:103A40007A0CA9E5BCE0E2EBFBE090E0981769F1A5
:103A50002D9121939F5FFACFC8EFDFEF7ACF80914E
:103A60007F0C9091800CA091810CB091820C892BDD
:103A70008A2B8B2B09F487CF0E94C88100917F0C81
:103A80001091800C2091810C3091820C6C197D0971
:103A90008E099F09061717072807390708F073CF03
:103AA00080917E0C0E94728B80E01092460C809375
:103AB000450C082F10E0CEEFDFEF882309F478CE15
:103AC000CDEFDFEF053011050CF472CECEE8DAE071
:103AD00082EC9DE00E94A17688872196CE018E58C7
:103AE0009A4080179107A4F3C091960A0091970A13
:103AF000602F70E090E080E00E9420B02DEC3CEC64
:103B00004CEC5DE30E947FB06B017C016C2F70E098
:103B100090E080E00E9420B09B01AC01C701B6019B
:103B20000E94C7B16B017C01C0928E0AD0928F0AAD
:103B3000E092900AF092910AD091980A1091990A15
:103B40006D2F6F7770E090E080E00E9420B04B0115
:103B50005C01612F70E090E080E00E9420B02DECCD
:103B60003CEC4CEC5DE30E947FB09B01AC01C501D5
:103B7000B4010E94C7B1D7FD71C06093920A7093DF
:103B8000930A8093940A9093950AC00FCD0FC10FAA
:103B900080919A0AC8130ACE20E030E048EC52E443
:103BA000C701B6010E94DBB2D0E0C0E0181614F4E1
:103BB000CBEFDFEF20E030E040EA50E4C701B60190
:103BC0000E9419B087FF02C0CAEFDFEFC090920ACF
:103BD000D090930AE090940AF090950A20E030E0AB
:103BE00040EF51ECC701B6010E9419B087FF02C037
:103BF000C9EFDFEF20E030E040EF52E4C701B6014B
:103C00000E94DBB218160CF0D3CDC8EFDFEFD0CD99
:103C100085EE05CF80917F0C9091800CA091810C56
:103C2000B091820C892B8A2B8B2B09F4FECE0E943B
:103C3000C88100917F0C1091800C2091810C3091F3
:103C4000820C6C197D098E099F0906171707280732
:103C5000390708F0EACE24CF85E0F3CE90588DCF17
:103C6000CF93DF93FB0122813381DC0113963C93D8
:103C70002E931297448155816681778114964D93D6
:103C80005D936D937C93179740855185628573850D
:103C900018964D935D936D937C931B971C96EF0143
:103CA0002C969C01275E3F4F49914D93A217B30775
:103CB000D9F7218D328DFC01328F218FDF91CF9189
:103CC00008950F931F93CF93DF938C01EB01FE01B7
:103CD00064912196662349F0D801ED91FC91019001
:103CE000F081E02DC8011995F2CFDF91CF911F919E
:103CF0000F910895EF92FF920F931F93CF93DF934D
:103D0000EC017B018A016CE174E00E94611E65E0B8
:103D100074E0CE010E94611E66ED73E0CE010E9448
:103D2000611EB701CE010E94607F67E779E0CE0196
:103D30000E94607F0115110521F0B801CE010E949B
:103D4000607F67E779E0CE01DF91CF911F910F91FE
:103D5000FF90EF900C94607FCF93DF93EC016BEBBF
:103D600073E00E94611E65E074E0CE010E94611E56
:103D70006DE873E0CE01DF91CF910C94611ECF937B
:103D8000DF93EC01FB01248135810E945B7ECE0133
:103D9000DF91CF910895EF92FF920F931F93CF93EE
:103DA000DF9300D000D0CDB7DEB78C017B016DE191
:103DB00074E00E94467E8AE0E816F1042CF466ED79
:103DC00076E0C8010E94217DB701CE0101960E94D4
:103DD000947BBE016F5F7F4FC8010E942B7DCE0197
:103DE00001960E94A77DC80126960FB6F894DEBF03
:103DF0000FBECDBFDF91CF911F910F91FF90EF903C
:103E000008952F923F924F925F926F927F928F927E
:103E10009F92AF92BF92CF92DF92EF92FF920F9359
:103E20001F93CF93DF93CDB7DEB7C258D1090FB63A
:103E3000F894DEBF0FBECDBF6C015B0188EE482E4B
:103E400083E0582E612C712C04EF13E09BE5892E42
:103E5000912C8C0E9D1E8CE0880E911C1B019FEFF7
:103E6000291A390AD6015996ED90FC90F7018581FF
:103E7000823008F493C082859385A485B5858F71BF
:103E80009927AA27BB27892B8A2B8B2B09F086C061
:103E900040E250E0BE016F5F7F4FC7010E94CA92AF
:103EA000803209F07BC08981882309F477C0853E80
:103EB00079F38E3269F38C8583FDEACF22961FAEAB
:103EC0001EAE229784E793E09FAF8EAF24961FAE7D
:103ED0002497BE016F5F7F4FE0E080E04EE2DB01A0
:103EE0009D91BD019032A1F0883049F426E730E081
:103EF0002C0F3D1F2E0F311DD9014C93EF5F26E78C
:103F000030E02C0F3D1F2E0F311DD9019C93EF5F28
:103F10008F5F8B3021F786E790E08C0F9D1F8E0F0F
:103F2000911DFC011082D60159966D917C9121E082
:103F3000AE014A585F4FCE01CE960E94D19388239E
:103F400069F1BE01625C7F4FCE0181960E94190D1E
:103F5000AE014A585F4FBE016F5D7F4FCE01855A5B
:103F60009F4F0E94870DCE01855A9F4F0E94690D79
:103F7000882309F4ACC0F12CFA141B042CF569E079
:103F8000CE0101960E94127ECE0101960E94201B56
:103F9000CE0101960E94A77DF394EECF6F961FAEDF
:103FA0001EAE6F97A3964CAE5DAE6EAE7FAEA3977E
:103FB0006D961FAF0EAF6D97E6961FAE1EAEE697DD
:103FC000A8961FAEA897CFCFB401CE0101960E944C
:103FD000467ECE0101960E94201BCE0101960E94D2
:103FE000A77DE696EEADFFADE697309709F447C0A2
:103FF0008581823008F443C068E674E0CE01019602
:104000000E94467ECE0101960E94091BCE010196B8
:104010000E94A77D6F968EAD9FAD6F979C838B831B
:10402000A3968CAD9DADAEADBFADA3978D839E83A2
:10403000AF83B887A7968CAD9DADAEADBFADA7974A
:1040400089879A87AB87BC871A8309838DE0F4013F
:10405000DE011D9601900D928A95E1F7E6968EADF0
:104060009FADE6979B8F8A8FB101CE0101960E948A
:10407000011FCE01855A9F4F0E94750DF3CE6BE153
:1040800074E0CE0101960E94467ECE0101960E9408
:10409000201BCE0101960E94A77DE696EEADFFADF6
:1040A000E69740E050E0BA01309721F04389548907
:1040B00065897689CE0101960E94C07BCE0101966A
:1040C0000E94091BCE0101960E94A77DD2CFCE5738
:1040D000DF4F0FB6F894DEBF0FBECDBFDF91CF919B
:1040E0001F910F91FF90EF90DF90CF90BF90AF9016
:1040F0009F908F907F906F905F904F903F902F9008
:104100000895CF92DF92EF92FF920F931F93CF9378
:10411000DF93CDB7DEB7C455D1090FB6F894DEBF33
:104120000FBECDBF65965FAF4EAF65972091DB0B9D
:104130003091DC0B2F5F3F4F3093DC0B2093DB0B78
:104140002091F80B2111C1C08B016C0181E080939B
:10415000F80B1092DC0B1092DB0B6DE174E0CE01DA
:10416000895B9F4F0E94467E6DE174E0CE01835BC8
:104170009F4F0E94467E50E040E06EE174E0C60131
:104180000E947A1E0130110509F08EC06DE174E0C5
:1041900088EE9FE00E948A7B6DE174E084EC9FE0F2
:1041A0000E948A7B6596EEADFFAD6597808188237E
:1041B00009F474C000E210E09E012F5F3F4F40E21F
:1041C00050E0BE016F5D7F4FCE018D5A9F4F0E9420
:1041D0006B78049739F3BE016F5D7F4FCE018F5B23
:1041E0009F4F0E94467EBE016F5B7F4FCE01895B71
:1041F0009F4F0E946E7DCE018F5B9F4F0E94A77DD7
:10420000BE016F5F7F4FCE018F5B9F4F0E94467E46
:10421000BE016F5B7F4FCE01835B9F4F0E946E7D1F
:10422000CE018F5B9F4F0E94A77D2D968EAD9FADD7
:104230002D970297029730F467E374E084EC9FE0D7
:104240000E948A7BBE01695B7F4F88EE9FE00E94DF
:104250002B7D63968EAD9FAD6397892B09F4A2CF1A
:1042600067E476E0CE018F5B9F4F0E94467EBE01E1
:10427000635B7F4FCE018F5B9F4F0E94C27C64E4E3
:1042800076E00E94AC7CBC0188EE9FE00E942B7D12
:10429000CE018F5B9F4F0E94A77D84CF68EE7FE0A9
:1042A00084EC9FE00E942B7D1092F80BCE01835B83
:1042B0009F4F0E94A77DCE01895B9F4F0E94A77DE3
:1042C0000FB6F894DEBF0FBECDBFCC5ADF4F0FB68E
:1042D000F894DEBF0FBECDBFDF91CF911F910F913C
:1042E000FF90EF90DF90CF9008950F931F93CF939F
:1042F000DF9300D000D0CDB7DEB720916D0B222325
:10430000A9F08C0168EC77E0CE0101960E94467E10
:10431000B801CE0101960E94C27CBC0185E29DE0FD
:104320000E94767FCE0101960E94A77D26960FB649
:10433000F894DEBF0FBECDBFDF91CF911F910F91DB
:1043400008950F931F93CF93DF93CDB7DEB72C97CC
:104350000FB6F894DEBF0FBECDBF8C010E94BE8A9F
:10436000BC01C8010E94CB1E0E94B68ABC01CE01CE
:1043700007960E94CB1E64E077E0CE0101960E9472
:10438000467EBE01695F7F4FCE0101960E94C27CCE
:10439000BC01C8010E942B7DCE0101960E94A77D21
:1043A000CE0107960E94A77D64E476E0C8010E94D2
:1043B000217D0E94AE8ABC01CE0101960E94CB1ED7
:1043C000BE016F5F7F4FC8010E942B7DCE01019619
:1043D0000E94A77D6EE374E0C8010E94217D0E94C7
:1043E000A68ABC01CE0101960E94CB1EBE016F5F62
:1043F0007F4FC8010E942B7DCE0101960E94A77DB0
:104400006EE374E0C8010E94217D0E949C8ABC0179
:10441000CE0101960E94CB1EBE016F5F7F4FC80187
:104420000E942B7DCE0101960E94A77DC8012C968B
:104430000FB6F894DEBF0FBECDBFDF91CF911F91B5
:104440000F9108950F931F93CF93DF93CDB7DEB7EE
:104450002C970FB6F894DEBF0FBECDBF8C010E9423
:10446000BE8ABC01C8010E94CB1E0E94B68ABC0154
:10447000CE0107960E94CB1E64E077E0CE01019644
:104480000E94467EBE01695F7F4FCE0101960E9469
:10449000C27CBC01C8010E942B7DCE0101960E9406
:1044A000A77DCE0107960E94A77D0E9414890E94D5
:1044B000A3896091D20B70E0CE0107960E94CB1EBB
:1044C00064E077E0CE0101960E94467EBE01695FFE
:1044D0007F4FCE0101960E94C27CBC01C8010E94A0
:1044E0002B7DCE0101960E94A77DCE0107960E94EA
:1044F000A77D64E476E0C8010E94217D0E94AE8A17
:10450000BC01CE0101960E94CB1EBE016F5F7F4FA2
:10451000C8010E942B7DCE0101960E94A77D6EE30B
:1045200074E0C8010E94217D0E94A68ABC01CE01D0
:1045300001960E94CB1EBE016F5F7F4FC8010E9493
:104540002B7DCE0101960E94A77D6EE374E0C80129
:104550000E94217D0E949C8ABC01CE0101960E948E
:10456000CB1EBE016F5F7F4FC8010E942B7DCE0125
:1045700001960E94A77DC8012C960FB6F894DEBF65
:104580000FBECDBFDF91CF911F910F910895CF92B4
:10459000DF92EF92FF920F931F93CF93DF9300D0A0
:1045A00000D0CDB7DEB77C01FB01848195818A0103
:1045B000081B190B101611069CF0C7010E942B7ED8
:1045C000C70126960FB6F894DEBF0FBECDBFDF91B0
:1045D000CF911F910F91FF90EF90DF90CF900895B2
:1045E000CE0101960E943D7ECC24C394D12C64E47C
:1045F00076E0CE0101960E94217DFFEFCF1ADF0AFF
:104600000C151D05A4F7BE016F5F7F4FC7010E9407
:104610002B7ECE0101960E94A77DD2CFDF92EF9232
:10462000FF920F931F93CF93DF93CDB7DEB76297BF
:104630000FB6F894DEBF0FBECDBF8C0110929F0A5B
:104640006DE174E0CE010D960E94467EFF24F39446
:1046500085E29DE00E94FF7420919F0A18161906BA
:104660007CF521112DC085E29DE00E94DD748A3029
:1046700009F07EC089899A89892B09F481C0F0925A
:104680009F0A60E474E0CE0101960E94467EBE015E
:10469000635F7F4FCE0101960E94C27CBC01CE01B8
:1046A00007960E943D7ECE0107960E947521CE019D
:1046B00007960E94A77DCE0101960E94A77D60C04B
:1046C000F12CE12CDD24D394222309F460C08989E4
:1046D0009A89019709F045C06FED74E0CE01079605
:1046E0000E94467EBE01695F7F4FCE010D960E94FB
:1046F000917CF12C811115C060E574E0CE0101962A
:104700000E94467EBE016F5F7F4FCE010D960E94D4
:10471000917CFF24F3948111F12CCE0101960E942B
:10472000A77DCE0107960E94A77DFF20A1F050E053
:1047300040E0BE01635F7F4FCE0101960E94BF1E25
:10474000BE016F5F7F4F8BE89FE00E946E7DCE01C0
:1047500001960E94A77D64E170E080E090E00E94F5
:10476000ED81BE01635F7F4FC8010E942B7E8EC02A
:104770008D3009F47FCF682FCE010D960E94FF7C0B
:104780006AE070E080E090E00E94ED8161CF88E80F
:104790009CE00E94FF741816190614F588E89CE046
:1047A0000E94DD748A30A9F08D3099F090919F0AB3
:1047B00091110FC0682FCE010D960E94FF7C8FEFE4
:1047C000E81AF80A65E070E080E090E00E94ED8170
:1047D000DECF89899A89892BA9F3D0929F0AF2CFDB
:1047E00064E170E080E090E00E94ED81EF2809F440
:1047F0003FC089899A89892BD9F180916D0B8823D3
:1048000089F168EC77E0CE0101960E94467EBE01F8
:104810006F5F7F4FCE010D960E94917CF82ECE01E6
:1048200001960E94A77DF1101DC069E474E0CE01DD
:1048300001960E94467ECE0101960E94201BCE0169
:1048400001960E94A77DBE01635F7F4FCE01019656
:104850000E943D7ECE0101960E94091BCE01019669
:104860000E94A77D64E170E080E090E00E94ED810D
:1048700089899A8920919F0A21112BCF009709F0ED
:1048800028CF6DE174E0C8010E94467ECE010D96EE
:104890000E94A77DC80162960FB6F894DEBF0FBED6
:1048A000CDBFDF91CF911F910F91FF90EF90DF90DF
:1048B00008950F931F93CF93DF93CDB7DEB72C9757
:1048C0000FB6F894DEBF0FBECDBF2C893D89FE0127
:1048D0007496AAEABBE090E080E032962817390788
:1048E00034F0408151814D935D930196F6CFCE5BBC
:1048F000DE4F88819981C254D140281739070CF0C6
:104900001CC2DC01AA0FBB1FA655B44F880F991F0C
:10491000FC01E855F44F8081918101968D939C9321
:104920008C8D9D8D90936A0B8093690B8E8D9F8DDE
:1049300090936C0B80936B0BAD968FADAD97BE01D2
:1049400064597F4F8F3209F001C2CE0107960E9451
:10495000467E62E574E0CE0101960E94467EBE016D
:10496000695F7F4FCE0101960E94C27CBC018CE73B
:1049700091E10E94577DCE0101960E94A77DCE0154
:1049800007960E94A77D6CE771E1CE0101960E9417
:104990003D7ECE0101960E94091BCE0101960E9428
:1049A000A77D68E674E0CE0101960E94467EBE01B6
:1049B0006F5F7F4F8CE791E10E94717C182FCE01D1
:1049C00001960E94A77D4091801150918111112381
:1049D00009F4C3C1BA01625071098CE791E10E94E8
:1049E000607C682FCE0101960E94127EBE016F5F2F
:1049F0007F4F8EE591E10E946E7DCE0101960E946F
:104A0000A77D6EE470E1CE0107960E94467E6AE6BD
:104A100074E0CE0101960E94467EBE01695F7F4F21
:104A2000CE0101960E94C27CBC0186E791E10E9402
:104A3000577DCE0101960E94A77DCE0107960E9468
:104A4000A77D24968FAD24971F928F9323968FADC9
:104A500023971F928F9322968FAD22971F928F9349
:104A600021968FAD21971F928F9380E794E09F93BB
:104A70008F938AE99BE09F938F930E94BCB5CE529F
:104A8000DF4F88819981C25DD04090938D028093E1
:104A90008C02BE016C527F4FCE0101960E94467E71
:104AA000BE016F5F7F4F80E791E10E946E7DCE0176
:104AB00001960E94A77DBE0161527F4FCE010196F3
:104AC0000E94467EBE016F5F7F4F8AE691E10E94A1
:104AD0006E7DCE0101960E94A77D40916E1150918E
:104AE0006F11425051096AE671E1CE0101960E94B0
:104AF000BF1ECE0101960E94F87B6C59609397020D
:104B0000CE0101960E94A77DCC5EDE4F688179813F
:104B10008A819B81C451D1400E9420B00FB6F89485
:104B2000DEBF0FBECDBF9B01AC010E94E0B2882367
:104B300089F08CE390E0A0E0B0E0CC5EDE4F8883AB
:104B40009983AA83BB83C451D140CD5EDE4F1882C6
:104B5000C351D140CD5EDE4F8881C351D1408823FF
:104B600099F0CC5EDE4F88819981AA81BB81C451C6
:104B7000D14080936E0290936F02A0937002B09325
:104B8000710281E08093500CC85EDE4F68817981AC
:104B90008A819B81C851D1409B01AC010E94E0B247
:104BA000882361F080E090E0A0E7B2E4C85EDE4FC9
:104BB00088839983AA83BB83C851D140C45EDE4FEA
:104BC00068817981CC51D140072E000C880B990B5C
:104BD0000E9420B09B01AC010E94E0B2882341F00A
:104BE00082E090E0C45EDE4F99838883CC51D1404F
:104BF000CE5BDE4F68817981C254D140072E000C14
:104C0000880B990B0E9420B09B01AC010E94E0B27E
:104C1000882341F083E090E0CE5BDE4F9983888368
:104C2000C254D140C45CDE4F08811981CC53D140BD
:104C3000B801012E000C880B990B0E9420B09B013B
:104C4000AC010E94E0B2811103C01016110644F0BD
:104C500080E590E0C45CDE4F99838883CC53D140DB
:104C6000C45CDE4F88819981CC53D14090933F0240
:104C700080933E0288E2FE01E551FF4FAEE6BBE0C5
:104C800001900D928A95E1F7CE5CDE4F8881998183
:104C9000AA81BB81C253D1408093290290932A02FA
:104CA000A0932B02B0932C02CA5CDE4F88819981BD
:104CB000AA81BB81C653D1408093250290932602DE
:104CC000A0932702B0932802C65CDE4F88819981A9
:104CD000CA53D14090935D0280935C02CC5BDE4F5F
:104CE00068817981C454D140072E000C880B990B40
:104CF0000E9420B09B01AC010E94E0B2882341F0E9
:104D000088E390E0CC5BDE4F99838883C454D14024
:104D1000CC5BDE4F88819981C454D14090938F023F
:104D200080938E022C960FB6F894DEBF0FBECDBFD7
:104D3000DF91CF911F910F9108958091AE0B9091CB
:104D4000AF0B9093B10B8093B00BEACDCE010796D9
:104D50000E94467E67E574E0FECD415051096CE744
:104D600071E1CE0101960E94BF1EBE016F5F7F4FB1
:104D70008EE591E10E946E7DCE0101960E94A77D95
:104D80006CE771E1CE0101960E943D7E68E674E019
:104D9000CE0101960E94AC7CBC018CE791E10E949F
:104DA000577D2BCEDF92EF92FF920F931F93CF93FD
:104DB000DF93CDB7DEB762970FB6F894DEBF0FBEB4
:104DC000CDBF2091F002222379F12091EF0222231E
:104DD00059F17A018C016F3F7F4FA1F560E080E0CF
:104DE0000E94D88CD12CB80184ED91E10E94687F9B
:104DF00064E275E084ED91E10E948A7FF80184818C
:104E000060E08D0D0E94D88C0E94BC846093530C8E
:104E10007093540C8093550C9093560CB701FF0C73
:104E2000880B990B0E94ED8162960FB6F894DEBF55
:104E30000FBECDBFDF91CF911F910F91FF90EF90EB
:104E4000DF90089560E080E00E94D88C0E94BC84CE
:104E500028EE33E040E050E00E9463B1CA01B9019E
:104E600020E831E541E050E00E9485B1AB01BC0192
:104E700020E0CE0101960E94E57DBE016F5F7F4F6D
:104E8000CE0107960E943D7E62EB78E0CE01079648
:104E90000E94AC7CBC01CE010D960E943D7ECE01ED
:104EA00007960E94A77DCE0101960E94A77DBE01B4
:104EB000635F7F4F84ED91E10E94687FD98860E055
:104EC0008D2D0E94D88CCE010D960E94A77D8BCF90
:104ED000CF93DF9300D000D0CDB7DEB70E941A0A7F
:104EE000CE0101960E94A1214AE050E06FEF7FEFD2
:104EF000CE0101960E94D226CE0101960E94A77D86
:104F000061E080E00E94D88CCE0101960E94011AD7
:104F100064ED71E1CE0101960E94027F6CE774E0BE
:104F200084ED91E10E94607F0E94BC846093E50B58
:104F30007093E60B8093E70B9093E80B26960FB6E1
:104F4000F894DEBF0FBECDBFDF91CF9108950F93D0
:104F50001F93CF93DF9300D000D0CDB7DEB78C0185
:104F6000CE0101960E94A1214AE050E06FEF7FEF51
:104F7000CE0101960E94D226CE0101960E94A77D05
:104F8000B801CE0101960E943D7E4AE050E06FEFED
:104F90007FEFCE0101960E943E0ACE0101960E944B
:104FA000A77D26960FB6F894DEBF0FBECDBFDF916A
:104FB000CF911F910F910895EF92FF920F931F933E
:104FC000CF93DF9300D01F92CDB7DEB78C017B016A
:104FD000FB0184858830A8F082E194E0F801918398
:104FE00080831282138214821582C8010F900F9061
:104FF0000F900F90DF91CF911F910F91FF90EF9045
:10500000089580E591E00E94247824E030E0AE012C
:105010004F5F5F4F6CE070E0F70184850E940B10DA
:10502000BE016F5F7F4FC8010E94AE7FDECF3F920F
:105030004F925F926F927F928F929F92AF92BF92A8
:10504000CF92DF92EF92FF920F931F93CF93DF9354
:10505000CDB7DEB7EA970FB6F894DEBF0FBECDBF6F
:105060007C012A013B0169010E94BC844B015C0167
:1050700087010D5B1F4FC8010E9485131816190682
:105080009CF00E94BC84681979098A099B0946161C
:1050900057066806790608F466C162E370E080E0AE
:1050A00090E00E94ED81E7CF42E250E0BE016F5FE9
:1050B0007F4FC8010E943C1389818230D1F0312C8E
:1050C000832DEA960FB6F894DEBF0FBECDBFDF91F9
:1050D000CF911F910F91FF90EF90DF90CF90BF90F5
:1050E000AF909F908F907F906F905F904F903F9088
:1050F0000895F801848995898334910501F76D81BC
:105100007E818F8198850E940DB34B015C01F60171
:1051100080829182A282B38246E050E0B701685F4C
:105120007F4FCE014D960E943BB5892B41F6F7018A
:1051300080819181A281B38188169906AA06BB0657
:1051400008F4BDCF84819581A681B7818815990522
:10515000AA05BB0508F4B3CF89899A89AB89BC89B4
:1051600086879787A08BB18B4EEC50E070E060E0B3
:10517000C8010E943C13312CC701829698AB8FA7BF
:10518000F701B696FAABE9AB08969CAB8BAB67011F
:105190009AE1C90ED11CBD96FEABEDABC70142969C
:1051A00098AF8FABFD97FAAFE9AF4701FEE18F0EE5
:1051B000911CF801818D928D181619060CF080CF84
:1051C000C8010E945B138333910509F4B2C014F542
:1051D0008130910509F464C044F4892B51F3C8016E
:1051E0000E945B13AC01552775C08330910509F40B
:1051F00062C00697A1F7C8010E945B13B82E44E075
:1052000050E0B401C8010E943C13EB2DE450FF0BA9
:10521000AF0160C08A33910509F45FC084F585331E
:105220009105B1F1C697D9F6C8010E945B135C01E4
:10523000B601CE0189960E94AE7F8BA59CA5ADA537
:10524000BEA5892B8A2B8B2BB1F0EDA9FEA940803E
:10525000518062807380B601CE0183960E94AE7F3A
:105260008DA19EA1AFA1B8A5A501481659066A0651
:105270007B0609F0B8CF44E050E0B60118C08B338C
:10528000910509F440C08F3F910509F492CFA7CF53
:10529000C8010E945B13C8010E945B13382E89CF9E
:1052A000C8010E945B1344E050E06FA978ADC801CB
:1052B0000E943C137ECFC8010E945B13B82E44E0CD
:1052C00050E069AD7AADC8010E943C138B2D84502B
:1052D000990BAC0170E060E0EACFC8010E945B135B
:1052E00044E050E069A97AA9C8010E943C13F70183
:1052F00066A177A180A591A50E940DB366A377A3AF
:1053000080A791A756CFC8010E945B1344E050E0EC
:105310006BA97CA9C8010E943C13F70162A573A583
:1053200084A595A50E940DB362A773A784A795A72E
:1053300040CFC8010E945B1344E050E06FA578A9FC
:10534000C8010E943C13F70162A173A184A195A139
:105350000E940DB362A373A384A395A366A777A746
:1053600080AB91AB26CF33243A94AACE2F923F92B2
:105370004F925F926F927F928F929F92AF92BF9265
:10538000CF92DF92EF92FF920F931F93CF93DF9311
:1053900000D000D0CDB7DEB78C010E9484A72FECDF
:1053A00037E040E050E00E9485B1DC01CB0101967E
:1053B000A11DB11DF80184839583A683B7838083E3
:1053C0009183A283B3835801F3E4AF0EB11CC501EE
:1053D0000E945D1464E470E0C5010E9431178823C7
:1053E00009F445C10E94BC842B013C01480182E4C0
:1053F000880E911C48EEC42E43E0D42EE12CF12CF3
:1054000052E0252E1E821D82D4018C918330B1F191
:10541000811166C0F80184819581A681B7810196CA
:10542000A11DB11D84839583A683B7830E94BC848C
:105430006419750986099709A70196010E9463B14D
:10544000A90161E0C8010E94F11781E0D4018C93A9
:105450008D819E810197C1F20E94BC8464197509F7
:1054600086099709D801D6962D913D914D915C9171
:10547000D997261737074807590720F6C5010E9414
:105480005D14F80184819581A681B7810196A11DE3
:10549000B11D84839583A683B7830E94BC84F801E1
:1054A000FE9660837183828393838D819E8126968D
:1054B0000FB6F894DEBF0FBECDBFDF91CF911F9125
:1054C0000F91FF90EF90DF90CF90BF90AF909F90A3
:1054D0008F907F906F905F904F903F902F900895A6
:1054E0008430F1F4F80184819581A681B781019619
:1054F000A11DB11D84839583A683B7830E94BC84BC
:105500006419750986099709A70196010E9463B17C
:10551000A90163E0C8010E94F117D4012C9298CF31
:10552000813051F5F80142AD53AD64AD75AD9E01CA
:105530002F5F3F4FC8010E941728382EF2E08F13CB
:1055400090C089819A81AB81BC81F8018483958365
:10555000A683B7830E94BC846419750986099709DC
:10556000A70196010E9463B1A90163E0C8010E94EE
:10557000F117D4013C926CCF823009F069CFF80169
:1055800042AD53AD64AD75AD9E012F5F3F4FC80175
:105590000E941728382EF5E08F135DC0E3E0D40198
:1055A000EC93F80182A193A1A4A1B5A1892B8A2B28
:1055B0008B2B41F484E893E0A0E0B0E082A393A3B6
:1055C000A4A3B5A3F80186A197A1A0A5B1A5892B95
:1055D0008A2B8B2B61F482A193A1A4A1B5A1B695CE
:1055E000A7959795879586A397A3A0A7B1A7F8013C
:1055F00082A593A5A4A5B5A5892B8A2B8B2BA9F4ED
:1056000082A193A1A4A1B5A1AC01BD0123E076952F
:105610006795579547952A95D1F7841B950BA60B4F
:10562000B70B82A793A7A4A7B5A7F80186A197A156
:10563000A0A5B1A586A797A7A0ABB1AB82A593A55E
:10564000A4A5B5A582AB93ABA4ABB5AB81E090E0CC
:105650009E838D83FDCE96E0891303C0D4011C92F6
:10566000F7CEBFEF3B12F4CEF4011082F1CE1E82D2
:105670001D821BCF8F929F92AF92BF92EF92FF92AB
:105680000F931F93CF93DF9300D000D0CDB7DEB739
:1056900000914C0C10914D0CF12CE12C01151105D1
:1056A00009F4DAC00E94BC844B015C0178012EE34E
:1056B000E20EF11CF70180819181A281B381A501E5
:1056C0009401281B390B4A0B5B0BCA01B901683ED8
:1056D00033E0730781059105A0F128EE33E040E047
:1056E00050E00E9463B1861A970AA80AB90AD70146
:1056F0008D929D92AD92BC921397F80186A597A5C5
:10570000A0A9B1A949015A01880C991CAA1CBB1C6B
:1057100088159905AA05BB0508F0B0C016A617A6FE
:1057200010AA11AAF80182A993A9A4A9B5A988155C
:105730009905AA05BB0508F0AAC012AA13AA14AAC3
:1057400015AAF80186A597A5A0A9B1A9892B8A2B2E
:105750008B2B09F0A5C0EE5BFF4F8081833009F0F1
:105760009FC084E08083C8010E94B62901967C0115
:10577000F80182A993A9A4A9B5A9892B8A2B8B2BFF
:10578000A1F4EE5BFF4F8081833011F081110DC0D9
:105790001082F8013E9684E1DF011D928A95E9F7B7
:1057A000C8010E94B62903967C01B2E0EB16F10411
:1057B00029F0E4E0EE16F10409F04EC080E591E036
:1057C0000E94247860914C0C70914D0C625F7F4F69
:1057D000CE0101960E94AE7FCE0103960E94111168
:1057E00060914C0C70914D0C6A5E7F4FCE0101961A
:1057F0000E94AE7F44E050E0BE016D5F7F4F81E0CC
:1058000090E00E94B30E60914C0C70914D0C6E5E56
:105810007F4FCE0101960E94AE7F44E050E0BE0172
:105820006D5F7F4F85E090E00E94B30E60914C0C5D
:1058300070914D0C625E7F4FCE0101960E94AE7F4B
:105840008B819C81AD81BE818093190E90931A0E3D
:10585000A0931B0EB0931C0EC70126960FB6F894AA
:10586000DEBF0FBECDBFDF91CF911F910F91FF9093
:10587000EF90BF90AF909F908F900895821B930BF5
:10588000A40BB50B86A797A7A0ABB1AB4BCF821BE0
:10589000930BA40BB50B82AB93ABA4ABB5AB51CFC1
:1058A000F12CE12C65CFEF92FF920F931F93CF93D2
:1058B000DF93CDB7DEB7E8970FB6F894DEBF0FBE23
:1058C000CDBF6DE174E0CE0187960E94467E6DE10A
:1058D00074E0CE018D960E94467E82E0E82EF12C87
:1058E0002496FFAEEEAE249786E0EBEFF2E0DE0109
:1058F000D39601900D928A95E1F786E0FE01F3962A
:10590000DE01AC5BBF4F01900D928A95E1F72C96BA
:105910001FAE1EAE2C9701E010E02E961FAF0EAF0B
:105920002E9788E0E1E0F3E0DE01599601900D92B8
:105930008A95E1F788E0FE017996DE01A25BBF4F10
:1059400001900D928A95E1F788E1E9E0F3E0DE014C
:10595000119601900D928A95E1F788E1FE0131964A
:10596000DE01AA5ABF4F01900D928A95E1F780910E
:10597000210390912203A0912303B0912403E29686
:105980008CAF9DAFAEAFBFAFE29760E874E0CE01E1
:1059900087960E948A7B60E0CE0187960E94FF7CFA
:1059A0004BA55CA5BE016E587F4FCE0187960E9425
:1059B000437964E476E0CE018D960E94327D66EDF7
:1059C00074E08EE591E10E948A7B60E0CE018D96C5
:1059D0000E94FF7C49A95AA9BE0166567F4FCE019D
:1059E0008D960E9443796DE174E0CE0187960E9406
:1059F0008A7B6DE174E0CE018D960E948A7BC25055
:105A0000DF4F19821882CE5FD04080918C02909136
:105A10008D02C050DF4F99838883C050D14080E011
:105A200090E0A0E7B2E4CA5BDE4F88839983AA8343
:105A3000BB83C654D140C65BDE4FF982E882CA54AC
:105A4000D14080E090E0A0E2B2E4C45BDE4F888306
:105A50009983AA83BB83CC54D14080E090E0A4E337
:105A6000B2E4C05BDE4F88839983AA83BB83C055B1
:105A7000D14084EB90E0CC5ADE4F99838883C455A3
:105A8000D14088E790E0CA5ADE4F99838883C65593
:105A9000D1408CE291E0A0E0B0E0C85ADE4F8883AC
:105AA0009983AA83BB83C855D140C45ADE4F19835A
:105AB0000883CC55D140C25ADE4FF982E882CE55D8
:105AC000D14060E080E791E10E94FF7C60E08AE6DF
:105AD00091E10E94FF7C4091741150917511BE01BB
:105AE0006E5F7E4F80E791E10E94437940916E1195
:105AF00050916F11BE01635F7E4F8AE691E10E9473
:105B0000437988E2EEE6FBE0DE01A75EBE4F01903E
:105B10000D928A95E1F78CE390E0A0E0B0E0CE5BD7
:105B2000DE4F88839983AA83BB83C254D140CF5B65
:105B3000DE4F1882C154D14084EE98E3AEE8B2E45F
:105B4000C05ADE4F88839983AA83BB83C056D14055
:105B500084EE98E3AEE8B1E4CC59DE4F88839983B4
:105B6000AA83BB83C456D140C859DE4F198308832A
:105B7000C856D14080E590E0C659DE4F99838883AE
:105B8000CA56D14083E090E0C059DE4F99838883A4
:105B9000C057D14088E390E0CE58DE4F9983888388
:105BA000C257D14084EF91E09093670280936602E0
:105BB000BE016E5B7F4F0E94680964EF71E080E078
:105BC00090E00E94ED816DE276E0CE0181960E9428
:105BD000347ECE0181960E94091BCE0181960E94DF
:105BE000A77DCE018D960E94A77DCE0187960E944B
:105BF000A77DE8960FB6F894DEBF0FBECDBFDF914C
:105C0000CF911F910F91FF90EF9008959F92AF92C7
:105C1000BF92CF92DF92EF92FF920F931F93CF9399
:105C2000DF93CDB7DEB7C859D1090FB6F894DEBF00
:105C30000FBECDBF5C017B016A0166E770E1CE015A
:105C400089579F4F0E94467E68E674E08E010F5F81
:105C50001F4FC8010E94467EB801CE0189579F4F51
:105C60000E94917C982EC8010E94A77D911014C0BB
:105C700068E674E0C8010E94467EBE0169577F4F06
:105C8000C8010E94C27CBC01CE0189579F4F0E946F
:105C9000577DC8010E94A77DB501CE0183579F4F54
:105CA0000E94467E68E874E0E114F10471F066E950
:105CB00074E021E0E216F10441F061EA74E032E0C0
:105CC000E316F10411F069EA74E0CE0189579F4FA1
:105CD0000E94217D60E0CE0189579F4F0E94FF7C8A
:105CE000B601C8010E943D7E6AE0C8010E94137D92
:105CF000BC01CE018D569F4F0E943D7EC8010E947F
:105D0000A77DC557DF4F48815981CB58D040B80196
:105D1000CE0189579F4F0E9443798091510C88236F
:105D200099F161EB74E0CE018F579F4F0E94467E40
:105D3000CE018F579F4F0E94201BCE018F579F4F40
:105D40000E94A77DBE0169577F4FCE018F579F4F9D
:105D50000E943D7ECE018F579F4F0E94201BCE0197
:105D60008F579F4F0E94A77DB801CE018F579F4F3D
:105D70000E94467ECE018F579F4F0E94201BCE016E
:105D80008F579F4F0E94A77DCC56DF4F8881C45903
:105D9000D0408F93CD56DF4F8881C359D0408F9329
:105DA000C257DF4F8881CE58D0408F93C357DF4F03
:105DB0008881CD58D0408F9381EC94E09F938F934E
:105DC0008EECE82E89E0F82EFF92EF920E94BCB58F
:105DD00040913E0250913F026AE97BE08DEF9FE0E7
:105DE0000E94EE150FB6F894DEBF0FBECDBF01972F
:105DF00009F07CC01F930F9387EC94E09F938F93DF
:105E000004ED1AE01F930F930E94BCB5B8018DEF0B
:105E10009FE00E944C7F8AE99BE09F938F9388EDDF
:105E200094E09F938F931F930F930E94BCB5B8018A
:105E30008DEF9FE00E944C7F6EE274E08DEF9FE05B
:105E40000E948A7F67E779E08DEF9FE00E94A77E3E
:105E5000F70101900020E9F7CF018F5C99409F93F3
:105E60008F9381EE94E09F938F931F930F930E94E3
:105E7000BCB5B8018DEF9FE00E944C7FB7018DEF5C
:105E80009FE00E94607F62E370E080E090E00E940B
:105E9000ED818DEF9FE00E94A0150FB6F894DEBF54
:105EA0000FBECDBF11E0CE018D569F4F0E94A77D42
:105EB000CE0183579F4F0E94A77DCE0189579F4FE8
:105EC0000E94A77D812FC856DF4F0FB6F894DEBF22
:105ED0000FBECDBFDF91CF911F910F91FF90EF903B
:105EE000DF90CF90BF90AF909F90089561E774E0EE
:105EF000CE018F579F4F0E94347ECE018F579F4F08
:105F00000E94091BCE018F579F4F0E94A77D6DE70E
:105F100074E0CE018F579F4F0E94347ECE018F5781
:105F20009F4F0E94201BCE018F579F4F0E94A77D3D
:105F30006EEC79E0CE018F579F4F0E94467ECE01D6
:105F40008F579F4F0E94091BCE018F579F4F0E9472
:105F5000A77D10E0A8CFEF92FF920F931F93CF93EE
:105F6000DF93CDB7DEB768970FB6F894DEBF0FBEEC
:105F7000CDBF81E08093F80B0E943A2B8C0160ED3D
:105F800077E080E090E00E94ED818BE0E82EF12C3C
:105F90000D7F0130110571F481E0E81AF10851F02C
:105FA0000E943A2B8C0160ED77E080E090E00E9447
:105FB000ED81EECF0E94AB827C0168EE73E080E061
:105FC00090E00E94ED810BE010E0EF2899F4015081
:105FD000110981F060ED77E080E090E00E94ED81B2
:105FE0000E94AB827C0168EE73E080E090E00E944A
:105FF000ED81EBCF87EB9EE00E94FF181092F80B2B
:106000000E9468276DE174E0CE0107960E94467EEB
:106010006CEA75E0CE010D960E94347ECE01439667
:106020000E94011A888D1F928F938F891F928F93E0
:106030008E891F928F938D891F928F9380E794E0B2
:106040009F938F9384ED9AE09F938F930E94BCB5AA
:1060500064ED7AE0CE0101960E94467EBE016F5F3C
:106060007F4FCE0107960E946E7DCE0101960E9461
:10607000A77DBE01635F7F4FCE0101960E943D7EEA
:10608000CE0101960E94201BCE0101960E94A77DA1
:10609000BE01695F7F4FCE0101960E943D7ECE0119
:1060A00001960E94091BCE0101960E94A77DBE01A8
:1060B000695F7F4FCE0101960E943D7EAE014F5F2A
:1060C0005F4F63E070E080E092E00E94062E182FA0
:1060D000CE0101960E94A77D0FB6F894DEBF0FBED9
:1060E000CDBF11112BC062EA75E0CE0101960E946E
:1060F000347ECE0101960E94201BCE0101960E94A3
:10610000A77DBE01635F7F4FCE0101960E943D7E59
:10611000CE0101960E94201BCE0101960E94A77D10
:106120006AEC7FE0CE0101960E943D7ECE01019691
:106130000E94091BCE0101960E94A77DCE010D96FB
:106140000E94A77DCE0107960E94A77D68960FB694
:10615000F894DEBF0FBECDBFDF91CF911F910F919D
:10616000FF90EF9008957F928F929F92AF92BF928F
:10617000CF92DF92EF92FF920F931F93CF93DF9313
:10618000CDB7DEB762970FB6F894DEBF0FBECDBFB6
:106190006FE875E0CE0101960E94347ECE01019633
:1061A0000E94091BCE0101960E94A77D04E010E029
:1061B00030EAC32E3AE0D32E40E3E42E53EEB52E60
:1061C00066E0A62E7CEE972EE1E3FE2EFEE48F2EF7
:1061D000A4E37A2E68EB72E28DE99FE00E9431170A
:1061E000F6018E2D11928A95E9F7B092A00AA0923D
:1061F000A20A9092A30AF092AC0A8092AD0AF092A1
:10620000AE0A7092AF0A60E472E0CE0101960E947D
:10621000AE7F4BE750E0BE016F5F7F4F8DE99FE09F
:106220000E94BA1740E350E060EA7AE08DE99FE00F
:106230000E944F178DE99FE00E94891768EE73E076
:1062400080E090E00E94ED818DE99FE00E9485133F
:10625000892B09F04FC00150110909F07CC08091D1
:10626000D00A9091D10AA091D20AB091D30A892B79
:106270008A2B8B2B09F089C06DE174E088EE9FE0DA
:106280000E948A7B68EE7FE0CE0101960E943D7EEF
:10629000AE014F5F5F4F70E060E082E792E00E94E6
:1062A000062E182FCE0101960E94A77D11110EC057
:1062B00067E775E0CE0101960E94347ECE0101961B
:1062C0000E94091BCE0101960E94A77D62960FB61F
:1062D000F894DEBF0FBECDBFDF91CF911F910F911C
:1062E000FF90EF90DF90CF90BF90AF909F908F90F6
:1062F0007F90089540E350E060EA7AE08DE99FE006
:106300000E943C136091C80A7091C90A76276727DA
:10631000762790E080E0CB01772766270091CA0AB4
:106320001091CB0A10270127102730E020E0602BC6
:10633000712B822B932B7E508A4A93480E94EF88C0
:106340000E9414896093D00A7093D10A8093D20A74
:106350009093D30A84CF68EE73E080E090E00E94CF
:10636000ED814091D00A5091D10A6091D20A70918A
:10637000D30A2AE085E29DE00E94B67E67E779E0D5
:1063800085E29DE00E94A77E25CF68EE73E080E065
:1063900090E00E94ED810E9414896093EF0B70934E
:1063A000F00B8093F10B9093F20B0E941489609391
:1063B000E90B7093EA0B8093EB0B9093EC0BCE01FF
:1063C00001960E942222CE0101960E94091BCE0155
:1063D00001960E94A77D0E94AE8ABC01CE0107965D
:1063E0000E94CB1E6EE374E0CE0107960E94217DD1
:1063F0000E94A68ABC01CE0101960E94CB1EBE015E
:106400006F5F7F4FCE0107960E942B7DCE010196D4
:106410000E94A77D6EE374E0CE0107960E94217D65
:106420000E949C8ABC01CE0101960E94CB1EBE0137
:106430006F5F7F4FCE0107960E942B7DCE010196A4
:106440000E94A77D66EF74E0CE0101960E94467E11
:10645000BE01695F7F4FCE0101960E94C27CBC01E4
:10646000CE010D960E943D7E4AE050E06FEF7FEF37
:10647000CE010D960E94D226CE010D960E94A77DD8
:10648000CE0101960E94A77DCE0107960E94A77DAE
:1064900068EE73E080E090E00E94ED810E94BE8A89
:1064A000BC01CE010D960E94CB1E0E94B68ABC0193
:1064B000CE0101960E94CB1E64E077E0CE010796E4
:1064C0000E94467EBE016F5F7F4FCE0107960E94FD
:1064D000C27CBC01CE010D960E942B7DCE01079699
:1064E0000E94A77DCE0101960E94A77D0E9414897B
:1064F0000E94A3896091D20B70E0CE0101960E94A8
:10650000CB1E64E077E0CE0107960E94467EBE0176
:106510006F5F7F4FCE0107960E94C27CBC01CE0107
:106520000D960E942B7DCE0107960E94A77DCE017D
:1065300001960E94A77D6CEF74E0CE0101960E9447
:10654000467EBE01635F7F4FCE0101960E94C27CF2
:10655000BC01CE0107960E943D7E4AE050E06FEFFD
:106560007FEFCE0107960E94D226CE0107960E94A9
:10657000A77DCE0101960E94A77DCE010D960E94B7
:10658000A77D68EE73E080E090E00E94ED81CE018F
:1065900001960E94A1214AE050E06FEF7FEFCE010B
:1065A00001960E94D2268ECECF92DF92EF92FF927A
:1065B0000F931F93CF93DF93CDB7DEB768970FB6D6
:1065C000F894DEBF0FBECDBF6DE174E0CE014396FF
:1065D0000E94467E61E877E0CE0101960E94347EFB
:1065E000CE0101960E94201BCE0101960E94A77D3C
:1065F0006AE671E1CE0101960E943D7ECE010196D0
:106600000E94091BCE0101960E94A77D61E777E0F9
:10661000CE0101960E94347ECE0101960E94201B7D
:10662000CE0101960E94A77D6CA17DA1CE010196AD
:106630000E94947BCE0101960E94091BCE01019617
:106640000E94A77D69E577E0CE0101960E94347E25
:10665000CE0101960E94201BCE0101960E94A77DCB
:10666000CE5ADE4F68817981C255D140CE01019664
:106670000E94947BCE0101960E94091BCE010196D7
:106680000E94A77D6CE477E0CE0101960E94347EE3
:10669000CE0101960E94201BCE0101960E94A77D8B
:1066A0000AEA1BE0EE24E394F12CCE5ADE4F8881F7
:1066B0009981C255D1408E159F050CF44AC0F8014E
:1066C00082819381C6979CF162E075E0CE010196CC
:1066D0000E94467ECE0101960E94201BCE010196AB
:1066E0000E94A77DF8016281738166537109CE0112
:1066F00001960E94947BCE0101960E94201BCE0140
:1067000001960E94A77D64E476E0CE0101960E9486
:10671000467ECE0101960E94201BCE0101960E946A
:10672000A77DFFEFEF1AFF0A0E5F1F4FBECF61EC90
:1067300076E0CE0101960E94467ECE0101960E942F
:10674000201BCE0101960E94A77DF8016281738112
:10675000CECF64E476E0CE0101960E94467ECE0163
:1067600001960E94091BCE0101960E94A77D6DE350
:1067700077E0CE0101960E94347ECE0101960E9400
:10678000201BCE0101960E94A77D6091690B70913C
:106790006A0BCE0101960E94947BCE0101960E9465
:1067A000201BCE0101960E94A77D64E476E0CE0115
:1067B00001960E94467ECE0101960E94201BCE01CA
:1067C00001960E94A77D60916B0B70916C0BCE01BE
:1067D00001960E94947BCE0101960E94091BCE0176
:1067E00001960E94A77D66E277E0CE0101960E94A5
:1067F000347ECE0101960E94201BCE0101960E949C
:10680000A77DBE01605D7F4FCE0101960E94467E4E
:10681000CE0101960E94201BCE0101960E94A77D09
:1068200064E476E0CE0101960E94467ECE01019698
:106830000E94201BCE0101960E94A77DBE016C5CC8
:106840007F4FCE0101960E94467ECE0101960E94A6
:10685000091BCE0101960E94A77D66E177E0CE017B
:1068600001960E94347ECE0101960E94091BCE0142
:1068700001960E94A77D8E010C5D1F4FEE24E394CC
:10688000F12C680188E0C80ED11C8CA19DA18E1549
:106890009F050CF449C0B701CE0107960E94947B76
:1068A00068EC77E0CE0101960E94467EBE01695FEA
:1068B0007F4FCE0101960E94C27CBC01CE010D9695
:1068C0000E943D7ECE010D960E94201BCE010D96AA
:1068D0000E94A77DCE0101960E94A77DCE0107965A
:1068E0000E94A77D64E077E0CE0101960E94467E7B
:1068F000CE0101960E94201BCE0101960E94A77D29
:10690000B801645E7F4FCE0101960E94467ECE01A3
:1069100001960E94091BCE0101960E94A77DEFEF10
:10692000EE1AFE0A8601ADCF65E077E0CE01019652
:106930000E94347ECE0101960E94201BCE0101965A
:106940000E94A77D7E01F2EBEF1AFEEFFF0A10E036
:1069500000E0F70161917F0170E0CE0101960E9495
:10696000947BCE0101960E94201BCE0101960E94CD
:10697000A77D0330110571F064E075E0CE0101964A
:106980000E94467ECE0101960E94201BCE010196F8
:106990000E94A77D0F5F1F4F04301105D1F664E4FC
:1069A00076E0CE0101960E94467ECE0101960E94BD
:1069B000091BCE0101960E94A77DC45BDE4F688152
:1069C0007981CC54D140072E000C880B990B0E9482
:1069D00020B09B01AC010E94E0B2882341F080E529
:1069E00090E0C45BDE4F99838883CC54D140C45B74
:1069F000DE4F88819981CC54D14090933F0280939F
:106A00003E026BEE76E0CE0101960E94347ECE010E
:106A100001960E94201BCE0101960E94A77D6AE983
:106A20007BE0CE0101960E94467ECE0101960E9437
:106A3000201BCE0101960E94A77D69EE76E0CE0173
:106A400001960E94347ECE0101960E94201BCE0149
:106A500001960E94A77D60913E0270913F02CE0197
:106A600001960E94947BCE0101960E94091BCE01E3
:106A700001960E94A77D6AED76E0CE0101960E9404
:106A8000347ECE0101960E94201BCE0101960E9409
:106A9000A77DBE016C5A7F4FCE0101960E94467EB3
:106AA000CE0101960E94091BCE0101960E94A77D8E
:106AB00066E075E0CE0101960E94467ECE01019609
:106AC0000E94201BCE0101960E94A77DBE01645842
:106AD0007F4FCE0101960E94467ECE0101960E9414
:106AE000091BCE0101960E94A77DC052DF4F88810D
:106AF0009981C05ED040892B71F462ED76E0CE01C1
:106B000001960E94347ECE0101960E94091BCE019F
:106B100001960E94A77DC052DF4F88819981C05E97
:106B2000D040019771F468EC76E0CE0101960E94A6
:106B3000347ECE0101960E94091BCE0101960E946F
:106B4000A77DC052DF4F88819981C05ED0400297F7
:106B500071F46FEB76E0CE0101960E94347ECE0197
:106B600001960E94091BCE0101960E94A77D69EB48
:106B700076E0CE0101960E94347ECE0101960E94FD
:106B8000201BCE0101960E94A77DCE51DF4F688168
:106B90007981C25ED040CE0101960E94947BCE01E5
:106BA00001960E94091BCE0101960E94A77D60EB11
:106BB00076E0CE0101960E94347ECE0101960E94BD
:106BC000201BCE0101960E94A77DCC5ADE4F888102
:106BD0009981C455D140C6970CF41FC162E075E09D
:106BE000CE0101960E94467ECE0101960E94201B96
:106BF000CE0101960E94A77DCC5ADE4F6881798133
:106C0000C455D14066537109CE0101960E94947B10
:106C1000CE0101960E94091BCE0101960E94A77D1C
:106C20004091E10B5091E20B6091E30B7091E40B0A
:106C300021E0CE0107960E94AF7D61E175E0CE01B3
:106C400001960E94467EBE01695F7F4FCE0101968C
:106C50000E94C27C6CE175E00E94AC7CBC01CE015C
:106C60000D960E943D7ECE010D960E94091BCE011D
:106C70000D960E94A77DCE0101960E94A77DCE01B0
:106C800007960E94A77D4091DD0B5091DE0B60912D
:106C9000DF0B7091E00B21E0CE0107960E94AF7DE3
:106CA00061E275E0CE0101960E94467EBE01695FF9
:106CB0007F4FCE0101960E94C27C6CE175E00E947C
:106CC000AC7CBC01CE010D960E943D7ECE010D969E
:106CD0000E94091BCE010D960E94A77DCE01019650
:106CE0000E94A77DCE0107960E94A77D62E976E00B
:106CF000CE0101960E94347ECE0101960E94201B97
:106D0000CE0101960E94A77D4091290250912A024E
:106D100060912B0270912C0225E0CE0101960E9419
:106D2000AF7DCE0101960E94091BCE0101960E9403
:106D3000A77D68E776E0CE0101960E94347ECE0101
:106D400001960E94201BCE0101960E94A77D4091D2
:106D5000250250912602609127027091280225E0B9
:106D6000CE0101960E94AF7DCE0101960E94091BC3
:106D7000CE0101960E94A77D68E676E0CE010196DD
:106D80000E94347ECE0101960E94201BCE01019606
:106D90000E94A77D60916C0270916D02CE010196F8
:106DA0000E94947BCE0101960E94091BCE010196A0
:106DB0000E94A77D66E576E0CE0101960E94347EB2
:106DC000CE0101960E94201BCE0101960E94A77D54
:106DD000C65BDE4F68817981CA54D140CE010196ED
:106DE0000E94947BCE0101960E94091BCE01019660
:106DF0000E94A77DCE0143960E94A77D68960FB69C
:106E0000F894DEBF0FBECDBFDF91CF911F910F91E0
:106E1000FF90EF90DF90CF90089561EC76E0CE0187
:106E200001960E94467ECE0101960E94201BCE0153
:106E300001960E94A77DCC5ADE4F68817981C455A6
:106E4000D140E2CE2F923F924F925F926F927F920B
:106E50008F929F92AF92BF92CF92DF92EF92FF926A
:106E60000F931F93CF93DF93CDB7DEB7EC970FB699
:106E7000F894DEBF0FBECDBF3C018B0170E060E037
:106E80000E94607C8F8F6DE174E0CE0149960E9474
:106E9000467E80916C0290916D02019709F07AC054
:106EA00082E090E00E945A8988E090E0909324026A
:106EB0008093230289E090E0909322028093210244
:106EC0008091670B9091680B9093660B8093650B94
:106ED00080911D0290911E02A0911F02B09120028C
:106EE0008093190290931A02A0931B02B0931C0284
:106EF0008091350290913602A0913702B09138020C
:106F00008093390290933A02A0933B02B0933C02E3
:106F10008091640B8093630B80915F0B9091600B69
:106F2000A091610BB091620B80935B0B90935C0B13
:106F3000A0935D0BB0935E0B8AE390E090931802F0
:106F4000809317028091E10B9091E20BA091E30BEB
:106F5000B091E40B8093960B9093970BA093980BB2
:106F6000B093990B809115029091160290931402A0
:106F7000809313028091290290912A02A0912B0202
:106F8000B0912C0280932D0290932E02A0932F0299
:106F9000B093300280916C0290916D02029709F0DB
:106FA0007AC083E090E00E945A898AE090E0909352
:106FB0002402809323028BE090E09093220280933E
:106FC00021028091590B90915A0B9093660B8093FC
:106FD000650B80910F0290911002A0911102B09167
:106FE00012028093190290931A02A0931B02B0938D
:106FF0001C028091310290913202A0913302B09133
:1070000034028093390290933A02A0933B02B093EA
:107010003C028091580B8093630B8091540B9091AC
:10702000550BA091560BB091570B80935B0B90932F
:107030005C0BA0935D0BB0935E0B8BE390E09093A1
:107040001802809317028091DD0B9091DE0BA091C6
:10705000DF0BB091E00B8093960B9093970BA0936E
:10706000980BB093990B80910D0290910E02909322
:107070001402809313028091250290912602A09120
:107080002702B091280280932D0290932E02A093A4
:107090002F02B09330022F8D2335C1F41092660B6E
:1070A0001092650B80916D0B882371F068E275E09A
:1070B000CE0101960E94467ECE0101960E94091BD8
:1070C000CE0101960E94A77DE12CFCC0C80101976A
:1070D000029708F038C281E090E0A0E0B0E0809331
:1070E000190290931A02A0931B02B0931C02D301C1
:1070F00014968D919C91029748F141E050E0B301C4
:10710000CE0101960E94BF1EBE016F5F7F4FCE0170
:1071100049960E946E7DCE0101960E94A77DCE0108
:1071200049960130110581F50E94ED7B20E030E0A9
:1071300040E251E40E947FB00E94A5B26093190220
:1071400070931A0280931B0290931C02BF8D81E002
:1071500090E09093660B8093650BB13401F58091BC
:107160006D0B882309F4B0CF6DE275E0CE01019676
:107170000E94467ECE0101960E94091BCE01019617
:107180000E94A77DE12C6BC00E94ED7B20912D0217
:1071900030912E0240912F0250913002CBCFEF8DD3
:1071A000E63409F075C160E0809121020E947A8086
:1071B00064E670E080E090E00E94ED8161E0809103
:1071C00023020E947A8064E670E080E090E00E94F2
:1071D000ED8160E0809121020E947A8064E670E097
:1071E00080E090E00E94ED8161E0809123020E94A6
:1071F0007A8064E670E080E090E00E94ED810230E9
:107200001105C1F4CE0149960E94ED7B9B01AC01B2
:107210006091960B7091970B8091980B9091990BC0
:107220000E94C6B16093960B7093970B8093980B56
:107230009093990B80916D0B882371F066E375E054
:10724000CE0101960E94467ECE0101960E94201B2F
:10725000CE0101960E94A77DEE24E394F12C80914B
:107260006D0B882379F14091190250911A026091B7
:107270001B0270911C022AE0CE0101960E94E57D5E
:10728000BE016F5F7F4FCE0107960E943D7E6AE48C
:1072900075E0CE0107960E94AC7CBC01CE010D9634
:1072A0000E943D7ECE010D960E94091BCE010D96D7
:1072B0000E94A77DCE0107960E94A77DCE01019670
:1072C0000E94A77D8091190290911A02A0911B0241
:1072D000B0911C02181619061A061B060CF0E7C519
:1072E0003F8D363409F4EFC4323509F4F0C460E060
:1072F000809121020E947A8064E670E080E090E054
:107300000E94ED816E2D809123020E947A8064E6B6
:1073100070E080E090E00E94ED816091650B8091CB
:1073200021020E947A8061E070E080E090E00E949B
:10733000ED8160E0809121020E947A8068EC70E02B
:1073400080E090E00E94ED81C12CD12C7601C394A5
:107350008091190290911A02A0911B02B0911C0217
:10736000C816D906EA06FB060CF0B3C46091650B9B
:10737000809121020E947A8061E070E080E090E0DC
:107380000E94ED8160E0809121020E947A806091EC
:10739000390270913A0280913B0290913C020E9426
:1073A000ED818091390290913A02A0913B02B09117
:1073B0003C020B97A105B1050CF464C060912D024D
:1073C00070912E0280912F02909130029B01AC01AE
:1073D0000E94C7B10E94A5B29B01AC01C701B601D2
:1073E0000E9485B1672B682B692B09F04BC00230D6
:1073F00011050CF447C069EB75E089E79FE00E9436
:10740000327DC701B6010E9420B020912D0230913B
:107410002E0240912F02509130020E9433B2AB01F4
:10742000BC0120E0CE0107960E94AF7D69E77FE0B6
:10743000CE0101960E943D7EBE01695F7F4FCE0165
:1074400001960E94C27C6CE175E00E94AC7CBC019C
:1074500089E79FE00E94577DCE0101960E94A77D9B
:10746000CE0107960E94A77D69E77FE0CE010196D5
:107470000E943D7ECE0101960E94A727CE01019673
:107480000E94A77D4FEFC41AD40AE40AF40A60CF21
:10749000FF8DF23509F076CE60E0809121020E94E6
:1074A0007A8064E670E080E090E00E94ED8160E028
:1074B000809123020E947A8064E670E080E090E090
:1074C0000E94ED8160E0809121020E947A8064E652
:1074D00070E080E090E00E94ED8160E08091230206
:1074E0000E947A8064E670E080E090E00E94ED8186
:1074F00002301105C1F4CE0149960E94ED7B9B013B
:10750000AC016091960B7091970B8091980B9091C4
:10751000990B0E94C7B16093960B7093970B809361
:10752000980B9093990B80916D0B882309F4CCCD27
:1075300060E475E0CE0101960E94467ECE01019680
:107540000E94201B1BCE0115110521F003301105EF
:1075500009F0BACD80916C0290916D0220E137E282
:1075600040E050E08130910521F420E43CE940E026
:1075700050E02EA73FA748AB59AB21E030E0309355
:10758000660B2093650B30935D0220935C0202979B
:1075900059F40330110541F4809144119091451143
:1075A00090935D0280935C0240915C0250915D0279
:1075B0005DA74CA7551F5527551F5AAB81E090E09A
:1075C00090935D0280935C0260E0809121020E94B2
:1075D0007A8064E670E080E090E00E94ED816AA924
:1075E000809123020E947A8064E670E080E090E05F
:1075F0000E94ED8160E0809121020E947A8064E621
:1076000070E080E090E00E94ED816AA98091230201
:107610000E947A8064E670E080E090E00E94ED8154
:107620008FEF9FEF9093140280931302812C912C83
:10763000540118A619A61AA61BA61CA21DA21EA2BA
:107640001FA218A219A21AA21BA2212C312C2101BF
:107650001FAA18AE19AE1AAE1BAA1CAA1DAA1EAAF2
:1076600061E0809121020E947A8061E070E080E018
:1076700090E00E94ED8160E0809121020E947A807A
:1076800061E070E080E090E00E94ED81C501B4010E
:1076900026E030E040E050E00E9485B1672B682B87
:1076A000692B09F0F8C0A2E0B0E0BCAFABAFC12CD1
:1076B000D12C760180911702863308F086532091F1
:1076C0007B00982F9870277F922B90937B00877078
:1076D000806480937C0080917A00806480937A003B
:1076E00080917A0086FDFCCF8091780060917900CE
:1076F000762F682F072E000C880B990B0E9420B064
:107700009B01AC01C701B6010E94C7B16B017C01AE
:1077100062E070E080E090E00E94ED812BAD3CAD36
:107720002130310509F0ADC020E030EC4FEF54E4DA
:10773000C701B6010E9433B26B017C0180916D0BD1
:10774000882399F12DEC3CEC4CE45EE3C701B601D3
:107750000E94DBB287FD29C022E0B701A601CE015D
:1077600007960E94AF7D61E575E0CE0101960E940B
:10777000467EBE01695F7F4FCE0101960E94C27CAA
:10778000BC01CE010D960E943D7ECE010D960E9459
:10779000091BCE010D960E94A77DCE0101960E9485
:1077A000A77DCE0107960E94A77D2AE939E949E91C
:1077B0005EE3C701B6010E94DBB287FD13C021144E
:1077C00031044104510411F4140125018CA19DA13F
:1077D000AEA1BFA1892B8A2B8B2B21F48CA29DA259
:1077E000AEA2BFA22DEC3CEC4CE45EE3C701B601B7
:1077F0000E9419B018160CF449C021143104410438
:10780000510409F448C028A139A14AA15BA1232B46
:10781000242B252B69F488A599A5AAA5BBA5892B9E
:107820008A2B8B2B09F401C188A299A2AAA2BBA220
:1078300028A139A14AA15BA12216330644065506A8
:1078400054F5809113029091140297FFF3C01092A7
:10785000140210921302220E331E441E551ED20132
:10786000C101B595A795979587958FAB98AFA9AFAF
:10787000BAAF18A219A21AA21BA2212C312C2101E5
:107880000AC0E1E0F0E0FCAFEBAF14CF211431040B
:107890004104510469F6E0901302F090140292E062
:1078A000E916F10434F4F7FCE1C00330110509F0E6
:1078B000DDC08EA49FA4A8A8B9A8AAE08A0E911C36
:1078C000A11CB11C8EA59FA5A8A9B9A988169906C7
:1078D000AA06BB060CF4C4CEE2E0EE16F1040CF4EA
:1078E00079C06BA97CA98DA99EA92FA938AD49ADF6
:1078F0005AAD621B730B840B950B0E9420B04B0199
:107900005C01B701FF0C880B990B0E9420B09B0112
:10791000AC01C501B4010E9433B220E030E044EB79
:1079200053E40E9433B26B017C01C0922D02D092CD
:107930002E02E0922F02F092300220E030E040E888
:107940005FE30E94DBB287FDABC080916C02909137
:107950006D028130910509F08FC0C0923C11D09228
:107960003D11E0923E11F0923F11C0922902D09257
:107970002A02E0922B02F0922C026CED75E0CE010F
:1079800001960E94347ECE0101960E94201BCE01FA
:1079900001960E94A77D40912D0250912E02609188
:1079A0002F027091300225E0CE0101960E94AF7D3A
:1079B000CE0101960E94091BCE0101960E94A77D6F
:1079C00084EF91E090936702809366026EE170E12C
:1079D0000E9468090330110531F03AA9E32E011520
:1079E000110509F06FCCC3010E94ED7B6B017C0196
:1079F000C092960BD092970BE092980BF092990B55
:107A000020E030E044EB53E4C701B6010E94DBB252
:107A100087FD6AC020E030E044EB53E4C701B601C3
:107A20000E94C6B16B017C01EBCF88A699A6AAA6DD
:107A3000BBA6FACE0115110509F02DCF0196909342
:107A400014028093130228A139A14AA15BA1220E3E
:107A5000331E441E551ED201C101B595A7959795B9
:107A600087958BAB9CABADABBEAB03CFBFEF8B1A97
:107A70009B0AAB0ABB0A26CF029709F07ECFC092C1
:107A80004011D0924111E0924211F0924311C09204
:107A90002502D0922602E0922702F09228026DCFB2
:107AA00060EC75E0CE0101960E94347ECE01019615
:107AB0000E94201BCE0101960E94A77D40912D02BD
:107AC00050912E0260912F027091300225E0CE017C
:107AD00001960E94AF7DCE0101960E94091BCE0146
:107AE00001960E94A77D76CF20E030E0A901C70172
:107AF000B6010E9419B087FF0BC020E030E044EBD4
:107B000053E4C701B6010E94C7B16B017C01ECCF01
:107B1000C0925B0BD0925C0BE0925D0BF0925E0B1F
:107B200048A459A46AA47BA48CA19DA1AEA1BFA125
:107B3000481A590A6A0A7B0A01151105D9F41092EC
:107B40005B0B10925C0B10925D0B10925E0BACA560
:107B5000BDA5C12CD12C7601C394812C912C54014C
:107B6000B7FF1CC0812C912C5401CC24CA94DC2C6E
:107B7000760114C0ECA5FDA5C12CD12C7601C394CF
:107B8000F7FF04C0CC24CA94DC2C760180905B0BF8
:107B900090905C0BA0905D0BB0905E0B20912D023D
:107BA00030912E0240912F0250913002C501B40154
:107BB0000E947FB04B015C01A3019201C701B60195
:107BC0000E9453B10E9420B020E030E040E05FE32B
:107BD0000E947FB09B01AC01C501B4010E94C6B1F7
:107BE0000E94A5B26093190270931A0280931B023F
:107BF00090931C0280916D0B882309F441C02AE008
:107C000048A559A56AA57BA5CE010D960E94E57DE4
:107C10002AE04CA15DA16EA17FA1CE0107960E9432
:107C2000E57D68E575E0CE0101960E94467EBE01C5
:107C3000695F7F4FCE0101960E94C27C64E476E0CA
:107C40000E94AC7CBE01635F7F4F0E94C27CBC017E
:107C5000CE0143960E943D7ECE0143960E94091BB1
:107C6000CE0143960E94A77DCE0101960E94A77D7A
:107C7000CE0107960E94A77DCE010D960E94A77D9A
:107C80008091190290911A02A0911B02B0911C02DE
:107C9000B7FF15C0B095A095909581959F4FAF4FB8
:107CA000BF4F8093190290931A02A0931B02B093C6
:107CB0001C02EE24E394F12CF6E4FF8F03CBE12CBD
:107CC00022E52F8FFFCAEE24E394F12C10CBE12C98
:107CD0000ECB0230110524F40115110509F0DFC0A7
:107CE00061E080E00E94D88C0230110524F4011577
:107CF000110509F09CC0C090960BD090970BE090B6
:107D0000980BF090990B20E030E044EB53E4C7016E
:107D1000B6010E94DBB287FD0BC020E030E044EBEF
:107D200053E4C701B6010E94C6B16B017C01EBCFE1
:107D300020E030E0A901C701B6010E9419B087FF19
:107D40000BC020E030E044EB53E4C701B6010E94D1
:107D5000C7B16B017C01ECCFC092960BD092970B10
:107D6000E092980BF092990B80916C0290916D02C9
:107D70000197B1F461E175E089E79FE00E948A7B99
:107D80008091960B9091970BA091980BB091990BC5
:107D90008093E10B9093E20BA093E30BB093E40B81
:107DA00080916C0290916D020297B1F461E275E0EE
:107DB00089E79FE00E948A7B8091960B9091970BB8
:107DC000A091980BB091990B8093DD0B9093DE0BF3
:107DD000A093DF0BB093E00B4091960B5091970B63
:107DE0006091980B7091990B20E0CE0107960E944C
:107DF000AF7D69E77FE0CE0101960E943D7EBE0126
:107E0000695F7F4FCE0101960E94C27C6DE175E0F3
:107E10000E94AC7CBC0189E79FE00E94577DCE01A7
:107E200001960E94A77DCE0107960E94A77D013092
:107E3000110539F54091190250911A0260911B0207
:107E400070911C0221E0CE0107960E94E57D60E65C
:107E500075E0CE0101960E94467EBE01695F7F4FAC
:107E6000CE0101960E94C27CBC0189E79FE00E947E
:107E7000577DCE0101960E94A77DCE0107960E94F4
:107E8000A77D69E77FE0CE0101960E943D7ECE018D
:107E900001960E94A727CE0101960E94A77D10920D
:107EA000190210921A0210921B0210921C02809169
:107EB0006C0290916D028130910509F083C0809130
:107EC000650B9091660B9093680B8093670B809184
:107ED000190290911A02A0911B02B0911C0280938A
:107EE0001D0290931E02A0931F02B0932002809166
:107EF000390290913A02A0913B02B0913C028093EA
:107F0000350290933602A0933702B09338028091E5
:107F1000630B8093640B80915B0B90915C0BA09141
:107F20005D0BB0915E0B80935F0B9093600BA09301
:107F3000610BB093620B8091960B9091970BA0917F
:107F4000980BB091990B8093E10B9093E20BA09367
:107F5000E30BB093E40B8091130290911402909381
:107F6000160280931502012B81F480912D029091CD
:107F70002E02A0912F02B09130028093290290939B
:107F80002A02A0932B02B0932C02CE0149960E94A4
:107F9000A77DEC960FB6F894DEBF0FBECDBFDF9184
:107FA000CF911F910F91FF90EF90DF90CF90BF90F6
:107FB000AF909F908F907F906F905F904F903F9089
:107FC0002F900895029709F78091650B9091660BA9
:107FD00090935A0B8093590B8091190290911A0239
:107FE000A0911B02B0911C0280930F02909310028B
:107FF000A0931102B09312028091390290913A023B
:10800000A0913B02B0913C028093310290933202E6
:10801000A0933302B09334028091630B8093580B8A
:1080200080915B0B90915C0BA0915D0BB0915E0B0E
:108030008093540B9093550BA093560BB093570B12
:108040008091960B9091970BA091980BB091990B02
:108050008093DD0B9093DE0BA093DF0BB093E00BCE
:10806000809113029091140290930E0280930D025E
:10807000012B09F08ACF80912D0290912E02A091C0
:108080002F02B09130028093250290932602A09394
:108090002702B093280279CF6F927F928F929F929E
:1080A000AF92BF92CF92DF92EF92FF920F931F9306
:1080B000CF93DF93CDB7DEB7C456D1090FB6F8948E
:1080C000DEBF0FBECDBF40E052EC61E070E085E264
:1080D0009DE00E94277840E855E260E070E088E883
:1080E0009CE00E94277861E088E00E94978161E02F
:1080F00089E00E94978160E08AE30E94978161E0B5
:1081000088E00E947A8060E089E00E947A8061E0E5
:108110008AE00E94978161E08BE00E94978160E095
:108120008BE30E94978161E08AE00E947A8060E0A0
:108130008BE00E947A800E94808184EF91E090938E
:1081400067028093660265EF7AE085E29DE00E9417
:108150008A7F67E779E085E29DE00E94A77E60ED77
:1081600077E080E090E00E94ED8185E29DE00E9452
:10817000DD74982E0EE110E091100BC085E29DE0B9
:108180000E94DD74982E6EE170E080E090E00E9425
:10819000ED810150110981F780916602909167028B
:1081A000A0E5AA2EA1E1BA2EBEE1EB2EB0E1FB2E96
:1081B0009C012E5130416901C6018E0D9F1D0E9408
:1081C0003DB1F70181937F01AE16BF06A9F760911B
:1081D000381170913911072E000C880B990B0E94F1
:1081E00020B09B01AC010E94E0B2882331F081E015
:1081F00090E0909339118093381160913A11709109
:108200003B11072E000C880B990B0E9420B09B019C
:10821000AC010E94E0B2882331F082E090E09093BC
:108220003B1180933A11F5E79F16B1F0609134113C
:108230007091351180913611909137110E9420B0C4
:108240009B01AC010E94E0B2811106C080911E101A
:1082500090911F108197E8F02DB73EB7225331401F
:108260000FB6F8943EBF0FBE2DBFADB7BEB7119687
:1082700082E391E0EEE1F0E101900D920197E1F7E8
:108280000E94532C0FB6F894DEBF0FBECDBFF5E7AA
:108290009F2EEDB7FEB7E253F1400FB6F894FEBF44
:1082A0000FBEEDBFADB7BEB7119682E391E0EEE130
:1082B000F0E101900D920197E1F70E9459240FB669
:1082C000F894DEBF0FBECDBF35E7931619F083E7F4
:1082D00098121BC0EDB7FEB7E253F1400FB6F89409
:1082E000FEBF0FBEEDBFADB7BEB7119682E391E002
:1082F000EEE1F0E101900D920197E1F70E94D43296
:108300000FB6F894DEBF0FBECDBF63EE7AE080ED0E
:108310009FE00E94327D6DEC7AE08AEC9FE00E9443
:10832000327D0E948081E7E2CE2ED12CE12CF12C0F
:10833000B12CA12C882483948092830CC092850C4C
:108340001092840C1092860C81E00E94938B811114
:10835000B0C1C092D8113FEFA31AB30A8FEFC81A69
:10836000D80AE80AF80A90E4C916D104E104F10435
:1083700019F7AB2831F462E875E085E29DE00E94D0
:108380004C7F0E9480811092D9118091DD11823042
:1083900018F098E09093D9119091DE11992339F05B
:1083A000813029F48091D91184608093D91162E3DE
:1083B00070E080E090E00E94ED816091DF1184ED3B
:1083C00091E10E94838C68EE73E080E090E00E946F
:1083D000ED8160E384ED91E10E94978C5BE4E52EF2
:1083E00056E4F52EC7010197F1F760E384ED91E1C2
:1083F0000E94978CC7010197F1F760E384ED91E14A
:108400000E94978C83E592E00197F1F760E284ED9A
:1084100091E10E94978C8091D91180620E94C78C53
:1084200084E08093DA118CE00E94C78C81E00E9486
:10843000C78C6BE3E62E6FE1F62EC7010197F1F7CB
:1084400082E08093DB1186E00E94C78C82E00E946C
:10845000C78CC7010197F1F780E40E94C78C7EE5C5
:10846000E72E72E0F72EF70161917F0184ED91E133
:108470000E94B08CF6E6EF16F2E0FF06A1F70E942C
:108480001A0A0E940A0A64E670E080E090E00E9406
:10849000ED8165EB7AE0CE0101960E94347ECE013B
:1084A00001960E94091BCE0101960E94A77D61E002
:1084B00085E30E94978161E085E30E947A8061E014
:1084C0008AE00E94978161E08AE00E947A8061E000
:1084D00089E30E9497818091B00E803308F050C0EC
:1084E00061E089E30E9497818091B00E282F30E0EF
:1084F000F901EE0FFF1FE20FF31FE35EF14F9081D2
:10850000907C996390831092B10E1092B20E2CE081
:10851000622F0E94E5B2829FB00111249B01200FBF
:10852000311FF901EE0FFF1FE20FF31FE35EF14F62
:10853000908196FD17C00F5F1F4F0C30110571F72A
:10854000813009F0CDC01092800082E080938100DC
:108550001092850010928400B19A80916F00826021
:1085600080936F00E091B00E8E2F90E0FC01EE0F33
:10857000FF1FE80FF91FE35EF14F80818064808365
:1085800068EC70E080E090E00E94ED8168EE73E0BE
:1085900080E090E00E94ED8164EA7AE0CE010196ED
:1085A0000E94347E4AE050E06FEF7FEFCE010196EB
:1085B0000E94D226CE0101960E94A77D1092D90D6D
:1085C0001092D70D1092D40D1092D30D84E08093A9
:1085D000D20D0E94BC848B0161E08091D20D0E947B
:1085E00097818EEC9DE00E94B40860E082E30E94D7
:1085F000978161E083E30E94978161E084E30E94B8
:10860000978161E085E30E94978161E085E30E94A4
:108610007A8083E58CBD8DB58E7F8DBDBAE0FB2E53
:108620008FEF0E94A907FA94F110FACF60E08091D1
:10863000D20D0E947A8020E030E0A90160E08EEC4B
:108640009DE00E94B30BF82E8093D80D21E0821795
:1086500009F472C00E94BC84601B710B613D7740BD
:1086600050F381E08093D30D8EEC9DE00E94B4081E
:1086700066E97AE0CE0101960E94347ECE01019631
:108680000E94091BCE0101960E94A77D65E87AE051
:10869000CE0101960E94347E4AE050E06FEF7FEFFA
:1086A000CE0101960E943E0ACE0101960E94A77D4E
:1086B00058C1843009F052CE67E675E085E29DE04E
:1086C0000E94607F20E1B701A60185E29DE00E9443
:1086D000B67E67E779E085E29DE00E94A77E3ECE08
:1086E000823061F410929000809391001092950076
:1086F0001092940088BB8093710034CF833069F46A
:108700001092A00082E08093A1001092A500109228
:10871000A40089BB8093720025CF811123CF1092D2
:10872000200182E080932101109225011092240102
:108730008ABB8093730016CF2AEA31E040E050E014
:1087400068E08EEC9DE00E94B30B82FF2AC0F0929D
:10875000D90D8091D90DC12CD12CE12CF0E4FF2E44
:10876000823019F0C12CD12C760120E030E0A90133
:1087700067E38EEC9DE00E94B30BA701960169E2CE
:108780008EEC9DE00E94B30B8093D80D8823D1F02E
:108790000E94BC84601B710B613D774030F388E020
:1087A00061CFA4E0FA2E0E94AE0B8093D80DFA940C
:1087B000F110F9CF8A3A11F082E054CF82E0809331
:1087C000D90DC7CF8091D90D8230D1F420E030E0AF
:1087D000A9016AE38EEC9DE00E94B30B882311F09F
:1087E00086E040CF0E94AE0B807C803C19F483E091
:1087F0008093D90D0E94AE0B0E94AE0B0E94AE0B6F
:108800008EEC9DE00E94B4088DB58E7F8DBD8CB539
:108810008C7F8CBD8CB58CBD81E00E947B798823D8
:1088200009F427C38091FD0D811122CF8091F10DB4
:10883000803109F025C382E08093FD0D10920F0E68
:108840001092100E1092110E1092120E8091F20DD5
:108850009091F30DB0E0A0E0E5E0880F991FAA1F0A
:10886000BB1FEA95D1F780930B0E90930C0EA0934B
:108870000D0EB0930E0E8AED9DE09093140E809332
:10888000130E81E08093FC0D1092FE0D1092FF0DEF
:108890001092000E1092010E1092020E1092030E12
:1088A0001092040E1092050E1092060E1092070EF2
:1088B0001092080E1092090E10920A0E69E77AE0E3
:1088C000CE0101960E94347ECE0101960E94091BC2
:1088D000CE0101960E94A77D41E068E674E0CE01DA
:1088E00001960E947B95BE016F5F7F4F8DE991E1FC
:1088F0000E94301E80919F119091A0119C838B83C8
:108900008091A1119091A211A091A311B091A411F5
:108910008D839E83AF83B8878091A5119091A61116
:10892000A091A711B091A81189879A87AB87BC87BE
:1089300084EF93E09A8389838DE0E9EAF1E1DE0137
:108940001D9601900D928A95E1F78091B611909154
:10895000B7119B8F8A8F70E060E0CE0101960E9474
:10896000011F68EE73E080E090E00E94ED8143E13A
:1089700062EB72E0CE0101960E947B95BE016F5FB3
:108980007F4F88EB91E10E94301E60E47AE08EEB2D
:108990009FE00E94327D65E37AE08EEB9FE00E94CB
:1089A000D57C88EB91E10E94690D882309F499C276
:1089B0001EAE1DAE84E793E09CAF8BAF21961FAE39
:1089C000219719A218A29F8F8E8F1BA2812C712C28
:1089D0007E019BE3E90EF11C08EF1DE074E7A72E72
:1089E00073E0B72E882D972DFC01EE54FD4F2081AA
:1089F0002F3209F40196DC01AE54BD4FFE01E85A56
:108A0000FF4F30E020E06F014D914F3249F0442399
:108A100039F001962F5F3F4F41932C303105A1F77C
:108A20002C0D3D1DF9011082FC01EE54FD4F2081FB
:108A30002F3209F40196882E792E8E549D4FFC0119
:108A400060801C821B82BA82A9821E8221E0A6015C
:108A5000B801CE0101960E94D193882309F45EC229
:108A6000CE0101960E94A80A611029C22DE0083F9C
:108A7000120719F0C8010E94A80A88EB91E10E9430
:108A8000750D66E970E080E090E00E94ED81109243
:108A90004E0C04E610E091100BC085E29DE00E94B0
:108AA000DD74982E64E170E080E090E00E94ED813A
:108AB0000150110981F760E17AE0CE0101960E9430
:108AC000347E48EC50E070E060E0CE0101960E94F8
:108AD0003E0ACE0101960E94A77D32E781E0931203
:108AE00080E00E94990982E090E00E945A896CE23D
:108AF00071E080E090E00E94ED8183E090E00E94D0
:108B00005A896CE271E080E090E00E94ED8101E022
:108B100010E010936D0200936C0210935D020093BD
:108B20005C026AEA75E083E79FE00E948A7B10930B
:108B30005D0200935C0263E77FE0CE0101960E9434
:108B40003D7E62E070E0CE0101960E942237CE01A8
:108B500001960E94A77D6FEF79E0CE0101960E94F9
:108B6000347ECE0101960E94091BCE0101960E941F
:108B7000A77D6FEE79E0CE0101960E94347E48EC2D
:108B800050E070E060E0CE0101960E94D226CE0156
:108B900001960E94A77D66ED76E083E79FE00E9444
:108BA0008A7B63E77FE0CE0101960E943D7E63E011
:108BB00070E0CE0101960E942237CE0101960E94FC
:108BC000A77D82E090E090936D0280936C026EED41
:108BD00079E0CE0101960E94347ECE0101960E947A
:108BE000091BCE0101960E94A77D62ED79E0CE01BE
:108BF00001960E94347E48EC50E070E060E0CE01C7
:108C000001960E94D226CE0101960E94A77D6AEAB3
:108C100075E083E79FE00E948A7B809144119091E8
:108C2000451197FF06C06EEA75E083E79FE00E945A
:108C30008A7B63E77FE0CE0101960E943D7E62E081
:108C400070E0CE0101960E942237CE0101960E946B
:108C5000A77D66ED76E083E79FE00E948A7B82E055
:108C600090E090936D0280936C0263E77FE0CE0109
:108C700001960E943D7E63E070E0CE0101960E9465
:108C80002237CE0101960E94A77D809144119091D8
:108C900045119195819591099093451180934411C7
:108CA00001E010E010935D0200935C0284EF91E01C
:108CB00090936702809366026EE170E10E946809FA
:108CC00064E670E080E090E00E94ED8110936D0218
:108CD00000936C026CEB79E0CE0101960E94347E29
:108CE000CE0101960E94091BCE0101960E94A77D2C
:108CF00061EB79E0CE0101960E94347E4AE050E0BB
:108D00006FEF7FEFCE0101960E94D226CE01019631
:108D10000E94A77D68EE73E080E090E00E94ED8104
:108D20000E94AB2F0E94B3308DB79EB78253914003
:108D30000FB6F8949EBF0FBE8DBFADB7BEB71196EC
:108D400082E391E0EEE1F0E101900D920197E1F70D
:108D50000E94D4321092F70B88E19DE69093280F81
:108D60008093270F2091490F0FB6F894DEBF0FBEF6
:108D7000CDBF2830D8F4822F90E0FC01EE0FFF1F0A
:108D8000EE0FFF1FE75DF04F42EB55E0518340834C
:108D90002F5F2093490F880F991F880F991FFC019F
:108DA000E55DF04F81E890E2918380832091490F47
:108DB0002830D8F4822F90E0FC01EE0FFF1FEE0F59
:108DC000FF1FE75DF04F48EB55E0518340832F5F75
:108DD0002093490F880F991F880F991FFC01E55DAB
:108DE000F04F8EEA93E79183808387EB9EE00E94A9
:108DF000FF186FE979E0CE0101960E94347ECE0122
:108E000001960E94091BCE0101960E94A77D109237
:108E1000F80B0E9414896093F90B7093FA0B8093FE
:108E2000FB0B9093FC0B80911D118093500C8823B9
:108E300051F00E9414896093EF0B7093F00B8093B4
:108E4000F10B9093F20BCC59DF4F0FB6F894DEBFC5
:108E50000FBECDBFDF91CF911F910F91FF90EF908B
:108E6000DF90CF90BF90AF909F908F907F906F904A
:108E7000089580E00E947B79882309F4F9CBD2CC55
:108E8000803209F0F5CB83E08093FD0D4091F40D25
:108E90005091F50D6091F60D7091F70D40930F0E06
:108EA0005093100E6093110E7093120E2BE03EE063
:108EB0008AED9DE00E94848F8111DDCCD9CB21E029
:108EC000A601B801C7010E94D193D82EFDE0083F4A
:108ED0001F0709F44DC0C8010E94A80AD1104DC057
:108EE00024C060E27AE0CE0101960E94347ECE0179
:108EF00001960E94201BCE0101960E94A77D62EB85
:108F000072E0CE0101960E94467ECE0101960E943B
:108F1000091BCE0101960E94A77DB9CDFDE0083F57
:108F20001F0719F0C8010E94A80A68E975E0CE0180
:108F300001960E94467ECE0101960E94201BCE0122
:108F400001960E94A77D62EB72E0CE0101960E941D
:108F5000467ECE0101960E94091BCE0101960E9419
:108F6000A77D6EEB7FE088EB91E10E94767F85CD57
:108F70008823D9F28E01025E1F4F902F812F870127
:108F8000E92EF82E2FCD2F923F924F925F926F9243
:108F90007F928F929F92AF92BF92CF92DF92EF9289
:108FA000FF920F931F93CF93DF93CDB7DEB7E39775
:108FB0000FB6F894DEBF0FBECDBF67E97FE0CE01EC
:108FC0008E960E943D7E0EA51FA50115110571F01C
:108FD000D8018D918D01882349F0082E000C990B42
:108FE0000E9433B5F80131978083F2CF6CEB75E0C6
:108FF000CE0101960E94467EBE016F5F7F4FCE017B
:109000008E960E94917C182FCE0101960E94A77D1A
:10901000112309F401C145E050E067E97FE0CE018A
:1090200001960E94BF1EBE016F5F7F4F83E79FE0E6
:109030000E946E7DCE0101960E94A77D83E79FE08E
:109040000E94037C60E083E79FE00E94FF7C4091E8
:10905000770F5091780F66E770E183E79FE00E94F9
:10906000437968E674E0CE0101960E94467EBE0117
:109070006F5F7F4F83E79FE00E94917C182FCE01A6
:1090800001960E94A77D62E574E0111102C067E5B8
:1090900074E0CE0101960E94467E63E77FE0CE0138
:1090A00001960E94C27CBC018CE791E10E94577D31
:1090B000CE0101960E94A77D8CE791E10E94037C7E
:1090C0004091801150918111415051096CE771E13B
:1090D000CE0101960E94BF1EBE016F5F7F4F8EE5DD
:1090E00091E10E946E7DCE0101960E94A77D8EE5E2
:1090F00091E10E94F87B0E9420B09B01AC010E948C
:10910000E0B2882309F448C0609180117091811108
:10911000625071098CE791E10E94607C682FCE015A
:1091200001960E94127EBE016F5F7F4F8EE591E136
:109130000E946E7DCE0101960E94A77D68E674E0D4
:10914000CE0101960E94467EBE016F5F7F4F8EE585
:1091500091E10E94917C182FCE0101960E94A77D7B
:109160001123D1F0609180117091811163507109C8
:109170008CE791E10E94607C682FCE0101960E94ED
:10918000127EBE016F5F7F4F8EE591E10E946E7D82
:10919000CE0101960E94A77D84EF91E09093670233
:1091A000809366026EE170E10E94680964E670E0F7
:1091B00080E090E00E94ED8180913D02882371F073
:1091C00067E97FE0CE0101960E943D7ECE010196C7
:1091D0000E947521CE0101960E94A77DCE018E9638
:1091E0000E94A77D81E0E3960FB6F894DEBF0FBE24
:1091F000CDBFDF91CF911F910F91FF90EF90DF9046
:10920000CF90BF90AF909F908F907F906F905F9026
:109210004F903F902F90089562EC75E0CE0101963B
:109220000E94467EBE016F5F7F4FCE018E960E94E8
:10923000917C182FCE0101960E94A77D112309F47D
:1092400047C045E050E067E97FE0CE0101960E940B
:10925000BF1EBE016F5F7F4F83E79FE00E946E7D60
:10926000CE0101960E94A77D83E79FE00E94037CC8
:1092700060E083E79FE00E94FF7C4091770F509170
:10928000780F6EE470E183E79FE00E9443796EE41B
:1092900070E1CE014C960E94467E6AE674E0CE01F3
:1092A00001960E94467EBE01645E7F4FCE0101960C
:1092B0000E94C27CBC0186E791E10E94577DCE01ED
:1092C00001960E94A77DCE014C960E94A77D64CF97
:1092D00068EC75E0CE0101960E94467EBE016F5F8C
:1092E0007F4FCE018E960E94917C182FCE01019661
:1092F0000E94A77D1123E1F043E050E067E97FE0A1
:10930000CE0101960E94BF1EBE016F5F7F4F83E7B3
:109310009FE00E946E7DCE0101960E94A77D63E7CB
:109320007FE0CE0101960E943D7ECE010196CDCF19
:109330006CEC75E0CE0101960E94467EBE016F5F27
:109340007F4FCE018E960E94917C182FCE01019600
:109350000E94A77D112301F144E050E067E97FE01E
:10936000CE0101960E94BF1EBE016F5F7F4F83E753
:109370009FE00E946E7DCE0101960E94A77D83E74B
:109380009FE00E94F87B7093DD106093DC10709377
:109390008D0260938C0200CF61ED75E0CE010196E5
:1093A0000E94467EBE016F5F7F4FCE018E960E9467
:1093B000917C182FCE0101960E94A77D112309F4FC
:1093C00049C045E050E067E97FE0CE0101960E9488
:1093D000BF1EBE016F5F7F4F83E79FE00E946E7DDF
:1093E000CE0101960E94A77D83E79FE00E94F87B53
:1093F000709339116093381184EF91E09093670274
:10940000809366026EE170E10E94680964E670E094
:1094100080E090E00E94ED8168EC77E0CE0101965B
:109420000E94467E67E97FE0CE0101960E94C27CE1
:10943000BC01CE014C960E943D7ECE014C960E940E
:10944000091BCE014C960E94A77DCE0101960E9479
:10945000A77DB2CE67ED75E0CE0101960E94467EF3
:10946000BE016F5F7F4FCE018E960E94917C182FB8
:10947000CE0101960E94A77D1123E1F044E050E067
:1094800067E97FE0CE0101960E94BF1EBE016F5FBB
:109490007F4F83E79FE00E946E7DCE0101960E9480
:1094A000A77D83E79FE00E94F87B70933B11609358
:1094B0003A11A2CF6CED75E0CE0101960E94467E76
:1094C000BE016F5F7F4FCE018E960E94917C182F58
:1094D000CE0101960E94A77D1123A1F044E050E047
:1094E00067E97FE0CE0101960E94BF1EBE016F5F5B
:1094F0007F4F83E79FE00E946E7DCE0101960E9420
:10950000A77D84CF61EE75E0CE0101960E94467E74
:10951000BE016F5F7F4FCE018E960E94917C182F07
:10952000CE0101960E94A77D1123A1F047E050E0F3
:1095300067E97FE0CE0101960E94BF1EBE016F5F0A
:109540007F4F83E79FE00E946E7DCE0101960E94CF
:10955000A77D2CCE69EE75E0CE0101960E94467E75
:10956000BE016F5F7F4FCE018E960E94917C182FB7
:10957000CE0101960E94A77D1111D8CF61EF75E051
:10958000CE0101960E94467EBE016F5F7F4FCE01E5
:109590008E960E94917C182FCE0101960E94A77D85
:1095A000112321F081E00E94990900CE6BEF75E054
:1095B000CE0101960E94467EBE016F5F7F4FCE01B5
:1095C0008E960E94917C182FCE0101960E94A77D55
:1095D000112319F00E94AB2FE9CD65E979E0CE01A6
:1095E00001960E94347EBE016F5F7F4FCE018E9642
:1095F0000E94917C182FCE0101960E94A77D112315
:1096000009F485C06AE879E0CE0101960E94347EB3
:10961000BE016F5F7F4FCE018E960E94917C182F06
:10962000CE0101960E94A77D112309F454C04AE09F
:1096300050E067E97FE0CE0101960E94BF1EBE01A7
:109640006F5F7F4F83E79FE00E946E7DCE010196A2
:109650000E94A77D83E79FE00E94F87B0E94EF882D
:109660000E9414896093EF0B7093F00B8093F10BC1
:109670009093F20B0E9414896093E90B7093EA0BAC
:109680008093EB0B9093EC0BCE014C960E94222220
:1096900062E076E0CE0101960E94467EBE01645EE5
:1096A0007F4FCE0101960E94C27CBC01CE01829602
:1096B0000E943D7ECE0182960E94091BCE018296B9
:1096C0000E94A77DCE0101960E94A77DCE014C96F7
:1096D0000E94A77D71CD4BE050E067E97FE0CE01AD
:1096E00001960E94BF1EBE016F5F7F4F83E79FE020
:1096F0000E946E7DCE0101960E94A77D83E79FE0C8
:109700000E94F87B60587F488F4F9F4FA7CF68E437
:1097100077E0CE0101960E94467EBE016F5F7F4FCB
:10972000CE018E960E94917C182FCE0101960E9448
:10973000A77D112309F46AC045E050E067E97FE0A6
:10974000CE0101960E94BF1EBE016F5F7F4F83E76F
:109750009FE00E946E7DCE0101960E94A77D0E942F
:1097600014896093EF0B7093F00B8093F10B90933F
:10977000F20B83E79FE00E94F87B60936E02709388
:109780006F02809370029093710260931E11709328
:109790001F11809320119093211120911D1120936E
:1097A000500C672B682B692B11F41092500C84EF2E
:1097B00091E090936702809366026EE170E10E94EF
:1097C000680964E670E080E090E00E94ED816BE75C
:1097D00079E0CE0101960E94347ECE0101960E946E
:1097E000201BCE0101960E94A77D40916E025091F0
:1097F0006F026091700270917102CE0101960E9419
:10980000C07BCE0101960E94091BDBC163E176E0BB
:10981000CE0101960E94467EBE016F5F7F4FCE0152
:109820008E960E94917C182FCE0101960E94A77DF2
:109830001123D9F14AE050E067E97FE0CE010196BB
:109840000E94BF1EBE016F5F7F4F83E79FE00E94B3
:109850006E7DCE0101960E94A77D83E79FE00E9466
:10986000F87B613071058105910519F481E08093E1
:109870001D1183E79FE00E94F87B672B682B692B03
:1098800011F410921D1180911D118093500C8823AA
:1098900009F4B2CD0E9414896093EF0B7093F00B22
:1098A0008093F10B9093F20BA7CD6EE176E0CE01A1
:1098B00001960E94467EBE016F5F7F4FCE018E965D
:1098C0000E94917C182FCE0101960E94A77D112342
:1098D000A1F048E050E067E97FE0CE0101960E94E8
:1098E000BF1EBE016F5F7F4F83E79FE00E946E7DCA
:1098F000CE0101960E94A77D8FCD67E276E0CE0172
:1099000001960E94467EBE016F5F7F4FCE018E960C
:109910000E94917C182FCE0101960E94A77D1123F1
:1099200021F145E050E067E97FE0CE0101960E9419
:10993000BF1EBE016F5F7F4F83E79FE00E946E7D79
:10994000CE0101960E94A77D83E79FE00E94F87BED
:109950006130710521F481E08093510C2DCC672B8F
:1099600009F02ACC1092510C27CC6DE276E0CE01A2
:1099700001960E94467EBE016F5F7F4FCE018E969C
:109980000E94917C182FCE0101960E94A77D112381
:1099900051F163E070E087E99FE00E94607C682FEE
:1099A000CE0101960E94127EBE016F5F7F4F83E75A
:1099B0009FE00E946E7DCE0101960E94A77D83E705
:1099C0009FE00E94037C83E79FE00E94F87B9B015D
:1099D000215031092330310508F0EECB70934D1141
:1099E00060934C11D9CB61E376E0CE0101960E94E1
:1099F000467EBE016F5F7F4FCE018E960E94917CA6
:109A0000182FCE0101960E94A77D112309F46AC088
:109A100066E070E087E99FE00E94607C682FCE01DD
:109A200001960E94127EBE016F5F7F4F83E79FE029
:109A30000E946E7DCE0101960E94A77D83E79FE084
:109A40000E94037C60E083E79FE00E94FF7C83E745
:109A50009FE00E94F87B6B01CB010197039708F010
:109A6000ABCB48E050E067E97FE0CE0101960E9471
:109A7000BF1EBE016F5F7F4F83E79FE00E946E7D38
:109A8000CE0101960E94A77D83E79FE00E94037CA0
:109A90008091770F9091780F0997A8F028E030E037
:109AA00050E040E063E77FE0CE0101960E945B7EDC
:109AB000BE016F5F7F4F83E79FE00E946E7DCE0106
:109AC00001960E94A77DB60113E0660F771F1A95D5
:109AD000E1F76E5C7F4E48E050E083E79FE00E9434
:109AE00043795ACB63E779E0CE0101960E94347E38
:109AF000BE016F5F7F4FCE018E960E94917C182F22
:109B0000CE0101960E94A77D112309F486C06DE164
:109B100074E0CE0101960E94467E47E050E0BE010F
:109B2000625D7F4FCE014C960E94BF1EBE01645EF7
:109B30007F4FCE0101960E946E7DCE014C960E9411
:109B4000A77D62E075E0CE014C960E94467EBE0184
:109B5000645E7F4FCE0101960E94917C182FCE014A
:109B60004C960E94A77D112379F141E050E0BE019F
:109B70006F5F7F4FCE014C960E94BF1ECE014C9668
:109B80000E94F87B8B010A5C1F4FCE014C960E940D
:109B9000A77D10934F1100934E1110938F020093E5
:109BA0008E0284EF91E090936702809366026EE1EB
:109BB00070E10E94680964E670E080E090E00E9435
:109BC000ED81CE01019684CD61EC76E0CE014C961C
:109BD0000E94467EBE01645E7F4FCE0101960E94C8
:109BE000917C182FCE014C960E94A77D112379F00D
:109BF00041E050E0BE016F5F7F4FCE014C960E9466
:109C0000BF1ECE014C960E94F87B8B01BECFCE01C9
:109C100001960E94F87B8B01BCCF6CE679E0CE0107
:109C200001960E94347EBE016F5F7F4FCE018E96FB
:109C30000E94917C182FCE0101960E94A77D1123CE
:109C400009F4AAC067E476E0CE0101960E94467E40
:109C500046E050E0BE016F5F7F4FCE018E960E94BE
:109C6000F2A58C01CE0101960E94A77D980146E0E5
:109C700050E0BE01625D7F4FCE0101960E945B7E87
:109C8000CE0101960E94F87B6B01CE0101960E94E5
:109C9000A77D6DE174E0CE0101960E94467EA80189
:109CA0004F5F5F4FBE01625D7F4FCE014C960E94B9
:109CB000BF1EBE01645E7F4FCE0101960E946E7D85
:109CC000CE014C960E94A77D62E075E0CE014C96D5
:109CD0000E94467EBE01645E7F4FCE0101960E94C7
:109CE000917C182FCE014C960E94A77D112321F163
:109CF00041E050E0BE016F5F7F4FCE014C960E9465
:109D0000BF1ECE014C960E94F87B8B010A5C1F4F50
:109D1000CE014C960E94A77DF6013196EE0FFF1FF3
:109D2000E25EFF4E11830083F601EE0FFF1FE65542
:109D3000F44F1183008335CF61EC76E0CE014C9671
:109D40000E94467EBE01645E7F4FCE0101960E9456
:109D5000917C182FCE014C960E94A77D112379F09B
:109D600041E050E0BE016F5F7F4FCE014C960E94F4
:109D7000BF1ECE014C960E94F87B8B01C9CFCE014D
:109D800001960E94F87B0091AC0B1091AD0B015035
:109D90001109060F171FC0CF67E374E0CE014C9680
:109DA0000E94467EBE01645E7F4FCE018E960E9469
:109DB000917C11E0811115C068E376E0CE01019637
:109DC0000E94467EBE016F5F7F4FCE018E960E943D
:109DD000917C11E0811101C010E0CE0101960E943A
:109DE000A77DCE014C960E94A77D112309F411C2D4
:109DF00064E476E0CE014C960E94467E6FE376E006
:109E0000CE0101960E94467EAE01445E5F4FBE01C8
:109E10006F5F7F4FCE018E960E94F9A4CE0101960E
:109E20000E94A77DCE014C960E94A77D64E476E057
:109E3000CE014C960E94467E61E476E0CE0101960A
:109E40000E94467EAE01445E5F4FBE016F5F7F4F52
:109E5000CE018E960E94F9A4CE0101960E94A77DA4
:109E6000CE014C960E94A77D64E476E0CE014C962C
:109E70000E94467E63E476E0CE0101960E94467E13
:109E8000AE01445E5F4FBE016F5F7F4FCE018E9685
:109E90000E94F9A4CE0101960E94A77DCE014C96A6
:109EA0000E94A77D67E476E0CE014C960E94467E34
:109EB00066E476E0CE0101960E94467EAE01445EE5
:109EC0005F4FBE016F5F7F4FCE018E960E94F9A457
:109ED000CE0101960E94A77DCE014C960E94A77DDF
:109EE00067E476E0CE014C960E94467E6CE678E010
:109EF000CE0101960E94467EAE01445E5F4FBE01D8
:109F00006F5F7F4FCE018E960E94F9A4CE0101961D
:109F10000E94A77DCE014C960E94A77DCE018E9611
:109F20000E94037C0E9414896093F30B7093F40BDE
:109F30008093F50B9093F60B56E0E52EF12C64E63A
:109F4000462E512C612C712C22242394312C570144
:109F5000B3E0AB0EB11C8AA99BA90197A816B9065C
:109F600008F02AC9B701CE018E960E94607C682F46
:109F7000CE014C960E94127E6701E2E0CE0ED11C0B
:109F8000FFEFEF1AFF0A9601A701BE01625D7F4F46
:109F9000CE0101960E945B7ECE0101960E94F87B65
:109FA0008B01CE0101960E94A77D0130110521F49D
:109FB00000913811109139110330110521F40091ED
:109FC0003A1110913B1164E476E0CE0101960E94B3
:109FD000467EA601BE016F5F7F4FCE018E960E9426
:109FE000F2A56C01CE0101960E94A77D6DE174E09F
:109FF000CE0101960E94467E480181E0881A9108B0
:10A000001C141D042CF59601A501BE01625D7F4F55
:10A01000CE0182960E945B7EBE016E5D7F4FCE01B7
:10A0200001960E946E7DCE0182960E94A77D93E0EC
:10A030008916910420F17601AFEFEA1AFA0ACE01EF
:10A0400001960E94A77DCE014C960E94A77D7FCFEE
:10A05000A501BE01625D7F4FCE0182960E94BF1EA8
:10A06000BE016E5D7F4FCE0101960E946E7DCE01D6
:10A0700082960E94A77DB3E08B16910400F770E0F2
:10A0800060E0CE014C960E94607C823509F061C090
:10A09000CE0101960E94F87B672B682B692BB1F4E7
:10A0A000F801EE0FFF1FE952FD4F11821082F801F7
:10A0B000EE0FFF1FEE0FFF1FE154FD4F82E090E017
:10A0C000A0E0B0E080839183A283B383CE010196A8
:10A0D0000E94F87B6130710581059105A9F5F801B1
:10A0E000EE0FFF1FE952FD4F31822082000F111F3A
:10A0F000000F111FF801E154FD4F80819181A28171
:10A10000B381181619061A061B0624F040825182E4
:10A1100062827382CE0101960E94F87B62307105E3
:10A12000810591053CF0F801E154FD4F6083718396
:10A13000828393830E94148901521D4FD8016D932D
:10A140007D938D939C9313971C141D040CF473CF73
:10A1500076CF8634E9F5CE0101960E94F87B672B15
:10A16000682B692B39F4F801EE0FFF1FEC5AFD4FF5
:10A1700011821082CE0101960E94F87B6130710538
:10A180008105910539F4F801EE0FFF1FEC5AFD4FE0
:10A1900031822082000F111F000F111FF801E154BE
:10A1A000FD4F80819181A281B381181619061A068C
:10A1B0001B0624F040825182628273820E941489BD
:10A1C00001521D4FF8016083718382839383BCCF5A
:10A1D000843461F4CE0101960E94F87B000F111FB8
:10A1E000000F111FF801EC5BFD4FA0CF843509F083
:10A1F000ABCFCE0101960E94F87B000F111F000F1C
:10A20000111FF801E154FD4F6083718382839383B2
:10A21000D5CF66E679E0CE0101960E94347EBE017C
:10A220006F5F7F4FCE018E960E94917C182FCE01DA
:10A2300001960E94A77D112309F49DC045E050E0DE
:10A2400067E97FE0CE0101960E94BF1EBE016F5FED
:10A250007F4F83E79FE00E946E7DCE0101960E94B2
:10A26000A77D83E79FE00E94037C60E083E79FE097
:10A270000E94FF7C64E075E0CE014C960E94467E11
:10A2800063E77FE0CE0101960E943D7EAE014E5D08
:10A290005F4FBE01645E7F4FCE0101960E940EA605
:10A2A000182FCE0101960E94A77DCE014C960E94E8
:10A2B000A77D112311F40C94DC488E010E5D1F4F15
:10A2C00058E4A52E51E1B52E60E4C62E62E0D62EEC
:10A2D000F12CE12CD8016D918D01F50161935F01A5
:10A2E000D6016D936D01CE0101960E9481A4CE012D
:10A2F00001960E94201BCE0101960E94A77DB3E02B
:10A30000EB16F10471F064E075E0CE0101960E9455
:10A31000467ECE0101960E94201BCE0101960E942E
:10A32000A77DEFEFEE1AFE0AF4E0EF16F10491F6C6
:10A330006DE174E0CE0101960E94467ECE01019649
:10A340000E94091BCE0101960E94A77D6EE170E17B
:10A3500080916602909167020E94680964E670E04D
:10A3600080E090E00E94ED816EE479E0CE010196FC
:10A370000E94347E46CA69E479E0CE0101960E94CB
:10A38000347EBE016F5F7F4FCE018E960E94917C1E
:10A39000182FCE0101960E94A77D112309F47CC0DD
:10A3A00044E050E067E97FE0CE0101960E94BF1EC5
:10A3B000BE016F5F7F4F83E79FE00E946E7DCE01FD
:10A3C00001960E94A77D83E79FE00E94037C60E0E6
:10A3D00083E79FE00E94FF7C4091770F5091780FB8
:10A3E0006AE97BE083E79FE00E94437964E075E0DF
:10A3F000CE014C960E94467E63E77FE0CE01019637
:10A400000E943D7EAE014E5D5F4FBE01645E7F4F98
:10A41000CE0101960E940EA6182FCE0101960E9431
:10A42000A77DCE014C960E94A77D112311F40C94B8
:10A43000DC488E010E5D1F4F4AE4E42E40E1F42E0D
:10A440006E0186E2C80ED11CD8016D918D01F70115
:10A4500061937F01CE0101960E9481A4CE010196F5
:10A460000E94091BCE0101960E94A77DC016D1064D
:10A4700059F784EF91E090936702809366026EE152
:10A4800070E10E94680964E670E080E090E00E945C
:10A49000ED816EE379E06ACF67E379E0CE01019662
:10A4A0000E94347EBE016F5F7F4FCE018E960E9468
:10A4B000917C182FCE0101960E94A77D1123F1F106
:10A4C00046E050E067E97FE0CE0101960E94BF1EA2
:10A4D000BE016F5F7F4F83E79FE00E946E7DCE01DC
:10A4E00001960E94A77D83E79FE00E94037C8091F4
:10A4F000770F9091780F892B11F40C94DC4883E747
:10A500009FE00E94F87B709347116093461170930F
:10A510003F0260933E0284EF91E090936702809344
:10A5200066026EE170E10E94680964E670E080E016
:10A5300090E00E94ED8163E279E018CF6CE179E070
:10A54000CE0101960E94347EBE016F5F7F4FCE0127
:10A550008E960E94917C182FCE0101960E94A77DB5
:10A560001123B9F06FE079E0CE0101960E94347EAC
:10A5700044E650E06FEF7FEFCE0101960E943E0A65
:10A58000CE0101960E94A77DF0E0E0E019950C94C1
:10A59000DC4867E079E0CE0101960E94347EBE017E
:10A5A0006F5F7F4FCE018E960E94917C182FCE0157
:10A5B00001960E94A77D112301F169E476E0CE01A6
:10A5C00001960E94467E64E671E1CE0101960E94EA
:10A5D000C27CBC0189E79FE00E94577DCE010196B5
:10A5E0000E94A77D69E77FE0CE0101960E943D7E33
:10A5F000CE0101960E94091B8DC460E079E0CE0176
:10A6000001960E94347EBE016F5F7F4FCE018E9611
:10A610000E94917C182FCE0101960E94A77D1123E4
:10A6200069F061EF78E089E79FE00E94327D6AE699
:10A6300071E189E79FE00E942B7DD4CF64E576E04D
:10A64000CE0101960E94467EBE016F5F7F4FCE0114
:10A650008E960E94917C182FCE0101960E94A77DB4
:10A66000112331F00E94B33010923D020C94DC486B
:10A670006DE576E0CE014C960E94467EBE01645E9A
:10A680007F4F87E99FE00E94917C11E0811115C006
:10A6900062E676E0CE0101960E94467EBE016F5FC3
:10A6A0007F4F87E99FE00E94917C11E0811101C0FA
:10A6B00010E0CE0101960E94A77DCE014C960E942B
:10A6C000A77D112309F441C067E476E0CE0101962D
:10A6D0000E94467E40919B0F50919C0F8D819E81E0
:10A6E000481B590BBE016F5F7F4F87E99FE00E94B7
:10A6F000ABA4AC014F5F5F4F67E97FE0CE014C96A2
:10A700000E94BF1EBE01645E7F4F83E79FE00E94F0
:10A710006E7DCE014C960E94A77DCE0101960E94CF
:10A72000A77D83E79FE00E94F87B6115710531F4F6
:10A7300081E08093F0020E94279896CF61307105E6
:10A7400009F092CF1092F002F6CF67E676E0CE01E4
:10A7500001960E94467EBE016F5F7F4FCE018E96AE
:10A760000E94917C182FCE0101960E94A77D112393
:10A7700009F43BC143E050E067E97FE0CE01019678
:10A780000E94BF1EBE016F5F7F4F83E79FE00E9464
:10A790006E7DCE0101960E94A77D63E77FE0CE012A
:10A7A00001960E943D7ECE0101960E947521CE0148
:10A7B00001960E94A77D84EF91E0909367028093B9
:10A7C000660263E77FE0CE0101960E943D7E60E075
:10A7D000CE0101960E94137DBC0180E791E10E94A9
:10A7E000577DCE0101960E94A77D63E77FE0CE01F1
:10A7F00001960E943D7E60E0CE0101960E94137D8D
:10A80000BC018AE691E10E94577DCE0101960E942B
:10A81000A77D40917411509175116EED70E180E744
:10A8200091E10E94437940916E1150916F1169EE50
:10A8300070E18AE691E10E9443796EE170E18091D6
:10A840006602909167020E9468096BE676E0CE018D
:10A8500001960E94467E63E77FE0CE0101960E944A
:10A86000C27CBC01CE0182960E943D7ECE01019643
:10A870000E94A77D8091DA109091DB10892B39F42A
:10A88000BE016E5D7F4F88E89CE00E94687F68EBA8
:10A890007BE080E090E00E94ED818091DA10909161
:10A8A000DB10029709F087C063E77FE0CE0188964E
:10A8B0000E943D7E63E776E0CE0101960E94467ECF
:10A8C000CE0101960E945398CE0101960E94A77D69
:10A8D00064EF71E080E090E00E94ED8166E776E051
:10A8E000CE0101960E94467ECE0101960E945398A9
:10A8F000CE0101960E94A77D6CED75E080E090E0AE
:10A900000E94ED816FE776E0CE0101960E94467EBF
:10A91000CE0101960E945398CE0101960E94A77D18
:10A9200064EF71E080E090E00E94ED816DE876E0F8
:10A93000CE0101960E94467ECE0101960E94539858
:10A94000CE0101960E94A77D64EF71E080E090E067
:10A950000E94ED816BE676E0CE0101960E94467E74
:10A96000BE01685D7F4FCE0101960E94C27CBC0192
:10A97000CE014C960E943D7ECE0101960E94A77D9D
:10A98000CE014C960E94037CBE01645E7F4FCE01D7
:10A9900001960E943D7ECE0101960E945398CE0101
:10A9A00001960E94A77DCE014C960E94A77DCE0104
:10A9B00088960E94A77D68EB7BE080E090E00E9493
:10A9C000ED816EED70E1CE0101960E94467ECE01D2
:10A9D00001960E947521CE0101960E94A77D1092DA
:10A9E0003D02CE0182960C94684B6BE976E0CE0175
:10A9F00001960E94467EBE016F5F7F4FCE018E960C
:10AA00000E94917C182FCE0101960E94A77D1123F0
:10AA100009F486C044E050E067E97FE0CE0101968A
:10AA20000E94BF1EBE016F5F7F4F83E79FE00E94C1
:10AA30006E7DCE0101960E94A77D60EA76E0CE0190
:10AA400001960E94467E63E77FE0CE0101960E9458
:10AA5000C27CBC01CE014C960E943D7ECE01019687
:10AA60000E94A77D8091DA109091DB10892B39F438
:10AA7000BE01645E7F4F88E89CE00E94687F68E8C2
:10AA800073E180E090E00E94ED818091DA10909176
:10AA9000DB10029759F567EA76E0CE0101960E9435
:10AAA000467E8091770F9091780F892B19F560EB96
:10AAB00076E0CE0101960E948A7BBE01645E7F4FE4
:10AAC000CE0182960E943D7ECE0182960E945398CE
:10AAD000CE0182960E94A77D68E873E180E090E055
:10AAE0000E94ED81CE0101960E94A77D10923D0249
:10AAF0000C94664BBE016F5F7F4FCE0182960E9421
:10AB00003D7ECE0182960E945398CE0182960E948D
:10AB1000A77D60E777E180E090E00E94ED81CDCFF6
:10AB200069EB76E0CE0101960E94467EBE016F5F22
:10AB30007F4FCE018E960E94917C182FCE010196F8
:10AB40000E94A77D112309F475C067E97FE083E7C0
:10AB50009FE00E94577D81E080933D0267E97FE09E
:10AB6000CE0101960E943D7ECE0101960E94752184
:10AB7000CE0101960E94A77D8091DA109091DB10A2
:10AB8000029709F163E77FE088E89CE00E94687F14
:10AB900068EB7BE080E090E00E94ED81CE010196C1
:10ABA0000E94EC98BE016F5F7F4F87E99FE00E9493
:10ABB0006E7DCE0101960E94A77D60ED77E080E07A
:10ABC00090E00E94ED818091DA109091DB10029765
:10ABD00071F463E77FE0CE0101960E943D7ECE01D5
:10ABE00001960E945398CE0101960E94A77D809104
:10ABF0009B0F90919C0F892B09F436CD68EC77E080
:10AC0000CE0101960E94467E67E97FE0CE01019663
:10AC10000E94C27CBC01CE014C960E943D7ECE01BA
:10AC20004C960E94091BCE014C960E94A77DCE0136
:10AC3000019650C26DEB76E0CE0101960E94467EF1
:10AC4000BE016F5F7F4FCE018E960E94917C182FC0
:10AC5000CE0101960E94A77D112309F495C1809130
:10AC6000DA109091DB10019709F0FECC63EC76E0EE
:10AC7000CE0188960E94467EBE01685D7F4F88E8BF
:10AC80009CE00E94687F6CE271E080E090E00E94AE
:10AC9000ED81CE0182960E94EC9864E670E080E03F
:10ACA00090E00E94ED8110E000E025E0C22ED12C62
:10ACB0003AE0A32EB12C6EEC76E0CE0101960E9414
:10ACC000467E50E040E0BE016F5F7F4FCE0182962E
:10ACD0000E94F2A57C01CE0101960E94A77DA701EA
:10ACE0004F5F5F4FBE016E5D7F4FCE0101960E94A8
:10ACF000BF1EBE016F5F7F4FCE0188960E946E7DA2
:10AD0000CE0101960E94A77D8CA59DA5892B09F1F6
:10AD100070E060E0CE0188960E94607C082E000CF6
:10AD2000990BC0970A97A8F460ED76E0CE010196E2
:10AD30000E94467EBE016F5F7F4FCE0188960E94C3
:10AD4000917CE82ECE0101960E94A77DFF24F3940A
:10AD5000E110F12C60E977E0CE0101960E94347E8B
:10AD600064E170E0CE0101960E94C8A6CE01019672
:10AD70000E94A77D0F5F1F4F62E370E080E090E0CC
:10AD80000E94ED81C801B6010E94F1B20197C1F4A1
:10AD9000CE0101960E940E238D819E81892B09F49C
:10ADA000BEC0BE016F5F7F4F87E99FE00E94577D65
:10ADB0000E94C347FF24F394CE0101960E94A77D11
:10ADC000CE0101960E94EC98BE016F5F7F4FCE01CD
:10ADD00082960E946E7DCE0101960E94A77D62E35D
:10ADE00070E080E090E00E94ED810436110519F0DA
:10ADF000FF2009F460CF80916D0B8823F1F068EC9F
:10AE000077E0CE014C960E94467EBE01685D7F4F82
:10AE1000CE014C960E94C27CBC01CE0101960E94DC
:10AE20003D7ECE0101960E94091BCE0101960E9433
:10AE3000A77DCE014C960E94A77D8CA59DA5892B50
:10AE400069F070E060E0CE0188960E94607C082E78
:10AE5000000C990BC0970A9708F47AC068ED76E069
:10AE6000CE0101960E94467ECE0182960E94A77D69
:10AE7000CE0188960E94A77D8D819E81009709F45E
:10AE800049C0E981FA812081222309F443C0079750
:10AE900008F440C068EE78E0CE014C960E94347E03
:10AEA00068EC70E0CE014C960E94C8A6CE014C968C
:10AEB0000E94A77DBE016F5F7F4FCE014C960E941E
:10AEC0003D7E40ED57E06FEF7FEFCE014C960E9444
:10AED0003E0ACE014C960E94A77D64EE76E0CE013C
:10AEE0004C960E94467E67E97FE0CE014C960E9418
:10AEF000C27CBC01CE0182960E943D7ECE0182962C
:10AF00000E94091BCE0182960E94A77DCE014C961D
:10AF10000E94A77DCE0101960E94A77DA5CB04319A
:10AF200011050CF449CFC801B5010E94F1B2892B7B
:10AF300009F042CFBE01685D7F4F88E89CE00E9427
:10AF4000687F68EC70E080E090E00E94ED8134CF93
:10AF500060ED76E0CE0101960E94467EBE016F5FF5
:10AF60007F4FCE0188960E94917C182FCE010196CA
:10AF70000E94A77D111172CFBE01685D7F4FCE0187
:10AF800001960E942B7E70CF62EF76E0CE01019693
:10AF90000E94467EBE016F5F7F4FCE018E960E945B
:10AFA000917C182FCE0101960E94A77D112309F4F0
:10AFB000EAC025E030E044E050E067E97FE0CE0100
:10AFC00001960E945B7EBE016F5F7F4F83E79FE02B
:10AFD0000E946E7DCE0101960E94A77D67E97FE009
:10AFE000CE0101960E943D7ECE0101960E94752100
:10AFF000CE0101960E94A77D83E79FE00E94F87B27
:10B000006130710509F069C07093DB106093DA104C
:10B010006FEB77E0CE0101960E94347ECE0101965F
:10B020000E947521CE0101960E94A77D67EF76E010
:10B03000CE014C960E94467E6AE671E1CE014C96A6
:10B040000E94C27CBC01CE0101960E943D7E48EC6C
:10B0500050E06FEF7FEFCE0101960E94D226CE0125
:10B0600001960E94A77DCE014C960E94A77D0E946A
:10B0700064A440E052EC61E070E088E89CE00E944B
:10B08000277884EF91E090936702809366026EE1E7
:10B0900070E10E94680966E077E0CE014C960E945C
:10B0A000467E64E671E1CE014C960E94C27CBC01F2
:10B0B000CE0101960E943D7E40ED57E06FEF7FEF9D
:10B0C000CE0101960E943E0ACE0101960E94A77D04
:10B0D000CE014C960E94A77DC7CA61157105D1F5B6
:10B0E0001092DB101092DA1061EB77E0CE0101963E
:10B0F0000E94347ECE0101960E947521CE010196F8
:10B100000E94A77D6DEF76E0CE014C960E94467EB0
:10B110006AE671E1CE014C960E94C27CBC01CE0170
:10B1200001960E943D7E48EC50E06FEF7FEFCE012C
:10B1300001960E94D226CE0101960E94A77DCE01E3
:10B140004C960E94A77D0E9464A440E855E260E00E
:10B1500070E093CF6230710509F086CA7093DB10FE
:10B160006093DA1060EA77E0CE0101960E94347EA7
:10B17000CE0101960E947521CE0101960E94A77D05
:10B1800061E077E0C1CF6BE077E0CE0101960E94ED
:10B19000467EBE016F5F7F4FCE018E960E94917CEE
:10B1A000182FCE0101960E94A77D112309F441C0FA
:10B1B00047E050E067E97FE0CE0101960E94BF1EA4
:10B1C000BE016F5F7F4F83E79FE00E946E7DCE01DF
:10B1D00001960E94A77D66ED76E0CE0101960E9461
:10B1E000467EBE016F5F7F4F83E79FE00E94917CA8
:10B1F000182FCE0101960E94A77D111110924F0CBD
:10B2000066ED74E0CE0101960E94467EBE016F5F3E
:10B210007F4F83E79FE00E94917C182FCE0101961B
:10B220000E94A77D112309F4E9CC81E080934F0CA3
:10B23000E5CC63E177E0CE0101960E94467EBE0137
:10B240006F5F7F4FCE018E960E94917C182FCE01AA
:10B2500001960E94A77D112381F146E050E067E945
:10B260007FE0CE0101960E94BF1EBE016F5F7F4F3F
:10B2700083E79FE00E946E7DCE0101960E94A77D2C
:10B2800083E79FE00E94ED7B60932211709323116E
:10B29000809324119093251184EF91E0909367029D
:10B2A000809366026EE170E10E94680964E670E0D6
:10B2B00080E090E00E94ED81A1CC6AE177E0CE01D0
:10B2C00001960E94467EBE016F5F7F4FCE018E9633
:10B2D0000E94917C182FCE0101960E94A77D112318
:10B2E00001F148E050E067E97FE0CE0101960E945D
:10B2F000BF1EBE016F5F7F4F83E79FE00E946E7DA0
:10B30000CE0101960E94A77D83E79FE00E94ED7B1E
:10B31000609328117093291180932A1190932B1117
:10B32000BBCF63E277E0CE0101960E94467EBE016C
:10B330006F5F7F4FCE018E960E94917C182FCE01B9
:10B3400001960E94A77D112301F149E050E067E9D1
:10B350007FE0CE0101960E94BF1EBE016F5F7F4F4E
:10B3600083E79FE00E946E7DCE0101960E94A77D3B
:10B3700083E79FE00E94ED7B60932C1170932D1169
:10B3800080932E1190932F1187CF6DE277E0CE013D
:10B3900001960E94467EBE016F5F7F4FCE018E9662
:10B3A0000E94917C182FCE0101960E94A77D112347
:10B3B000F1F049E050E067E97FE0CE0101960E949C
:10B3C000BF1EBE016F5F7F4F83E79FE00E946E7DCF
:10B3D000CE0101960E94A77D83E79FE00E94ED7B4E
:10B3E0000E94A5B2709333116093321155CF67E379
:10B3F00077E0CE0101960E94467EBE016F5F7F4FCF
:10B40000CE018E960E94917C182FCE0101960E944B
:10B41000A77D1123F1F04AE050E067E97FE0CE011B
:10B4200001960E94BF1EBE016F5F7F4F83E79FE0C2
:10B430000E946E7DCE0101960E94A77D83E79FE06A
:10B440000E94ED7B0E94A5B2709331116093301180
:10B4500023CF62E477E0CE0101960E94467EBE01D2
:10B460006F5F7F4FCE018E960E94917C182FCE0188
:10B4700001960E94A77D112311F14BE050E067E98E
:10B480007FE0CE0101960E94BF1EBE016F5F7F4F1D
:10B4900083E79FE00E946E7DCE0101960E94A77D0A
:10B4A00083E79FE00E94ED7B0E94A5B26093341178
:10B4B000709335118093361190933711EDCE6EE471
:10B4C00077E0CE0101960E94467EBE016F5F7F4FFE
:10B4D000CE018E960E94917C182FCE0101960E947B
:10B4E000A77D1123E1F045E050E067E97FE0CE0160
:10B4F00001960E94BF1EBE016F5F7F4F83E79FE0F2
:10B500000E946E7DCE0101960E94A77D83E79FE099
:10B510000E94F87B7093271160932611BDCE64E5DD
:10B5200077E0CE0101960E94467EBE016F5F7F4F9D
:10B53000CE018E960E94917C182FCE0101960E941A
:10B54000A77D112359F00E9414896093F30B709327
:10B55000F40B8093F50B9093F60B86C86AE577E0C1
:10B56000CE0101960E94467EBE016F5F7F4FCE01E5
:10B570008E960E94917C182FCE0101960E94A77D85
:10B58000112389F143E050E0BE01625D7F4FCE019F
:10B5900001960E94BF1EBE016F5F7F4F83E79FE051
:10B5A0000E946E7DCE0101960E94A77D8091770F4B
:10B5B0009091780F892B41F083E79FE00E94F87B00
:10B5C00070936D0260936C0280916C0290916D0299
:10B5D0000197029708F412CB81E090E090936D02FE
:10B5E00080936C020BCB6BE377E0CE014C960E940C
:10B5F000467EBE01645E7F4FCE018E960E94917C96
:10B6000011E0811115C06DE977E0CE0101960E942D
:10B61000467EBE016F5F7F4FCE018E960E94917C69
:10B6200011E0811101C010E0CE0101960E94A77DBA
:10B63000CE014C960E94A77D112309F468C06BE3EC
:10B6400077E0CE0101960E94467EBE016F5F7F4F7C
:10B65000CE018E960E94917C182FCE0101960E94F9
:10B66000A77D1123A1F046E050E0BE01625D7F4F4F
:10B67000CE0101960E94BF1EBE016F5F7F4F83E720
:10B680009FE00E946E7DCE0101960E94A77D6DE92C
:10B6900077E0CE0101960E94467EBE016F5F7F4F2C
:10B6A000CE018E960E94917C182FCE0101960E94A9
:10B6B000A77D1123A1F042E050E0BE01625D7F4F03
:10B6C000CE0101960E94BF1EBE016F5F7F4F83E7D0
:10B6D0009FE00E946E7DCE0101960E94A77D809121
:10B6E000770F9091780F892B09F488CA63E77FE080
:10B6F000CE0101960E943D7E61E070E0CE01019690
:10B700000E942237CE0101960E94A77D77CA67E684
:10B7100077E0CE0182960E94467EBE016E5D7F4F2D
:10B72000CE018E960E94917C11E0811129C06EE5B8
:10B7300077E0CE014C960E94467EBE01645E7F4F4C
:10B74000CE018E960E94917C11E0811115C066E6B3
:10B7500077E0CE0101960E94467EBE016F5F7F4F6B
:10B76000CE018E960E94917C11E0811101C010E003
:10B77000CE0101960E94A77DCE014C960E94A77D26
:10B78000CE0182960E94A77D112309F4E6C067E6E8
:10B7900077E0CE0101960E94467EBE016F5F7F4F2B
:10B7A000CE018E960E94917C182FCE0101960E94A8
:10B7B000A77D112309F466C046E050E0BE01625D3A
:10B7C0007F4FCE0101960E94BF1EBE016F5F7F4F6B
:10B7D00083E79FE00E946E7DCE0101960E94A77DC7
:10B7E00083E79FE00E94ED7B6B017C0120E030E06D
:10B7F000A9010E94DBB218160CF08EC0A7019601B9
:10B8000060E070E08AE794E40E9433B20E94A5B23F
:10B810006093390270933A0280933B0290933C020A
:10B820008091390290913A02A0913B02B0913C0282
:10B83000181619061A061B0664F081E090E0A0E0D5
:10B84000B0E08093390290933A02A0933B02B09308
:10B850003C0280916C0290916D028130910509F05B
:10B8600068C08091390290913A02A0913B02B09158
:10B870003C028093350290933602A0933702B09336
:10B880003802BCC947E050E0BE01625D7F4FCE0187
:10B8900001960E94BF1EBE016F5F7F4F83E79FE04E
:10B8A0000E946E7DCE0101960E94A77D6EE774E036
:10B8B000CE0101960E94467EBE016F5F7F4FCE0192
:10B8C0008E960E94917C182FCE0101960E94A77D32
:10B8D000112331F081E090E090936D0280936C022F
:10B8E00064E776E0CE0101960E94467EBE016F5F5E
:10B8F0007F4FCE018E960E94917C182FCE0101962B
:10B900000E94A77D112309F46BCF82E090E0909311
:10B910006D0280936C0264CF81E090E0A0E0B0E023
:10B920008093390290933A02A0933B02B0933C0279
:10B9300077CF029709F062C98091390290913A025B
:10B94000A0913B02B0913C0280933102909332026D
:10B95000A0933302B093340251C96EE677E0CE0172
:10B960004C960E94467EBE01645E7F4FCE018E964D
:10B970000E94717C11E0811115C063E777E0CE0170
:10B9800001960E94467EBE016F5F7F4FCE018E966C
:10B990000E94917C11E0811101C010E0CE0101965E
:10B9A0000E94A77DCE014C960E94A77D112309F429
:10B9B0008DC268EF77E0CE0101960E94467EBE01FF
:10B9C0006F5F7F4FCE018E960E94917C182FCE0123
:10B9D00001960E94A77D112309F4FBC001E010E04D
:10B9E00010936D0200936C0210935D0200935C0251
:10B9F0006AEA75E083E79FE00E948A7B10935D020C
:10BA000000935C0281E090E0A0E0B0E08093390216
:10BA100090933A02A0933B02B0933C02809335028C
:10BA200090933602A0933702B093380263E77FE029
:10BA3000CE0101960E943D7E62E070E0CE0101964B
:10BA40000E942237CE0101960E94A77D67ED78E023
:10BA5000CE0101960E94347ECE0101960E94091B00
:10BA6000CE0101960E94A77D67EC78E0CE01019699
:10BA70000E94347ECE0101960E94A727CE01019636
:10BA80000E94A77D66ED76E083E79FE00E948A7BB7
:10BA900063E77FE0CE0101960E943D7E63E070E0A7
:10BAA000CE0101960E942237CE0101960E94A77D09
:10BAB00082E090E090936D0280936C0266EB78E0F8
:10BAC000CE0101960E94347ECE0101960E94091B90
:10BAD000CE0101960E94A77D6AEA78E0CE01019628
:10BAE0000E94347ECE0101960E94A727CE010196C6
:10BAF0000E94A77D6AEA75E083E79FE00E948A7B47
:10BB0000809144119091451197FF06C06EEA75E04F
:10BB100083E79FE00E948A7B63E77FE0CE01019686
:10BB20000E943D7E62E070E0CE0101960E942237C5
:10BB3000CE0101960E94A77D66ED76E083E79FE047
:10BB40000E948A7B82E090E090936D0280936C0269
:10BB500063E77FE0CE0101960E943D7E63E070E0E6
:10BB6000CE0101960E942237CE0101960E94A77D48
:10BB700084EF91E090936702809366026EE170E13A
:10BB80000E94680964E670E080E090E00E94ED8128
:10BB900081E090E090936D0280936C021092DA0243
:10BBA0001092D90282E090E0A0E0B0E08093C3025E
:10BBB0009093C402A093C502B093C6020E94148958
:10BBC0006093E3027093E4028093E5029093E602AF
:10BBD00015C86EE677E0CE0101960E94467EBE0152
:10BBE0006F5F7F4FCE018E960E94917C182FCE0101
:10BBF00001960E94A77D11110C94FE556EE774E02A
:10BC0000CE0101960E94467EBE016F5F7F4FCE013E
:10BC10008E960E94917C182FCE0101960E94A77DDE
:10BC2000112331F081E090E090936D0280936C02DB
:10BC300064E776E0CE0101960E94467EBE016F5F0A
:10BC40007F4FCE018E960E94917C182FCE010196D7
:10BC50000E94A77D112331F082E090E090936D0265
:10BC600080936C0281E090E0A0E0B0E08093390224
:10BC700090933A02A0933B02B0933C0280916C02F5
:10BC800090916D028130910509F099C090935D0209
:10BC900080935C0263E777E0CE0101960E94467EC6
:10BCA000BE016F5F7F4FCE018E960E94917C182F50
:10BCB000CE0101960E94A77D112319F146E050E0C4
:10BCC000BE01625D7F4FCE014C960E94BF1E6AE7A7
:10BCD00077E0CE0101960E94467EBE01645E7F4FF2
:10BCE000CE0101960E94C27CBC0183E79FE00E94C6
:10BCF000577DCE0101960E94A77DCE014C960E94F1
:10BD0000A77D8091390290913A02A0913B02B091B7
:10BD10003C028093350290933602A0933702B09391
:10BD200038026AEA75E083E79FE00E948A7B63E756
:10BD30007FE0CE0101960E943D7E62E070E0CE0180
:10BD400001960E942237CE0101960E94A77D69E9E3
:10BD500078E0CE0101960E94347ECE0101960E94C9
:10BD6000091BCE0101960E94A77D81E090E090938F
:10BD70005D0280935C0266ED76E083E79FE00E94BF
:10BD80008A7B63E77FE0CE0101960E943D7E63E0FF
:10BD900070E0CE0101960E942237CE0101960E94EA
:10BDA000A77D69E878E0CE0101960E94347ECE013D
:10BDB00001960E94A727CE0101960E94A77D80913F
:10BDC0006C0290916D02029711F00C94FE556AEA94
:10BDD00075E083E79FE00E948A7B809144119091F7
:10BDE000451197FF06C06EEA75E083E79FE00E9469
:10BDF0008A7B01E010E010935D0200935C0263E730
:10BE00007FE0CE0101960E943D7E62E070E0CE01AF
:10BE100001960E942237CE0101960E94A77D66ED11
:10BE200076E083E79FE00E948A7B68E778E0CE01B6
:10BE300001960E94347ECE0101960E94091BCE011C
:10BE400001960E94A77D63E77FE0CE0101960E94E4
:10BE50003D7E63E070E0CE0101960E942237CE0164
:10BE600001960E94A77D6CE678E0CE0101960E94C3
:10BE7000347ECE0101960E94A727CE0101960E9432
:10BE8000A77D8091441190914511919581959109DB
:10BE9000909345118093441110935D0200935C02CE
:10BEA00084EF91E090936702809366026EE170E107
:10BEB0000E94680964E670E080E090E00E94ED81F5
:10BEC00010936D0200936C020C94FE556CE777E0C2
:10BED000CE0188960E94467EBE01685D7F4FCE01EE
:10BEE0008E960E94917C01E081113DC06DEC77E05F
:10BEF000CE0182960E94467EBE016E5D7F4FCE01CE
:10BF00008E960E94917C01E0811129C06CEC77E053
:10BF1000CE014C960E94467EBE01645E7F4FCE01EC
:10BF20008E960E94917C01E0811115C063E877E054
:10BF3000CE0101960E94467EBE016F5F7F4FCE010B
:10BF40008E960E94917C01E0811101C000E0CE013B
:10BF500001960E94A77DCE014C960E94A77DCE013E
:10BF600082960E94A77DCE0188960E94A77D00231D
:10BF700009F41FC26CE777E0CE0101960E94467E6D
:10BF8000BE016F5F7F4FCE018E960E94917C082F7D
:10BF9000CE0101960E94A77D46E050E0011117C036
:10BFA0006DEC77E0CE0101960E94467EBE016F5F88
:10BFB0007F4FCE018E960E94917C082FCE01019674
:10BFC0000E94A77D002309F48BC042E050E0BE012F
:10BFD000625D7F4FCE0101960E94BF1EBE016F5F62
:10BFE0007F4F83E79FE00E946E7DCE0101960E9405
:10BFF000A77D8091770F9091780F892B11F40C9485
:10C00000FE556AE777E0CE014C960E94467EBE015F
:10C01000645E7F4F83E79FE00E94917C811114C092
:10C020006CEB78E0CE0101960E94467EBE016F5F08
:10C030007F4F83E79FE00E94917C11E0811110E027
:10C04000CE0101960E94A77DCE014C960E94A77D4D
:10C05000C12CD12C7601112309F46AC183E79FE03A
:10C060000E94ED7B6B017C0180916C0290916D02CE
:10C07000019709F09FC083E79FE00E94ED7B9B0141
:10C08000AC016091960B7091970B8091980B9091F9
:10C09000990B0E94C7B16093960B7093970B809396
:10C0A000980B9093990B8090960B9090970BA09083
:10C0B000980BB090990B20E030E044EB53E4C501BD
:10C0C000B4010E94DBB287FD86C020E030E044EB83
:10C0D00053E4C501B4010E94C6B14B015C01EBCF32
:10C0E00043E050E0BE01625D7F4FCE0101960E94A9
:10C0F000BF1EBE016F5F7F4F83E79FE00E946E7D92
:10C10000CE0101960E94A77D6EE774E0CE010196F4
:10C110000E94467EBE016F5F7F4FCE018E960E94C9
:10C12000917C082FCE0101960E94A77D0023B1F0DB
:10C1300081E090E090936D0280936C028091E10B1E
:10C140009091E20BA091E30BB091E40B8093960BDE
:10C150009093970BA093980BB093990B64E776E0BC
:10C16000CE0101960E94467EBE016F5F7F4FCE01D9
:10C170008E960E94917C082FCE0101960E94A77D89
:10C18000002309F436CF82E090E090936D02809313
:10C190006C028091DD0B9091DE0BA091DF0BB091D2
:10C1A000E00B8093960B9093970BA093980BB09312
:10C1B000990B1FCF83E79FE00E94ED7B9B01AC01B1
:10C1C0006091960B7091970B8091980B9091990BC1
:10C1D0000E94C6B160CF20E030E0A901C501B401E2
:10C1E0000E9419B087FF0BC020E030E044EB53E41D
:10C1F000C501B4010E94C7B14B015C01ECCF809234
:10C20000960B9092970BA092980BB092990B20E00E
:10C2100030E0A901C701B6010E94DBB287FD15C05D
:10C220006CEB78E0CE0101960E94467E63E77FE0EA
:10C23000CE0101960E94C27CBC0183E79FE00E9470
:10C24000577DCE0101960E94A77D20E030E0A90134
:10C25000C701B6010E9419B087FF6AC080916C02C5
:10C2600090916D02019799F520E030E0A901C70196
:10C27000B6010E94DBB218160CF092C020E030E04C
:10C2800040E251E4C701B6010E94C7B122E0AB0110
:10C29000BC01CE014C960E94AF7D6AE777E0CE01EB
:10C2A00001960E94467EBE01645E7F4FCE010196DC
:10C2B0000E94C27CBC0183E79FE00E94577DCE01B3
:10C2C00001960E94A77DCE014C960E94A77D809189
:10C2D0006C0290916D02019759F120E030E0A901C4
:10C2E000C701B6010E94DBB2B701A60118160CF017
:10C2F000705822E0CE014C960E94AF7D6AE777E04D
:10C30000CE0101960E94467EBE01645E7F4FCE0143
:10C3100001960E94C27CBC0183E79FE00E94577D8A
:10C32000CE0101960E94A77DCE014C960E94A77D6A
:10C3300081E090E090935D0280935C0263E77FE090
:10C34000CE0101960E943D7E62E070E0CE01019632
:10C350000E942237CE0101960E94A77D20E030E0A6
:10C36000A901C701B6010E9419B087FD02C00C9453
:10C37000FE5580916C0290916D02019711F00C9422
:10C38000FE5567E877E083E79FE00E948A7B63E7DA
:10C390007FE0CE0101960E943D7E62E070E0AEC972
:10C3A000A701960160E070E080E291E40E94C6B1CE
:10C3B0006DCF6CE877E0CE0182960E94467EBE018A
:10C3C0006E5D7F4FCE018E960E94917C11E08111AF
:10C3D00029C06BE877E0CE014C960E94467EBE01F4
:10C3E000645E7F4FCE018E960E94917C11E0811198
:10C3F00015C062E977E0CE0101960E94467EBE013B
:10C400006F5F7F4FCE018E960E94917C11E081116B
:10C4100001C010E0CE0101960E94A77DCE014C968E
:10C420000E94A77DCE0182960E94A77D112309F468
:10C430009BC0CE018E960E94037C6AEA75E083E77A
:10C440009FE00E948A7B6EE774E0CE0101960E9415
:10C45000467EBE016F5F7F4FCE018E960E94917C1B
:10C46000182FCE0101960E94A77D112331F081E0A3
:10C4700090E090936D0280936C0264E776E0CE01C9
:10C4800001960E94467EBE016F5F7F4FCE018E9661
:10C490000E94917C182FCE0101960E94A77D112346
:10C4A00091F082E090E090936D0280936C02809115
:10C4B00044119091451197FF06C06EEA75E083E73D
:10C4C0009FE00E948A7B81E090E090935D028093E0
:10C4D0005C0263E77FE0CE0101960E943D7E62E050
:10C4E00070E0CE0101960E942237CE0101960E9493
:10C4F000A77D6CE877E0CE0101960E94467EBE01E2
:10C500006F5F7F4FCE018E960E94917C182FCE01D7
:10C5100001960E94A77D45E050E0111102C046E05F
:10C5200050E0BE01625D7F4FCE0101960E94BF1EAA
:10C53000BE016F5F7F4F83E79FE00E946E7DCE015B
:10C5400001960E94A77D8091770F9091780F892B9B
:10C5500011F40C94FE5563E77FE0CE0101960E9432
:10C560003D7E63E070E0CAC86AE977E0CE0182965A
:10C570000E94467EBE016E5D7F4FCE018E960E9468
:10C58000917C11E0811129C069E977E0CE014C96D8
:10C590000E94467EBE01645E7F4FCE018E960E9451
:10C5A000917C11E0811115C060EA77E0CE0101961F
:10C5B0000E94467EBE016F5F7F4FCE018E960E9425
:10C5C000917C11E0811101C010E0CE0101960E9422
:10C5D000A77DCE014C960E94A77DCE0182960E9437
:10C5E000A77D112309F426C16AE977E0CE010196FF
:10C5F0000E94467EBE016F5F7F4FCE018E960E94E5
:10C60000917C182FCE0101960E94A77D112309F479
:10C6100043C045E050E0BE01625D7F4FCE01019610
:10C620000E94BF1EBE016F5F7F4F83E79FE00E94A5
:10C630006E7DCE0101960E94A77D8091770F90912B
:10C64000780F892B61F083E79FE00E94ED7B609378
:10C65000960B7093970B8093980B9093990BC090C7
:10C66000960BD090970BE090980BF090990B20E0F0
:10C6700030E044EB53E4C701B6010E94DBB287FD12
:10C6800055C020E030E044EB53E4C701B6010E94FE
:10C69000C6B16B017C01EBCF46E050E0BE01625DAC
:10C6A0007F4FCE0101960E94BF1EBE016F5F7F4F7C
:10C6B00083E79FE00E946E7DCE0101960E94A77DD8
:10C6C0006EE774E0CE0101960E94467EBE016F5F68
:10C6D0007F4FCE018E960E94917C182FCE0101963D
:10C6E0000E94A77D112331F081E090E090936D02CC
:10C6F00080936C0264E776E0CE0101960E94467E4C
:10C70000BE016F5F7F4FCE018E960E94917C182FE5
:10C71000CE0101960E94A77D112309F48ECF82E0FD
:10C7200090E090936D0280936C0287CF20E030E020
:10C73000A901C701B6010E9419B087FF0BC020E014
:10C7400030E044EB53E4C701B6010E94C7B16B016E
:10C750007C01ECCFC092960BD092970BE092980B95
:10C76000F092990B80916C0290916D02019771F497
:10C77000C092E10BD092E20BE092E30BF092E40B5B
:10C7800061E175E089E79FE00E948A7B8091960BCA
:10C790009091970BA091980BB091990B20916C02FE
:10C7A00030916D022230310571F48093DD0B90934E
:10C7B000DE0BA093DF0BB093E00B61E275E089E73D
:10C7C0009FE00E948A7B4091960B5091970B60915D
:10C7D000980B7091990B21E0CE014C960E94AF7D91
:10C7E00069E77FE0CE0101960E943D7EBE01645E56
:10C7F0007F4FCE0101960E94C27C6CE175E00E94E1
:10C80000AC7CBC0189E79FE00E94577DCE01019678
:10C810000E94A77DCE014C960E94A77D69E77FE02C
:10C82000CE0101960E943D7ECE0101960E94A7276F
:10C830000C94825B68EA77E0CE0182960E94467E85
:10C84000BE016E5D7F4FCE018E960E94917C11E0FD
:10C85000811129C067EA77E0CE014C960E94467E9E
:10C86000BE01645E7F4FCE018E960E94917C11E0E6
:10C87000811115C06DEA77E0CE0101960E94467ED7
:10C88000BE016F5F7F4FCE018E960E94917C11E0BA
:10C89000811101C010E0CE0101960E94A77DCE015A
:10C8A0004C960E94A77DCE0182960E94A77D1123FF
:10C8B00009F412C2C0903902D0903A02E0903B02D3
:10C8C000F0903C0263EB77E0CE0101960E94467E39
:10C8D000BE016F5F7F4FCE018E960E94917C182F14
:10C8E000CE0101960E94A77D112309F465C044E0A2
:10C8F00050E0BE01625D7F4FCE0101960E94BF1ED7
:10C90000BE016F5F7F4F83E79FE00E946E7DCE0187
:10C9100001960E94A77D80916C0290916D028130FA
:10C92000910509F093C0C0903502D0903602E09096
:10C930003702F090380281E090E0A0E0B0E0809310
:10C94000350290933602A0933702B093380280915B
:10C95000770F9091780F892B09F090C068EB77E002
:10C9600083E79FE00E948A7B8091770F9091780FF8
:10C97000892B81F063E77FE0CE0101960E943D7E26
:10C9800070E060E0CE0101960E942237CE01019650
:10C990000E94A77D80916C0290916D02813091057B
:10C9A00009F08CC1C0923502D0923602E092370273
:10C9B000F09238020C94FE5545E050E0BE01625DF5
:10C9C0007F4FCE0101960E94BF1EBE016F5F7F4F59
:10C9D00083E79FE00E946E7DCE0101960E94A77DB5
:10C9E0006EE774E0CE0101960E94467EBE016F5F45
:10C9F0007F4FCE018E960E94917C182FCE0101961A
:10CA00000E94A77D112331F081E090E090936D02A8
:10CA100080936C0264E776E0CE0101960E94467E28
:10CA2000BE016F5F7F4FCE018E960E94917C182FC2
:10CA3000CE0101960E94A77D112309F46CCF82E0FC
:10CA400090E090936D0280936C0265CF029709F09D
:10CA50007ECFC0903102D0903202E0903302F0904D
:10CA6000340281E090E0A0E0B0E080933102909346
:10CA70003202A0933302B093340269CF6EEB77E0B9
:10CA8000CE0101960E94467EBE016F5F7F4F83E715
:10CA90009FE00E94717C182FCE0101960E94A77D15
:10CAA000112309F477CF83E79FE00E94ED7B20E01C
:10CAB00030E0A9010E9419B0811128C080916C0258
:10CAC00090916D02019731F461EC77E083E79FE08C
:10CAD0000E948A7B80916C0290916D02029731F4E2
:10CAE00068EB77E083E79FE00E948A7B8091770F75
:10CAF0009091780F892B09F44DCF63E77FE0CE0149
:10CB000001960E943D7E61E070E03CCF67E476E0F4
:10CB1000CE0101960E94467EBE016F5F7F4F83E784
:10CB20009FE00E94717C182FCE0101960E94A77D84
:10CB3000112309F42FCF41E050E063E77FE0CE01FD
:10CB400001960E94BF1ECE0101960E94ED7B4B0113
:10CB50005C01CE0101960E94A77D20E030E0A90192
:10CB6000C501B4010E9419B0181634F0812C912C23
:10CB700090E8A92E9FE3B92E00916C0210916D02EE
:10CB80000130110509F075C0A501940160E070E461
:10CB90008CE995E40E9433B260932D0270932E02CB
:10CBA00080932F029093300260933C1170933D115B
:10CBB00080933E1190933F116093290270932A0253
:10CBC00080932B0290932C02B801CE014C960E94C8
:10CBD000947B66EC77E0CE0101960E94467EBE0112
:10CBE000645E7F4FCE0101960E94C27CBC01CE01E3
:10CBF00082960E943D7ECE0182960E94201BCE012D
:10CC000082960E94A77DCE0101960E94A77DCE014B
:10CC10004C960E94A77D6AE578E0CE0101960E94BD
:10CC2000347ECE0101960E94201BCE0101960E9407
:10CC3000A77D40912D0250912E0260912F0270919C
:10CC4000300225E0CE0101960E94AF7DCE01019613
:10CC50000E94091BCE0101960E94A77D84EF91E0FE
:10CC600090936702809366026EE170E10E9468090A
:10CC700091CE0230110509F0A7CFA501940160E023
:10CC800070E48CE196E40E9433B260932D027093BD
:10CC90002E0280932F029093300260934011709384
:10CCA0004111809342119093431160932502709338
:10CCB0002602809327029093280286CF029711F0D4
:10CCC0000C94FE55C0923102D0923202E0923302AF
:10CCD000F09234020C94FE556BEC77E0CE01829614
:10CCE0000E94467EBE016E5D7F4FCE018E960E94F1
:10CCF000917C11E0811129C06AEC77E0CE014C965D
:10CD00000E94467EBE01645E7F4FCE018E960E94D9
:10CD1000917C11E0811115C060ED77E0CE010196A4
:10CD20000E94467EBE016F5F7F4FCE018E960E94AD
:10CD3000917C11E0811101C010E0CE0101960E94AA
:10CD4000A77DCE014C960E94A77DCE0182960E94BF
:10CD5000A77D112309F429C18AA99BA9059710F47D
:10CD60000C94FE5544E050E0BE01625D7F4FCE0161
:10CD700001960E94BF1EBE016F5F7F4F83E79FE059
:10CD80000E946E7DCE0101960E94A77D6BEC77E03C
:10CD9000CE0101960E94467EBE016F5F7F4FCE019D
:10CDA0008E960E94917C182FCE0101960E94A77D3D
:10CDB000112309F49BC044E050E0BE01625D7F4F47
:10CDC000CE0101960E94BF1EBE016F5F7F4F83E7B9
:10CDD0009FE00E946E7DCE0101960E94A77D83E7B1
:10CDE0009FE00E94ED7B20E030E0A9010E94DBB2D1
:10CDF000181614F00C94FE5583E79FE00E94ED7B1B
:10CE000060932D0270932E0280932F029093300234
:10CE100020916C0230916D022130310509F0B0C0D3
:10CE200060933C1170933D1180933E1190933F119C
:10CE30006093290270932A0280932B0290932C0214
:10CE4000B901CE014C960E94947B66EC77E0CE014E
:10CE500001960E94467EBE01645E7F4FCE01019620
:10CE60000E94C27CBC01CE0182960E943D7ECE0112
:10CE700082960E94201BCE0182960E94A77DCE0141
:10CE800001960E94A77DCE014C960E94A77D68E482
:10CE900078E0CE0101960E94347ECE0101960E9478
:10CEA000201BCE0101960E94A77D40912D0250913A
:10CEB0002E0260912F027091300225E0CE01019682
:10CEC0000E94AF7DCE0101960E94091BCE01019602
:10CED0000E94A77D84EF91E09093670280936602A1
:10CEE0006EE170E10E9468090C94FE5545E050E047
:10CEF000BE01625D7F4FCE0101960E94BF1EBE0142
:10CF00006F5F7F4F83E79FE00E946E7DCE010196A9
:10CF10000E94A77D6EE774E0CE0101960E94467ED6
:10CF2000BE016F5F7F4FCE018E960E94917C182FBD
:10CF3000CE0101960E94A77D112331F081E090E09F
:10CF400090936D0280936C0264E776E0CE010196C7
:10CF50000E94467EBE016F5F7F4FCE018E960E947B
:10CF6000917C182FCE0101960E94A77D112309F410
:10CF700036CF82E090E090936D0280936C022FCFC9
:10CF80002230310509F05CCF60934011709341115C
:10CF9000809342119093431160932502709326026F
:10CFA00080932702909328024BCF69ED75E0CE0164
:10CFB0004C960E94467EBE01645E7F4FCE018E96E7
:10CFC0000E94917C11E0811115C066ED77E0CE01E1
:10CFD00001960E94467EBE016F5F7F4FCE018E9606
:10CFE0000E94917C11E0811101C010E0CE010196F8
:10CFF0000E94A77DCE014C960E94A77D112309F4C3
:10D0000063C069ED75E0CE0101960E94467EBE01C7
:10D010006F5F7F4FCE018E960E94917C182FCE01BC
:10D0200001960E94A77D112399F042E050E067E944
:10D030007FE0CE0101960E94BF1EBE016F5F7F4F51
:10D0400083E79FE00E946E7DCE0101960E94A77D3E
:10D0500066ED77E0CE0101960E94467EBE016F5FCD
:10D060007F4FCE018E960E94917C182FCE010196A3
:10D070000E94A77D112399F043E050E067E97FE02B
:10D08000CE0101960E94BF1EBE016F5F7F4F83E7F6
:10D090009FE00E946E7DCE0101960E94A77D83E7EE
:10D0A0009FE00E94F87B653B710510F40C94FE55DF
:10D0B00065E378E0CE0101960E94347ECE010196B0
:10D0C0000E94201B0C94825B6AED77E0CE010196F2
:10D0D0000E94467EBE016F5F7F4FCE018E960E94FA
:10D0E000917C182FCE0101960E94A77D112309F48F
:10D0F00074C026E030E044E050E067E97FE0CE0114
:10D1000001960E945B7EBE016F5F7F4F83E79FE0C9
:10D110000E946E7DCE0101960E94A77D67E476E0B5
:10D12000CE0101960E94467E40919B0F50919C0F2C
:10D130008D819E81481B590BBE016F5F7F4F87E930
:10D140009FE00E94ABA4AC014F5F5F4F67E97FE0B7
:10D15000CE014C960E94BF1EBE01645E7F4F83E7E6
:10D160009FE00E946E7DCE014C960E94A77DCE016D
:10D1700001960E94A77D83E79FE00E94ED7B88E2F5
:10D18000EEE6FBE0A5EFB0E101900D928A95E1F7A4
:10D1900084EF91E090936702809366026EE170E104
:10D1A0000E94680964E178E089E79FE00E94327D8F
:10D1B00044E050E067E97FE0CE0101960E94BF1E87
:10D1C000BE016F5F7F4F89E79FE00E942B7DCE01FC
:10D1D00001960E94A77D0C94F2526EED77E0CE018D
:10D1E00001960E94467EBE016F5F7F4FCE018E96F4
:10D1F0000E94917C182FCE0101960E94A77D1111EB
:10D200000C94D85866EE77E0CE0101960E94467ED7
:10D21000BE016F5F7F4FCE018E960E94917C182FCA
:10D22000CE0101960E94A77D112371F141E068E9CA
:10D2300072E0CE0101960E947B95BE016F5F7F4F29
:10D2400082E891E10E94301E82E891E10E94690D1E
:10D25000811104C068EC77E00C94B65182E891E14A
:10D260000E94AE07892B51F082E891E10E94D30D14
:10D27000682F85E29DE00E944175F0CF82E891E140
:10D280000E94750D0C94DC486DEE77E0CE0101969E
:10D290000E94467EBE016F5F7F4FCE018E960E9438
:10D2A000917C182FCE0101960E94A77D1123E9F0F1
:10D2B0008DB79EB7825391400FB6F8949EBF0FBEB4
:10D2C0008DBFADB7BEB7119682E391E0EEE1F0E11C
:10D2D00001900D920197E1F70E94D4320FB6F894B5
:10D2E000DEBF0FBECDBF0C94DC4866EF77E0CE0109
:10D2F00001960E94467EBE016F5F7F4FCE018E96E3
:10D300000E94917C182FCE0101960E94A77D1123C7
:10D3100009F457C0EDB7FEB7E253F1400FB6F894E9
:10D32000FEBF0FBEEDBFADB7BEB7119682E391E071
:10D33000EEE1F0E101900D920197E1F70E94532C8C
:10D340000FB6F894DEBF0FBECDBF63E078E0CE012C
:10D3500001960E94347EADB7BEB7A253B1400FB65E
:10D36000F894BEBF0FBEADBF119682E391E0EEE12F
:10D37000F0E101900D920197E1F70E9459240FB658
:10D38000F894DEBF0FBECDBF8DB79EB782539140DC
:10D390000FB6F8949EBF0FBE8DBFADB7BEB7119646
:10D3A00082E391E0EEE1F0E101900D920197E1F767
:10D3B0000E94D4320FB6F894DEBF0FBECDBF0C94DE
:10D3C000E14D68EF77E0CE0101960E94467EBE01F6
:10D3D0006F5F7F4FCE018E960E94917C182FCE01F9
:10D3E00001960E94A77D1123F9F061EF77E0CE014D
:10D3F00001960E94347EBE016F5F7F4FCE014C9636
:10D400000E943D7ECE014C960E94091BCE014C9697
:10D410000E94A77DEDB7FEB7E253F1400FB6F89436
:10D42000FEBF0FBEEDBFB9CF6CEF77E0CE01019626
:10D430000E94467EBE016F5F7F4FCE018E960E9496
:10D44000917C182FCE0101960E94A77D112309F42B
:10D45000F5C065ED77E0CE0182960E94347EBE0174
:10D460006E5D7F4FCE0101960E943D7EAE014F5F03
:10D470005F4F62E070E08FE792E00E94062E182F67
:10D48000CE0101960E94A77D111122C0BE016E5DE2
:10D490007F4FCE014C960E943D7E60E078E0CE0149
:10D4A0004C960E94AC7C6AEC7FE00E94C27CBC017E
:10D4B000CE0101960E943D7ECE0101960E94091B7D
:10D4C000CE0101960E94A77DCE014C960E94A77DB9
:10D4D00068EE73E080E090E00E94ED81BE016E5D39
:10D4E0007F4FCE0101960E943D7EAE014F5F5F4FA0
:10D4F00063E070E082E792E00E94062E182FCE01D2
:10D5000001960E94A77D111122C0BE016E5D7F4F62
:10D51000CE014C960E943D7E60E178E0CE014C96B3
:10D520000E94AC7C6AEC7FE00E94C27CBC01CE0110
:10D5300001960E943D7ECE0101960E94091BCE01FC
:10D5400001960E94A77DCE014C960E94A77D68EEB1
:10D5500073E080E090E00E94ED816EEB7FE0CE0111
:10D5600001960E943D7EAE014F5F5F4F61E070E02B
:10D5700082EB92E00E94062E182FCE0101960E94A7
:10D58000A77D111121C06EEB7FE0CE014C960E9469
:10D590003D7E60E178E0CE014C960E94AC7C6AEC66
:10D5A0007FE00E94C27CBC01CE0101960E943D7EBC
:10D5B000CE0101960E94091BCE0101960E94A77D13
:10D5C000CE014C960E94A77D68EE73E080E090E06B
:10D5D0000E94ED8180914F0C882311F40C94F1543A
:10D5E00043E162EB72E0CE0101960E947B95BE01A1
:10D5F0006F5F7F4F88EB91E10E94301E88EB91E1D5
:10D600000E94690D882311F40C94F1546EEB7FE0B5
:10D6100088EB91E10E94767F66E970E080E090E01F
:10D620000E94ED8188EB91E10E94750D62E370E04C
:10D6300080E090E00E94ED810C94F1546CE178E080
:10D64000CE0101960E94467EBE016F5F7F4FCE01E4
:10D650008E960E94917C182FCE0101960E94A77D84
:10D660001123C1F00CEA1BE082EBE82E8BE0F82ED0
:10D67000D8018C910E5F1F4F60E00E947A806CE2AF
:10D6800071E080E090E00E94ED81E016F10681F704
:10D690000C94DC4860E278E0CE0101960E94467E60
:10D6A000BE016F5F7F4FCE018E960E94917C182F36
:10D6B000CE0101960E94A77D1123A9F00CEA1BE080
:10D6C000F80180810E5F1F4F61E00E947A806CE25A
:10D6D00071E080E090E00E94ED81FBE0023B1F07DB
:10D6E00079F70C94DC4865E278E0CE0101960E945F
:10D6F000467EBE016F5F7F4FCE018E960E94917C69
:10D70000182FCE0101960E94A77D112311F40C94CD
:10D71000DC4827E030E046E050E067E97FE0CE01FA
:10D7200001960E945B7EBE016F5F7F4F83E79FE0A3
:10D730000E946E7DCE0101960E94A77D83E79FE047
:10D740000E94F87B672B71F410926D0B67E97FE004
:10D75000CE0101960E943D7ECE0101960E94752168
:10D760000C948A5781E080936D0BF0CF2F923F92FB
:10D770004F925F926F927F928F929F92AF92BF92E1
:10D78000CF92DF92EF92FF920F931F93CF93DF938D
:10D7900000D000D01F921F92CDB7DEB760918E02ED
:10D7A00070918F0280918C0290918D020E94371BA4
:10D7B00084E1482E512C612C712C312C212C8FEFBF
:10D7C000281A380AC301B2010E94ED8160918E02CD
:10D7D00070918F0280918C0290918D020E94371B74
:10D7E0008C0183E02816310434F08EE128163104D0
:10D7F00044F4012B51F084E1480E511C611C711C52
:10D80000DECF0115110509F0A6C080918C02909120
:10D810008D028B30910509F086C080905411909054
:10D820005511A0905611B0905711C0905011D09042
:10D830005111E0905211F090531164E670E080E0D5
:10D8400090E00E94ED8161E275E0CE0101960E94B8
:10D85000347ECE0101960E94A727CE0101960E9438
:10D86000A77D61E082E00E94D88C21E0B501A4018F
:10D87000CE0101960E94AF7DBE016F5F7F4F84EDA8
:10D8800091E10E94687FCE0101960E94A77D6FED15
:10D8900084ED91E10E94B08C6CE175E084ED91E142
:10D8A0000E948A7F20E0B701A601CE0101960E9466
:10D8B000AF7DBE016F5F7F4F84ED91E10E94687F75
:10D8C000CE0101960E94A77D6CE278E084ED91E1A3
:10D8D0000E94607F89829A82AB82BC82CD82DE8286
:10D8E000EF82F88629813A814B815C816D817E814E
:10D8F0008F81988528960FB6F894DEBF0FBECDBFF6
:10D90000DF91CF911F910F91FF90EF90DF90CF901B
:10D91000BF90AF909F908F907F906F905F904F904F
:10D920003F902F9008958631910509F476CF0C979A
:10D9300009F083CF8090920A9090930AA090940A65
:10D94000B090950AC0908E0AD0908F0AE090900A0D
:10D95000F090910A72CF0F3F8FEF1807CCF06EE076
:10D9600075E0CE0101960E94347E4AE050E070E0FE
:10D9700060E0CE0101960E94D226CE0101960E945F
:10D98000A77D6BEE74E089E79FE00E94327D32C094
:10D990000E3F8FEF1807B9F16DED74E0CE010196DF
:10D9A0000E94347E4AE050E070E060E0CE010196D3
:10D9B0000E94D226CE0101960E94A77D6EEC74E0F3
:10D9C00089E79FE00E94327DB801CE0101960E9456
:10D9D000947BBE016F5F7F4F89E79FE00E942B7DA4
:10D9E000CE0101960E94A77D68EB74E089E79FE075
:10D9F0000E94D57C19821A821B821C821D821E8283
:10DA00001F8218866FCF6DEA74E0CE0101960E94E6
:10DA1000347E4AE050E070E060E0CE0101960E9462
:10DA2000D226CE0101960E94A77D6DE874E0ABCFAF
:10DA30002F923F924F925F926F927F928F929F921E
:10DA4000AF92BF92CF92DF92EF92FF920F931F930C
:10DA5000CF93DF93CDB7DEB7AC970FB6F894DEBFA8
:10DA60000FBECDBF8C017B018091DB0B9091DC0B55
:10DA700001969093DC0B8093DB0B2091F80B222313
:10DA800041F06AE070E00E94F1B2181619060CF439
:10DA9000C0C281E08093F80B1092DC0B1092DB0B7C
:10DAA00050E040E06EE174E0C8010E947A1E82E01E
:10DAB000E816F10409F4C6C26DE174E088EB9FE05A
:10DAC0000E948A7B60918E0270918F0280918C02FD
:10DAD00090918D020E94371B1C0160E37BE0C8011E
:10DAE0000E94611E6EE278E0C8010E94607F6EE5D0
:10DAF00071E1CE0101960E943D7EBE016F5F7F4FB6
:10DB0000C8010E94687FCE0101960E94A77D67E34D
:10DB100078E0C8010E94607F68E176E0C8010E9459
:10DB20008A7F64E671E1CE0101960E943D7EBE01CE
:10DB30006F5F7F4FC8010E94687F6EE076E0C8018A
:10DB40000E948A7F66E770E1CE0109960E94467EB8
:10DB5000BE01675F7F4FC8010E94687F61E076E089
:10DB6000C8010E948A7F6EED70E1CE010F960E947F
:10DB7000467EBE01615F7F4FC8010E94687F6AEFE9
:10DB800075E0C8010E948A7FCE010F960E94A77D92
:10DB9000CE0109960E94A77DCE0101960E94A77D25
:10DBA0000E94BC8428EE33E040E050E00E9463B164
:10DBB00029013A0160EF75E0C8010E948A7FCE0119
:10DBC00001960E942222BE016F5F7F4FC8010E9412
:10DBD000687FCE0101960E94A77DC301B20120E1BA
:10DBE0003EE040E050E00E9485B14B015C01B9018C
:10DBF000CE0187960E94CB1E4CE3C42ED12CE12C83
:10DC0000F12CC501B401A70196010E9485B1B901AB
:10DC1000CE0101960E94CB1E64E077E0CE0109960A
:10DC20000E94467EBE016F5F7F4FCE0109960E9423
:10DC3000C27CBC01CE0187960E942B7DCE01099645
:10DC40000E94A77DCE0101960E94A77DC301B2016B
:10DC5000A70196010E9485B1CE0101960E94CB1EBC
:10DC600064E077E0CE0109960E94467EBE016F5FB8
:10DC70007F4FCE0109960E94C27CBC01CE018796DF
:10DC80000E942B7DCE0109960E94A77DCE010196B0
:10DC90000E94A77D6DE378E0CE0109960E94467E42
:10DCA000BE01695D7F4FCE0109960E94C27C60E48F
:10DCB00078E00E94AC7CBC01CE0101960E943D7EC2
:10DCC000BE016F5F7F4FC8010E94687FCE01019641
:10DCD0000E94A77DCE0109960E94A77D6EE478E0A0
:10DCE000C8010E94607FCE0101960E94011AB8010E
:10DCF000CE0101960E94027F69E478E0C8010E948B
:10DD00004C7F0E94B66B29833A834B835C836D837F
:10DD10007E838F83988749815A816B817C8121E042
:10DD2000CE010F960E94AF7DBE01615F7F4FCE0195
:10DD300009960E943D7E66E578E0CE0109960E9434
:10DD4000AC7CBC0188EB9FE00E94577DCE01099618
:10DD50000E94A77DCE010F960E94A77D6DE578E019
:10DD6000CE010F960E94467E68EB7FE0CE010F96B3
:10DD70000E94C27CBC01CE0109960E943D7EBE017C
:10DD8000675F7F4FC8010E94687FCE0109960E949D
:10DD9000A77DCE010F960E94A77D4D815E816F8188
:10DDA000788521E0CE0109960E94AF7DBE01675FB4
:10DDB0007F4F88EB9FE00E946E7DCE0109960E9406
:10DDC000A77D6FE678E0CE010F960E94467E68EB55
:10DDD0007FE0CE010F960E94C27C60E878E00E944E
:10DDE000AC7CBC01CE0109960E943D7EBE01675FFE
:10DDF0007F4FC8010E94687FCE0109960E94A77DCF
:10DE0000CE010F960E94A77D4091E10B5091E20B4D
:10DE10006091E30B7091E40B22E0CE010F960E941B
:10DE2000AF7D67E878E0CE0145960E94467EBE0150
:10DE3000615F7F4FCE0145960E94C27C69E978E020
:10DE40000E94AC7CBC01CE0109960E943D7EBE01C1
:10DE5000675F7F4FC8010E94687FCE0109960E94CC
:10DE6000A77DCE0145960E94A77DCE010F960E9408
:10DE7000A77D4091DD0B5091DE0B6091DF0B70911F
:10DE8000E00B22E0CE010F960E94AF7D62EA78E0BF
:10DE9000CE0145960E94467EBE01615F7F4FCE0156
:10DEA00045960E94C27C69E978E00E94AC7CBC0186
:10DEB000CE0109960E943D7EBE01675F7F4FC8017B
:10DEC0000E94687FCE0109960E94A77DCE014596EB
:10DED0000E94A77DCE010F960E94A77DE6EF2E1629
:10DEE000EFEF3E062CF46BE27CE0C8010E94611E5D
:10DEF00068E07BE0C8010E94611E9EE1E92E90E18E
:10DF0000F92E27EDA22E22E0B22ECC24C394D12CE0
:10DF10004701F8E08F0E911C82E0A80EB11C8091A1
:10DF20001E1090911F108C159D050CF464C0B60155
:10DF3000CE010F960E94947B68EC77E0CE01459667
:10DF40000E94467EBE01615F7F4FCE0145960E94D2
:10DF5000C27C64E476E00E94AC7CBC01CE010996F0
:10DF60000E943D7EBE01675F7F4FC8010E94687FAF
:10DF7000B701645E7F4FCE014B960E94467EBE0184
:10DF8000655E7F4FC8010E94687F60EB78E0C80142
:10DF90000E94607FF50160817181660F771F660FB7
:10DFA000771F665D7F4ECE0181960E94467EBE0140
:10DFB0006F5D7F4FC8010E94687F65EB78E0C80104
:10DFC0000E94607FCE0181960E94A77DCE014B9674
:10DFD0000E94A77DCE0109960E94A77DCE0145969D
:10DFE0000E94A77DCE010F960E94A77DFFEFCF1A5A
:10DFF000DF0A74018DCFCE0187960E94A77D81E054
:10E000008093520C69EE7BE0C8010E94611E109261
:10E01000F80BAC960FB6F894DEBF0FBECDBFDF9104
:10E02000CF911F910F91FF90EF90DF90CF90BF9015
:10E03000AF909F908F907F906F905F904F903F90A8
:10E040002F9008956BE27CE0C8010E94611EDACF38
:10E050008F929F92AF92BF92CF92DF92EF92FF92F8
:10E060000F931F93CF93DF93CDB7DEB7A0970FB673
:10E07000F894DEBF0FBECDBF6DE174E082EE9FE08D
:10E080000E948A7B6DE174E086ED9FE00E948A7BAE
:10E0900048E4842E42E0942E5EE1C52E50E1D52E58
:10E0A00061EDA62E62E0B62E77EDE72E72E0F72E38
:10E0B00001E010E0F40181919191A191B1914F01A2
:10E0C000892B8A2B8B2B19F5F70182819381F5011E
:10E0D0002081318182179307D1F0880F991FFC01AD
:10E0E000E759F44FD801AA0FBB1FA655B44F608162
:10E0F0008C910E947A80F70182819381F50191834E
:10E10000808364E670E080E090E00E94ED81F5019C
:10E11000619171915F0180911E1090911F10801785
:10E1200091070CF4E2C2CE0145960E94947BB8019F
:10E13000CE010F960E94947BB601645E7F4FCE01A4
:10E1400009960E94467E64E476E0CE0101960E9424
:10E15000467EBE01675F7F4FCE0101960E94C27C62
:10E160006BEB78E00E94AC7CBE01615F7F4F0E9448
:10E17000C27C67E476E00E94AC7CBE016B5E7F4FA0
:10E180000E94C27CBC0182EE9FE00E942B7DCE01EA
:10E1900001960E94A77DCE0109960E94A77DCE011F
:10E1A0000F960E94A77DCE0145960E94A77D0F5F26
:10E1B0001F4FF8E0CF0ED11C22E0E20EF11C04301C
:10E1C000110509F077CFE0913811F0913911EE0F78
:10E1D000FF1FE153FD4F60817181CE0101960E94C6
:10E1E000947B46E050E0BE016F5F7F4FCE01099601
:10E1F0000E94C722BE01675F7F4F86ED9FE00E94AD
:10E200002B7DCE0109960E94A77DCE0101960E942A
:10E21000A77DE0913A11F0913B11EE0FFF1FE15302
:10E22000FD4F60817181CE0101960E94947B46E092
:10E2300050E0BE016F5F7F4FCE0109960E94C7225A
:10E24000BE01675F7F4F86ED9FE00E942B7DCE0170
:10E2500009960E94A77DCE0101960E94A77D64E4E5
:10E2600076E0CE0145960E94467E0E94BC8428EE50
:10E2700033E040E050E00E9463B169017A016DE152
:10E2800074E0CE014B960E94467E6DE174E088EE0C
:10E290009FE00E948A7BCE0101960E94222244E1E7
:10E2A00050E0BE016F5F7F4FCE0109960E94C722EA
:10E2B000BE01675F7F4F88EE9FE00E946E7DCE01BA
:10E2C00009960E94A77DCE0101960E94A77D2AE0B3
:10E2D000B701A601CE0109960E94E57D48E050E015
:10E2E000BE01675F7F4FCE010F960E94C72268EE86
:10E2F0007FE0CE0101960E943D7EBE01615F7F4FAF
:10E30000CE0101960E94C27CBC018CED9FE00E9470
:10E31000577DCE0101960E94A77DCE010F960E94E7
:10E32000A77DCE0109960E94A77D2AE0B701A6012C
:10E33000CE0109960E94E57D6EEB78E0CE01019654
:10E340000E94467EBE01675F7F4FCE0101960E940C
:10E35000C27CBE016B5E7F4F0E94C27CBC0188EE16
:10E360009FE00E942B7DCE0101960E94A77DCE01E9
:10E3700009960E94A77D4091E10B5091E20B6091BC
:10E38000E30B7091E40B21E0CE0101960E94AF7D7A
:10E39000BE016F5F7F4FCE014B960E946E7DCE0116
:10E3A00001960E94A77D65EC78E0CE0101960E945F
:10E3B000467EBE01655E7F4FCE0101960E94C27C03
:10E3C000BE016B5E7F4F0E94C27CBC0188EE9FE065
:10E3D0000E942B7DCE0101960E94A77DBE01655E45
:10E3E0007F4FCE0101960E943D7E46E050E0BE0187
:10E3F0006F5F7F4FCE0109960E94C722BE01675F03
:10E400007F4F8CED9FE00E942B7DCE0109960E94EC
:10E41000A77DCE0101960E94A77D4091DD0B509112
:10E42000DE0B6091DF0B7091E00B21E0CE010196D5
:10E430000E94AF7DBE016F5F7F4FCE014B960E9461
:10E440006E7DCE0101960E94A77D63ED78E0CE013E
:10E4500001960E94467EBE01655E7F4FCE01019609
:10E460000E94C27CBE016B5E7F4F0E94C27CBC01D9
:10E4700088EE9FE00E942B7DCE0101960E94A77D31
:10E48000BE01655E7F4FCE0101960E943D7E46E053
:10E4900050E0BE016F5F7F4FCE0109960E94C722F8
:10E4A000BE01675F7F4F8CED9FE00E942B7DCE0108
:10E4B00009960E94A77DCE0101960E94A77D6091DA
:10E4C0008E0270918F0280918C0290918D020E9439
:10E4D000371B9093EE0B8093ED0B892B71F06091BD
:10E4E0008E0270918F0280918C0290918D020E9419
:10E4F000371B9093EE0B8093ED0B8091ED0B909179
:10E50000EE0B8C3F9F4F0CF410C10E94B66B298319
:10E510003A834B835C836D837E838F8398874981A5
:10E520005A816B817C8121E0CE0109960E94AF7DEA
:10E53000BE01675F7F4FCE014B960E946E7DCE017C
:10E5400009960E94A77D6DED78E0CE0109960E94A4
:10E55000467EBE01655E7F4FCE0109960E94C27C59
:10E56000BE016B5E7F4F0E94C27CBC0188EE9FE0C3
:10E570000E942B7DCE0109960E94A77DBE01655E9B
:10E580007F4FCE0109960E943D7E46E050E0BE01DD
:10E59000675F7F4FCE010F960E94C722BE01615F69
:10E5A0007F4F8CED9FE00E942B7DCE010F960E9445
:10E5B000A77DCE0109960E94A77D4D815E816F8166
:10E5C000788521E0CE0109960E94AF7DBE01675F8C
:10E5D0007F4FCE014B960E946E7DCE0109960E9420
:10E5E000A77D68EE78E0CE0109960E94467EBE01C6
:10E5F000655E7F4FCE0109960E94C27CBE016B5EB4
:10E600007F4F0E94C27CBC0188EE9FE00E942B7D60
:10E61000CE0109960E94A77DBE01655E7F4FCE01A7
:10E6200009960E943D7E46E050E0BE01675F7F4F45
:10E63000CE010F960E94C722BE01615F7F4F8CED15
:10E640009FE00E942B7DCE010F960E94A77DCE01F8
:10E6500009960E94A77D62EE7FE088EE9FE00E940F
:10E660002B7D64E476E0CE0101960E94467E66ED45
:10E670007FE0CE0101960E94C27CBC018CED9FE040
:10E680000E942B7DCE0101960E94A77D6CED7FE05C
:10E69000CE0101960E943D7ECE0101960E94091B8B
:10E6A000CE0101960E94A77D6AE070E080E090E0D4
:10E6B0000E94ED81CE014B960E94A77DCE0145962A
:10E6C0000E94A77DA0960FB6F894DEBF0FBECDBF07
:10E6D000DF91CF911F910F91FF90EF90DF90CF903E
:10E6E000BF90AF909F908F900895CE0145960E9465
:10E6F000947BB801CE010F960E94947BB6016C5EAC
:10E700007F4FCE0109960E94467E64E476E0CE01FA
:10E7100001960E94467EBE01675F7F4FCE01019643
:10E720000E94C27C6AEB78E01DCD6EEE78E088EE48
:10E730009FE00E94217D6DEF78E08CED9FE00E94CC
:10E74000217D64E079E088EE9FE00E94217D6DEFFD
:10E7500078E08CED9FE00E94217D7DCFBF92CF922B
:10E76000DF92EF92FF920F931F93CF93DF93CDB77A
:10E77000DEB7C455D1090FB6F894DEBF0FBECDBFCA
:10E780006C018B0165965FAF4EAF65978091DB0B97
:10E790009091DC0B01969093DC0B8093DB0B8091C6
:10E7A000F80B81113CC0BB24B394B092F80B1092CB
:10E7B000DC0B1092DB0B6DE174E0CE01895B9F4FA7
:10E7C0000E94467E6DE174E0CE01835B9F4F0E9404
:10E7D000467E50E040E06EE174E0C6010E947A1E81
:10E7E0000130110509F0A6C06DE174E088EE9FE0EC
:10E7F0000E948A7B6596EEADFFAD659780818111A1
:10E8000024C00E942870B092520CCE01835B9F4FAF
:10E810000E94A77DCE01895B9F4F0E94A77D0FB606
:10E82000F894DEBF0FBECDBFCC5ADF4F0FB6F894C1
:10E83000DEBF0FBECDBFDF91CF911F910F91FF9033
:10E84000EF90DF90CF90BF9008956596EEADFFAD4D
:10E8500065978081882309F467C000E210E09E017B
:10E860002F5F3F4F40E250E0BE016F5D7F4FCE0112
:10E870008D5A9F4F0E946B78049739F3BE016F5DEC
:10E880007F4FCE018F5B9F4F0E94467EBE016F5B24
:10E890007F4FCE01895B9F4F0E946E7DCE018F5BC3
:10E8A0009F4F0E94A77DBE016F5F7F4FCE018F5BA0
:10E8B0009F4F0E94467EBE016F5B7F4FCE01835B00
:10E8C0009F4F0E946E7DCE018F5B9F4F0E94A77D60
:10E8D000BE01695B7F4F88EE9FE00E942B7D6396AF
:10E8E0008EAD9FAD6397892B09F4AFCF67E476E0D7
:10E8F000CE018F5B9F4F0E94467EBE01635B7F4FC0
:10E90000CE018F5B9F4F0E94C27C64E476E00E9440
:10E91000AC7CBC0188EE9FE00E942B7DCE018F5B1A
:10E920009F4F0E94A77D91CF68EE7FE084EC9FE02F
:10E930000E94577D1092F80B68CF089508950895AE
:10E940000895AF92BF92CF92DF92EF92FF920F9312
:10E950001F93CF93DF936C017B018B01040F151F75
:10E96000EB015E01AE18BF08C017D10759F06991DD
:10E97000D601ED91FC910190F081E02DC601199531
:10E98000892B79F7C501DF91CF911F910F91FF90EE
:10E99000EF90DF90CF90BF90AF900895FC01538D22
:10E9A000448D252F30E0842F90E0821B930B541769
:10E9B00010F0CF96089501970895FC01918D828DF6
:10E9C000981761F0A28DAE0FBF2FB11D5D968C918F
:10E9D000928D9F5F9F73928F90E008958FEF9FEFCE
:10E9E0000895FC01918D828D981731F0828DE80F8A
:10E9F000F11D858D90E008958FEF9FEF0895FC0144
:10EA0000918D228D892F90E0805C9F4F821B910910
:10EA10008F739927089588E89CE00E94FF7421E095
:10EA2000892B09F420E0822F089585E29DE00E9461
:10EA3000FF7421E0892B09F420E0822F0895FC0166
:10EA4000A48DA80FB92FB11DA35ABF4F2C91848D4F
:10EA500090E001968F739927848FA689B7892C93AC
:10EA6000A089B1898C91837080648C93938D848DFF
:10EA7000981306C00288F389E02D80818F7D808302
:10EA80000895EF92FF920F931F93CF93DF93EC01C2
:10EA900081E0888F9B8D8C8D98131AC0E889F98945
:10EAA000808185FF15C09FB7F894EE89FF89608348
:10EAB000E889F98980818370806480839FBF81E0C9
:10EAC00090E0DF91CF911F910F91FF90EF9008950B
:10EAD000F62E0B8D10E00F5F1F4F0F731127E02EE6
:10EAE0008C8D8E110CC00FB607FCFACFE889F9891E
:10EAF000808185FFF5CFCE010E941F75F1CFEB8D90
:10EB0000EC0FFD2FF11DE35AFF4FF0829FB7F894F1
:10EB10000B8FEA89FB8980818062CFCFCF93DF930F
:10EB2000EC01888D8823B9F0AA89BB89E889F98925
:10EB30008C9185FD03C0808186FD0DC00FB607FC5A
:10EB4000F7CF8C9185FFF2CF808185FFEDCFCE018D
:10EB50000E941F75E9CFDF91CF91089580E090E08A
:10EB6000892B29F00E94157581110E94000080E018
:10EB700090E0892B49F080E090E0892B29F00E94F9
:10EB8000000081110E94000080E090E0892B49F094
:10EB900080E090E0892B29F00E94000081110E9402
:10EBA000000080E090E0892B29F00E940B75811114
:10EBB0000C94000008958150823108F05AC0E82F6B
:10EBC000F0E08827E951FA488F4F0C9405B3077697
:10EBD0000B76F975FF75037639760E76147618760E
:10EBE0001E76227626762C763076397634763A760C
:10EBF0003E76809180008F77809380000895809189
:10EC000080008F7DF9CF80918000877FF5CF84B51C
:10EC10008F7784BD089584B58F7DFBCF8091B00040
:10EC20008F778093B00008958091B0008F7DF9CFE9
:10EC3000809190008F77809390000895809190004C
:10EC40008F7DF9CF80919000877FF5CF8091A000D4
:10EC50008F778093A00008958091A0008F7DF9CFD9
:10EC60008091A000877FF5CF809120018F778093DE
:10EC700020010895809120018F7DF9CF809120019E
:10EC8000877FF5CFCF93DF93282F30E0F901E65847
:10EC9000F34F8491F901E55CF24FD491F901EF57FC
:10ECA000F24FC491CC23A1F081110E94DB75EC2FAF
:10ECB000F0E0EE0FFF1FE05AF34FA591B491EC91F5
:10ECC000ED2381E090E009F480E0DF91CF91089599
:10ECD00080E090E0FACF20910C12260F3327331FEB
:10ECE00021323105ECF420917D0CFC0190E080E0B4
:10ECF000243069F082E00895A0910C122191AC01BA
:10ED000044515E4EA40FB52FB11D2C93019686176A
:10ED100098F380910C12680F60930C1280E00895B4
:10ED200081E00895E091460C8091450CE81730F49D
:10ED3000F0E0EE54F44F808190E008958FEF9FEF64
:10ED400008959091460C8091450C2FEF3FEF981756
:10ED500048F4E92FF0E0EE54F44F208130E09F5F5B
:10ED60009093460CC90108958091450C9091460CF2
:10ED7000891B990B0895CF92DF92EF92FF920F9328
:10ED80001F93CF93DF937C01CB018A012091830CE9
:10ED9000222389F0EB016B01C40ED51ECC15DD05D5
:10EDA00069F06991D701ED91FC910190F081E02D1E
:10EDB000C7011995F3CF642F0E946B76C801DF91CC
:10EDC000CF911F910F91FF90EF90DF90CF9008951A
:10EDD000CF93DF931F92CDB7DEB769832091830C69
:10EDE0002223F9F02091860C203258F021E030E007
:10EDF000FC013383228390E080E00F90DF91CF917C
:10EE000008958091840CE82FF0E0EB56FA4E99813A
:10EE100090838F5F8093840C8093860C81E090E0D8
:10EE2000ECCF61E0CE0101960E946B76F7CF0E9495
:10EE30002EB50F931F93CF93DF93EC0188819981B7
:10EE4000009759F02A813B812617370730F081E07F
:10EE5000DF91CF911F910F9108958B016F5F7F4FCD
:10EE60000E944DB4009759F0998388831B830A83CD
:10EE70002C813D81232B59F7FC011082E8CF80E0E3
:10EE8000E7CFEF92FF920F931F93CF93DF9361151C
:10EE9000710541F480E0DF91CF911F910F91FF90B8
:10EEA000EF90089541155105B1F07B01EC010C8103
:10EEB0001D81040F151FB8010E941977882351F393
:10EEC000288139818C819D81B701820F931F0E9417
:10EED0007EB51D830C8381E0DECFCF93DF93EC0101
:10EEE00088819981009711F00E94C4B31982188219
:10EEF0001D821C821B821A82DF91CF910895EF92AE
:10EF0000FF920F931F93CF93DF93EC017B018A0154
:10EF1000BA010E94197781110BC0CE010E946D7752
:10EF2000CE01DF91CF911F910F91FF90EF90089547
:10EF30001D830C83B701888199810E947EB5F0CF33
:10EF40008091E6118823A9F14091680250916902ED
:10EF500060916A0270916B0229E233E18091291578
:10EF600090912A150E94AC0C811102C080E0089596
:10EF70004091E7115091E8116091E9117091EA1107
:10EF8000411551056105710591F029E233E1809148
:10EF9000291590912A150E94AC0C882339F3109200
:10EFA000E7111092E8111092E9111092EA111092F3
:10EFB000E61181E008958F929F92AF92BF92EF92F7
:10EFC000FF920F931F93CF934B015C01C42F80914D
:10EFD000680290916902A0916A02B0916B02881553
:10EFE0009905AA05BB0549F10E94A07781110BC0C4
:10EFF00080E0CF911F910F91FF90EF90BF90AF9065
:10F000009F908F90089589E2E82E83E1F82E00E02A
:10F0100012E030E020E0B501A40180912915909123
:10F020002A150E94050C882319F380926802909299
:10F030006902A0926A02B0926B024091E6114C2BD9
:10F040004093E61181E0D5CF8CBD9DBD0895CF934F
:10F05000DF93EC019A01AB01E889F98982E08083B2
:10F06000211581EE38074105510581F160E079E015
:10F070008DE390E00E9463B12150310941095109AB
:10F080005695479537952795EC85FD851082EE8539
:10F09000FF852083188EEC89FD8986E08083EA89CC
:10F0A000FB89808180618083EA89FB898081886017
:10F0B0008083EA89FB89808180688083EA89FB8973
:10F0C00080818F7D8083DF91CF910895E889F989D0
:10F0D000108220E1D9CF2F923F924F925F926F9290
:10F0E0007F928F929F92AF92BF92CF92DF92EF92D8
:10F0F000FF920F931F93CF93DF9300D0CDB7DEB76E
:10F100001C013B014A0129015801FC01C080D1804A
:10F1100070E060E0C3010E9463B5A80170E060E0A8
:10F12000C2010E9463B5F601808110E000E0811108
:10F1300062C004E010E004C07601F101F182E082D7
:10F14000C8010F900F900F90DF91CF911F910F91F9
:10F15000FF90EF90DF90CF90BF90AF909F908F90F7
:10F160007F906F905F904F903F902F9008956B32FB
:10F1700009F482C06D3309F04EC081818823E9F221
:10F18000F7018FEFE81AF80A6081653209F452C07E
:10F190000CF048C0662309F456C082E0A816B104FA
:10F1A0000CF061C0012B09F46BC003E010E0E8CF64
:10F1B00081818983882309F282818A837601811182
:10F1C00004C0F2E0EF0EF11CB8CF83E0E80EF11CB2
:10F1D0001B8240E150E070E060E0CE0101960E94A9
:10F1E000DCA719C0F3016083F1E08F1A9108C30115
:10F1F00001963C0167017601FFEFEF1AFF0AF60165
:10F200006081663209F499CF0CF0B1CF662309F41E
:10F2100093CF653269F2F2E08F1691041CF701E09A
:10F2200010E0E8CF663209F488CF6B3209F0B5CF31
:10F2300060E2B3CF81818983882301F182818A834F
:10F24000811103C032967F0178CF7F0193E0E90EF0
:10F25000F11C1B8240E150E070E060E0CE010196BD
:10F260000E94DCA79ACFF2016083F1E0AF1AB108E7
:10F27000C20101962C0184CF60E2CDCFF701E3CF2C
:10F2800002E010E07DCF0F931F93CF93DF934115E2
:10F29000510541F0FC01048115810115110539F476
:10F2A000FB011082DF91CF911F910F910895415082
:10F2B00051094017510708F48A01EB01FC016081F4
:10F2C0007181A801CE010E9493B5C00FD11F188291
:10F2D000E9CF20E3FC0120833296862F82958F7040
:10F2E0006F706A3030F4605D6293682F8111F5CFE2
:10F2F0000895695CF9CF8F929F92AF92BF92CF929F
:10F30000DF92EF92FF92CF932EEC3DE030932A15DF
:10F3100020932915882309F46DC040E060E070E077
:10F32000CB010E94DB7781110BC080E0CF91FF9071
:10F33000EF90DF90CF90BF90AF909F908F90089507
:10F340008091E7148F7789F78091F3149091F414EA
:10F35000A091F514B091F61484369105A105B1057C
:10F3600020F3C090EF14D090F014E090F114F090DE
:10F37000F214C114D104E104F104B9F240E0C70170
:10F38000B6010E94DB77882381F28091341390913B
:10F3900035138115924049F6A0913913AA2329F219
:10F3A00060913713709138136115710509F4BDCF61
:10F3B00020913613222309F4B8CFA093EC0D2093AB
:10F3C000DE0D90E080E030E0E1E0F0E0C82FAF013A
:10F3D000082E02C0440F551F0A94E2F72417350780
:10F3E00069F041E0480F01968930910579F7409323
:10F3F000E70D9BCFC12CD12C7601C0CF8093E70DB8
:10F4000020913F133091401350E040E02115310529
:10F4100041F420914D1330914E1340914F13509170
:10F4200050132093DF0D3093E00D4093E10D509386
:10F43000E20D46015701860E971EA11CB11C809259
:10F44000ED0D9092EE0DA092EF0DB092F00DE091C7
:10F450003A13F0913B13F093F30DE093F20DB0E00B
:10F460000E94A4B1DC01CB01880D991DAA1DBB1D12
:10F470008093F40D9093F50DA093F60DB093F70DD6
:10F4800025E0EE0FFF1F2A95E1F7E150FE4FEF2F29
:10F49000FF27E6958E0F9F1FA11DB11D8093E80DDC
:10F4A0009093E90DA093EA0DB093EB0D80903C137F
:10F4B00090903D13B12CA12C8114910441F48090C3
:10F4C000491390904A13A0904B13B0904C13C81A54
:10F4D000D90AEA0AFB0AC80CD91CEA1CFB1C04C0A6
:10F4E000F694E794D794C794CA95D2F7C092E30DE7
:10F4F000D092E40DE092E50DF092E60D85EFC8168E
:10F500008FE0D806E104F10428F48CE08093F10D3B
:10F5100081E00CCF80E125EFC2162FEFD206E10487
:10F52000F104A0F38091551390915613A0915713B5
:10F53000B09158138093F40D9093F50DA093F60DB0
:10F54000B093F70D80E2E2CF8F929F92AF92BF927D
:10F55000CF92DF92EF92FF920F931F93CF93DF939F
:10F56000CDB7DEB760970FB6F894DEBF0FBECDBF44
:10F570007C0190914A0C992351F108E0933309F4EE
:10F5800004E06B0180E591E00E9424789E012F5FEA
:10F590003F4F5901490110E0812F0E949D0FF40156
:10F5A00081934F018823D9F01F5F0113F5CF00E04D
:10F5B000F50181915F018D3161F0883151F08A51FF
:10F5C000823038F00F5F1013F3CF0E94181118E04B
:10F5D0008AC060E170E0802F0E94FB0F102FA12EE7
:10F5E000B12CF501EE0FFF1FEB5CF34F118210827F
:10F5F00083EE93E00197F1F742E870E060E0812F3D
:10F600000E94DE0F4FEF62E070E0812F0E94DE0F5C
:10F61000B601C114D10491F48091900290919102AD
:10F6200001968115F0EC9F0708F471C09093910248
:10F63000809390026091900270919102812F0E94BC
:10F64000C80F86E0E5E2F3E0DE01199601900D9225
:10F650008A95E1F7F70183818F778C8784818D8785
:10F6600085818E87A7014E5F5F4F24E030E06CE01C
:10F6700070E0812F0E94A10FB601812F0E94B20F6E
:10F6800026E030E0AE01475F5F4F66E070E0812F1B
:10F690000E94A10F61E070E0812F0E94FB0F27E024
:10F6A0002A9DC0012B9D900D11249C012350344FA5
:10F6B0007901F9011182108222E030E0AE01415F50
:10F6C0005F4F68E270E0812F0E940B108F85988950
:10F6D000982789279827F7019383828316821582BA
:10F6E00014820E941811812F60960FB6F894DEBF25
:10F6F0000FBECDBFDF91CF911F910F91FF90EF9083
:10F70000DF90CF90BF90AF909F908F90089580E052
:10F7100090EC8CCFFB0101900020E9F73197AF010D
:10F72000461B570B0C947F770F931F93CF93DF9358
:10F73000CDB7DEB762970FB6F894DEBF0FBECDBF70
:10F740008C01CB01F8011182108213821282158282
:10F7500014824AE0BE016F5F7F4F0E9423A9BE0161
:10F760006F5F7F4FC8010E948A7B62960FB6F89444
:10F77000DEBF0FBECDBFDF91CF911F910F910895D6
:10F780000F931F93CF93DF93CDB7DEB7A1970FB63B
:10F79000F894DEBF0FBECDBF8C01CB01BA01F801DA
:10F7A0001182108213821282158214822AE0AE0125
:10F7B0004F5F5F4F0E945DA9BE016F5F7F4FC80121
:10F7C0000E948A7BA1960FB6F894DEBF0FBECDBF14
:10F7D000DF91CF911F910F910895FC01808191815C
:10F7E000009711F00C94DFA860E070E0CB01089561
:10F7F000FC0180819181009711F00C94E3A860E0F6
:10F8000070E0CB010895AF92BF92CF92DF92EF925A
:10F81000FF920F931F93CF93DF93DC01CD90DC9089
:10F820001197C114D10439F01496CD91DC918C015B
:10F830007601209761F4DF91CF911F910F91FF9096
:10F84000EF90DF90CF90BF90AF9008957501570172
:10F85000BFEFAB1ABB0AF7018081082E000C990B91
:10F860000E940AA9892B91F72197CC0DDD1D888173
:10F87000082E000C990B0E940AA9892B29F0CE159D
:10F88000DF0510F02197F3CFAE014F5F5F4F4E19A8
:10F890005F09D80115965C934E931497CE14DF043C
:10F8A00020F4B701C6010E9448B5D801ED91FC9142
:10F8B000119714968D919C91E80FF91F1082BBCF80
:10F8C000FC01248135816217730748F4808191819E
:10F8D000009729F0860F971FFC018081089580E032
:10F8E0000895FC0124813581FB0144815581241751
:10F8F0003507A0F0FC0180819181009779F0FB0130
:10F90000608171816115710549F0241B350B820FEF
:10F91000931F0E9475B521E0892B09F020E0822F0A
:10F920000895FB0144815581FC0124813581241710
:10F93000350778F080819181009759F0FB01608153
:10F9400071816115710529F00E9485B521E0892B2F
:10F9500009F020E0822F0895CF93DF93EC01FB01A3
:10F9600001900020E9F73197AF01461B570B0E9429
:10F970004177811103C0CE010E946D77CE01DF91E6
:10F98000CF910895CF93DF93EC01FB014481558122
:10F99000608171810E944177811103C0CE010E9474
:10F9A0006D77CE01DF91CF910895EF92FF920F9383
:10F9B0001F93CF93DF93EC017B01CB010E941AA927
:10F9C0000097A9F00C811D81080F191FB801CE0105
:10F9D0000E941977882361F0288139818C819D816B
:10F9E000B701820F931F0E9413A91D830C8381E02E
:10F9F000DF91CF911F910F91FF90EF900895CF93DA
:10FA0000DF931F921F92CDB7DEB769831A8241E060
:10FA100050E0BE016F5F7F4F0E9441770F900F90C3
:10FA2000DF91CF910895CF93DF93EC010E94FF7C8B
:10FA3000811103C0CE010E946D77CE01DF91CF917D
:10FA40000895FB0101900020E9F73197AF01461BB3
:10FA5000570B0C944177FB01448155816081718182
:10FA60000C944177EF92FF920F931F93CF93DF9304
:10FA7000EC018B01CB010E941AA97C01BC01CE01D3
:10FA80000E94197781110BC0CE010E946D77CE01C3
:10FA9000DF91CF911F910F91FF90EF900895FD821C
:10FAA000EC82B801888199810E9413A9F0CFCF938D
:10FAB000DF93EC01FB018617970749F060817181A4
:10FAC0006115710541F0448155810E947F77CE0117
:10FAD000DF91CF9108950E946D77F9CF0F931F9317
:10FAE000CF93DF938C01EB01FC0180819181009722
:10FAF000E1F06881798161157105A9F04281538136
:10FB00002C813D814217530770F00E947EB58C8195
:10FB10009D81F801958384831D821C82DF91CF91A2
:10FB20001F910F9108950E94C4B388819981F801B3
:10FB3000918380838A819B81938382838C819D8141
:10FB400095838483198218821B821A82E5CFFC0177
:10FB500080819181009711F00C94C4B30895EF92C5
:10FB6000FF920F931F93CF93DF93CDB7DEB7A1978B
:10FB70000FB6F894DEBF0FBECDBF7C01CB01BA013A
:10FB8000F70111821082138212821582148242E0E0
:10FB9000420F8E010F5F1F4F0E941AA7009789F036
:10FBA000BC01C7010E948A7BA1960FB6F894DEBF04
:10FBB0000FBECDBFDF91CF911F910F91FF90EF90BE
:10FBC0000895C7010E946D77EFCF0F931F93CF93D6
:10FBD000DF93CDB7DEB7A2970FB6F894DEBF0FBEA6
:10FBE000CDBF8C01CB01BA01F801118210821382C2
:10FBF00012821582148230E0AE014F5F5F4F0E9487
:10FC00002EA9BE016F5F7F4FC8010E948A7BA2961A
:10FC10000FB6F894DEBF0FBECDBFDF91CF911F911D
:10FC20000F910895CF93DF931F921F92CDB7DEB748
:10FC3000FC01118210821382128215821482698360
:10FC40001A82BE016F5F7F4F0E948A7B0F900F90D8
:10FC5000DF91CF910895FC011182108213821282EC
:10FC6000158214820C946E7DFC0111821082138225
:10FC70001282158214820C94327DFC011182108252
:10FC800013821282158214820C94577DFC0111821A
:10FC9000108213821282158214826115710551F04F
:10FCA000FB0101900020E9F73197AF01461B570B8C
:10FCB0000C947F770895AF92BF92CF92DF92EF922C
:10FCC000FF920F931F93CF93DF936C015B017A0137
:10FCD00089012417350720F48F2D7901042F182F5F
:10FCE0006DE174E0C6010E94467ED5011496CD9167
:10FCF000DC91EC16FD06E0F40C171D0708F4E80192
:10FD0000D501ED91FC911197EC0FFD1F1081108230
:10FD10006D917C916E0D7F1DC60161157105A1F07D
:10FD20000E948A7BF50180819181C80FD91F1883B9
:10FD3000C601DF91CF911F910F91FF90EF90DF905F
:10FD4000CF90BF90AF9008950E946D77EBCFFB01ED
:10FD500001900020E9F73197AF01461B570BDC01FA
:10FD6000ED91FC910280F381E02D19948F929F9286
:10FD7000AF92BF92EF92FF920F931F93CF93DF93B7
:10FD8000CDB7DEB7A1970FB6F894DEBF0FBECDBFDB
:10FD90007C01FA01CB0119A2223008F42AE08E017D
:10FDA0000F5D1F4F822E912CB12CA12CBF01A501FC
:10FDB00094010E9463B1F901CA016A300CF5605DDB
:10FDC000D8016E938D01232B242B252B79F790E0FE
:10FDD00080E0109721F0BD01C7010E94A77EA19687
:10FDE0000FB6F894DEBF0FBECDBFDF91CF911F914C
:10FDF0000F91FF90EF90BF90AF909F908F900895DC
:10FE0000695CDECF8F929F92AF92BF92CF92DF92CA
:10FE1000EF92FF920F931F93CF93DF937C01EB013F
:10FE20006C0182E0C80ED11C4701E5E08E0E911CEA
:10FE300010E000E0F60141916F0150E070E060E0F9
:10FE40002AE0CE010E94B67E5C01E881F981019032
:10FE5000F081E02D6EE2CE0119958A0D9B1D080FF1
:10FE6000191FC814D90431F7F701458150E070E03B
:10FE700060E02AE0CE010E94B67E800F911FDF91E4
:10FE8000CF911F910F91FF90EF90DF90CF90BF9097
:10FE9000AF909F908F9008950F931F93CF93DF9310
:10FEA000EC010E94A77E8C0167E779E0CE010E94F9
:10FEB000A77E800F911FDF91CF911F910F91089521
:10FEC0006115710511F00C94A77E90E080E0089513
:10FED000DB0114964D915C9115976D917C91DC013D
:10FEE000ED91FC910280F381E02D19940F931F9303
:10FEF000CF93DF93EC010E94687F8C0167E779E084
:10FF0000CE010E94A77E800F911FDF91CF911F919C
:10FF10000F910895EF92FF920F931F93CF93DF936A
:10FF20008C017B01D0E0C0E0F701EC0FFD1F649174
:10FF3000662361F0D801ED91FC910190F081E02DF4
:10FF4000C8011995892B11F02196EECFCE01DF91D2
:10FF5000CF911F910F91FF90EF900895DC0182E106
:10FF600094E08D939D9384E0FB0101900D928A951E
:10FF7000E1F708951F920F920FB60F9211240BB65E
:10FF80000F922F933F934F935F936F937F938F9332
:10FF90009F93AF93BF93EF93FF9388E89CE00E94F9
:10FFA0001F75FF91EF91BF91AF919F918F917F91BD
:10FFB0006F915F914F913F912F910F900BBE0F90DA
:10FFC0000FBE0F901F9018951F920F920FB60F92B1
:10FFD00011240BB60F922F938F939F93EF93FF9360
:10FFE000E091980CF091990C8081E0919E0CF09139
:10FFF0009F0C82FD1DC090818091A10C8F5F8F733B
:020000021000EC
:100000002091A20C821741F0E091A10CF0E0E8579A
:10001000F34F958F8093A10CFF91EF919F918F915A
:100020002F910F900BBE0F900FBE0F901F90189541
:100030008081F2CF1F920F920FB60F9211240BB650
:100040000F922F933F934F935F936F937F938F9371
:100050009F93AF93BF93EF93FF9385E29DE00E9440
:100060001F75FF91EF91BF91AF919F918F917F91FC
:100070006F915F914F913F912F910F900BBE0F9019
:100080000FBE0F901F9018951F920F920FB60F92F0
:1000900011240BB60F922F938F939F93EF93FF939F
:1000A000E091350DF091360D8081E0913B0DF0919E
:1000B0003C0D82FD1DC0908180913E0D8F5F8F733E
:1000C00020913F0D821741F0E0913E0DF0E0EB5D95
:1000D000F24F958F80933E0DFF91EF919F918F91FD
:1000E0002F910F900BBE0F900FBE0F901F90189581
:1000F0008081F2CF1F93CF93DF93282F30E0F90157
:10010000E658F34F8491F901E55CF24FD491F9017F
:10011000EF57F24FC491CC23A9F0162F81110E9402
:10012000DB75EC2FF0E0EE0FFF1FE95FF24FA591BA
:10013000B4918FB7F894EC91111108C0D095DE23DB
:10014000DC938FBFDF91CF911F910895DE2BF8CF05
:10015000AF92BF92CF92DF92EF92FF920F931F93D5
:10016000CF93DF936B017A01EC01CE5EDC4E2881E8
:100170003CE0389F8001399F100D1124A090E515B7
:10018000B12C27FF1FC0FB011182108288818F5F75
:10019000888388819801280F311D87FD3A95F601E3
:1001A0002A153B051CF488818C30C4F18081918133
:1001B000049680349C4908F473C0F60180819181D3
:1001C000049670C088819801280F311D87FD3A95EB
:1001D0002A153B05DCF68881A801480F511D87FDD3
:1001E0005A95FA01EE0FFF1FE40FF51FE35EF14F82
:1001F000808186FFCBCF8881F801E80FF11D87FD54
:10020000FA95CF01EE0FFF1FE80FF91FE35EF14FE4
:10021000808160E08F730E947A80B8CF8081918165
:100220002881A801420F511D27FD5A959A01FA0114
:10023000EE0FFF1FE20FF31FE35EF14F21813281CA
:10024000820F931FF7019183808388819801280F83
:10025000311D87FD3A95F901EE0FFF1FE20FF31FE5
:10026000E35EF14F808186FF22C08881080F111D57
:1002700087FD1A95F801EE0FFF1FE00FF11FE35EF7
:10028000F14F808161E08F73DF91CF911F910F91CA
:10029000FF90EF90DF90CF90BF90AF900C947A805A
:1002A00080E49CE9F701918380838FEF8883DF915D
:1002B000CF911F910F91FF90EF90DF90CF90BF9063
:1002C000AF90089510927D0C81E080937C0C109289
:1002D000570C61E084E10E947A8061E085E10E9430
:1002E0007A80E9EBF0E080818E7F808380818D7F52
:1002F000808388E48093B80085E48093BC000895EF
:100300001092460C1092450C1092840C1092860CA0
:100310000E9462818EE994E79093281380932713BB
:100320008FE994E790932613809325130895CF9334
:10033000DF9390E0FC01E55CF24F24918F57924FE0
:10034000FC0184918823D1F090E0880F991FFC0173
:10035000EF5DF24FA591B491FC01E95FF24FC591B9
:10036000D49161110EC09FB7F8948C91E22FE09563
:100370008E238C932881E223E8839FBFDF91CF9166
:1003800008958FB7F894EC91E22BEC938FBFF6CFE2
:100390003FB7F89480911B1390911C13A0911D13EB
:1003A000B0911E1326B5A89B05C02F3F19F00196EA
:1003B000A11DB11D3FBFBA2FA92F982F8827BC01BF
:1003C000CD01620F711D811D911D42E0660F771FE7
:1003D000881F991F4A95D1F708958F929F92AF92E7
:1003E000BF92CF92DF92EF92FF926B017C010E944D
:1003F000C8814B015C01C114D104E104F104B9F0DE
:100400000E94C881681979098A099B09683E73406E
:100410008105910580F321E0C21AD108E108F108B5
:1004200088EE880E83E0981EA11CB11CE4CFFF90DB
:10043000EF90DF90CF90BF90AF909F908F900895F6
:10044000AF92BF92CF92DF92EF92FF920F931F93E2
:10045000CF93DF93C82FD62F1092581110925911B5
:1004600010925A1110925B1110925C1161E00E947F
:10047000978160E08C2F0E947A806D2F70E090E071
:1004800080E00E94ED8160E08C2F0E9497818BE9D3
:1004900090E00197F1F700E911E08C2F0E9442767D
:1004A000892B81F401501109C1F78EEF9FEFDF9185
:1004B000CF911F910F91FF90EF90DF90CF90BF9061
:1004C000AF90089500E911E08C2F0E9442760197C9
:1004D00021F401501109C1F7E8CF18E2D0E800E09B
:1004E00090E9E92EFF24F3948C2F0E944276892B09
:1004F00029F481E0E81AF108B9F7D7CF0E94C88142
:100500006B017C0180E9A82EBB24B3948C2F0E9440
:100510004276019729F481E0A81AB108B9F7C5CF4E
:100520000E94C8816C197D098E099F096932710585
:100530008105910538F0E02FF0E0E05BFE4E80850C
:100540008D2B8087D69511F40F5FD0E8115041F6BE
:1005500090E080E0ACCF0F931F93CF93DF9300D058
:1005600000D01F921F92CDB7DEB780918B158111FD
:100570002AC0109273151092721588EE93E0A0E0D5
:10058000B0E08093741590937515A0937615B09391
:1005900077158CE993E0909371158093701582E143
:1005A00094E090937F1580937E15109280151092A1
:1005B0008115109282151092831588E0809388151A
:1005C00081E080938B158DE295E190934D0C8093A3
:1005D0004C0C80912C1581119DC060E372E080E08D
:1005E00090E00E94ED811FB7F89480912B15811146
:1005F00027C0E6EBFDE08491E0E7FDE09491E82F71
:10060000F0E0EE0FFF1FEF5DF24FA591B491EC917A
:10061000E92321F461E085E30E947A8061E085E3CB
:100620000E9497818CB580618CBD8CB580648CBD37
:1006300061E084E30E94978161E083E30E949781F7
:1006400080912B158F5F80932B151FBFEBE8FDE08A
:10065000E491F0E0EE0FFF1FE95FF24F8591949176
:100660009093490C8093480CE5E4FDE0E491E0931D
:10067000470C61E08AE00E9497810E94010E80E5AC
:1006800091E00E94247884E380934A0C80E80E94E1
:100690008A0F0E94740F882309F4F5C088E00E9435
:1006A0008A0F0E94610F883009F0EDC080E10E943E
:1006B0008A0F0E94610F803109F0E5C080E00E943E
:1006C0008A0F0E94610F182F8111DDC041E050E0B8
:1006D000BE016F5F7F4F8FE190E00E940B0E89811A
:1006E000833009F0D0C080E480934B0C42E06EE18F
:1006F00070E0812F0E94DE0F42E06FE170E0812FF9
:100700000E94DE0F1F5F183089F70E94181181E0E8
:1007100080932C1580E591E00E94247846E050E01B
:1007200062E972E089E090E00E94B30E82E194E019
:100730009A8389831B821C821D821E82CE010396AE
:100740000E9411110E94181180914C0C90914D0C37
:10075000DC0192961D921D921D921C929597FC01B0
:1007600016A217A210A611A69A961D921D921D926E
:100770001C929D9740E65AEE60E070E046AB57ABA6
:1007800060AF71AF40EA5FE060E070E0DA964D93F1
:100790005D936D937C93DD973E9624E1DF011D927E
:1007A0002A95E9F726E0E2E9F2E0DC0118960190EB
:1007B0000D922A95E1F7FC01EE5BFF4F10820E943B
:1007C000B6298C01019709F0CBC080E591E00E9429
:1007D000247860914C0C70914D0C625F7F4FCE017C
:1007E00001960E94AE7FCE0103960E941111609186
:1007F0004C0C70914D0C6A5E7F4FCE0101960E94A9
:10080000AE7F44E050E0BE016D5F7F4F81E090E03D
:100810000E94B30E60914C0C70914D0C6E5E7F4F38
:10082000CE0101960E94AE7F44E050E0BE016D5FB4
:100830007F4F85E090E00E94B30E0E9418116091F6
:100840004C0C70914D0C625E7F4FCE0101960E9460
:10085000AE7F8B819C81AD81BE818093190E909378
:100860001A0EA0931B0EB0931C0E0E94C8817F73BA
:10087000809190029091910268277927709391025C
:10088000609390026DC087E380934A0C80E80E94D9
:100890008A0F0E94740F882329F188E00E948A0F32
:1008A0000E94610F8830F1F480E10E948A0F0E945B
:1008B000610F182F8031B1F480E00E948A0F0E94EE
:1008C000610F81110FC041E050E0BE016F5F7F4FAB
:1008D00089E390E00E940B0E8981843019F4109313
:1008E0004B0C13CF83E380934A0C80E80E948A0F5D
:1008F0000E94740F882371F180E10E948A0F0E9488
:10090000610F803139F582E10E948A0F0E94610FE8
:10091000823101F580E00E948A0F0E94610F8111EF
:1009200019C084E080934B0C15E5188741E050E036
:10093000BE01685F7F4F8BE190E00E94B30E1F8382
:1009400041E050E0BE01695F7F4F8AE190E00E9484
:10095000B30EDBCE10924A0C0E94181110E000E09A
:10096000C80128960FB6F894DEBF0FBECDBFDF9149
:10097000CF911F910F9108952FB7F894609117139D
:10098000709118138091191390911A132FBF089525
:10099000CF92DF92EF92FF92CF93DF938091C90EB7
:1009A000883050F0CFEFDFEFCE01DF91CF91FF9095
:1009B000EF90DF90CF900895E091EE0EE11142C0EC
:1009C0000E94BC846B017C0128EEC20E23E0D21E83
:1009D000E11CF11C8DEB9EE00E947E15882311F333
:1009E0008091240F882331F08091EF0E9091F00ECA
:1009F000892BC1F28DEB9EE00E94E113EC01CF3F09
:100A0000DC0771F08091240F882371F28091EF0E42
:100A10009091F00E01979093F00E8093EF0EC4CF5B
:100A20000E94BC84C616D706E806F90698F610920E
:100A3000EE0E8DEB9EE00E94D9158DEB9EE00E949C
:100A4000A015B2CFE150E093EE0EF0E0ED54F14F7F
:100A5000C38DD0E0A9CF0F931F93CF93DF93EC0109
:100A60008C01F80181918F018823A1F10E94C88433
:100A7000F8012291022E000C330B8217930789F3A1
:100A80008F3F980781F0A091EE0E91E09A0F90931E
:100A9000EE0EB0E0AD54B14F5B968C93903219F4EA
:100AA0008FE18093EE0E2FE1EC17FD07C9F09291D4
:100AB0009F3FD1F3A091EE0E81E08A0F8093EE0E5E
:100AC000B0E0AD54B14F5B969C93803269F72093B0
:100AD000EE0EEACF81E0DF91CF911F910F91089543
:100AE00080E0F9CF0F931F93CF93DF93EC010E9427
:100AF000BC848B010E94AE0B8F3F69F00E94BC84C6
:100B0000601B710B6C177D07A8F380E0DF91CF911C
:100B10001F910F91089581E0F9CF4F925F926F92EC
:100B20007F928F929F92AF92BF92CF92DF92EF927D
:100B3000FF920F931F93CF93DF93CDB7DEB76397E9
:100B40000FB6F894DEBF0FBECDBF7C016B013A013A
:100B5000FB0120E090E080E06AE03191332309F46A
:100B600061C040ED430F4A3008F04DC0689FA001BE
:100B7000699F500D1124CA01C097830F911D37FD45
:100B80009A958F3F910549F340F3F70142815381D4
:100B9000648175818091DB159091DC15A091DD1544
:100BA000B091DE15481759076A077B0709F40DC293
:100BB0008701085F1F4F0E94BC846F7077277C5F9E
:100BC000C8010E943117813009F004C282E194E02B
:100BD0009A838983F70182819381A481B5818B8374
:100BE0009C83AD83BE8345E350E0BE016F5F7F4FC2
:100BF000C8010E94BA17892BA9F5D12CC12CC801B4
:100C00000E945D1417C03E3209F0BFCF233009F4B3
:100C1000BCCFD301A20FB11D12968C932F5F90E031
:100C200080E09BCF233009F0B0CFF3018583CC2443
:100C3000C394D12CC60163960FB6F894DEBF0FBEE5
:100C4000CDBFDF91CF911F910F91FF90EF90DF907B
:100C5000CF90BF90AF909F908F907F906F905F905C
:100C60004F9008950E94BC84F7017783668342E029
:100C700050E0B7016A5F7F4FC8010E944F1781E0C3
:100C800090E09A83898342E050E0BE016F5F7F4F1E
:100C9000C8010E944F1780E091E09A83898342E067
:100CA00050E0BE016F5F7F4FC8010E944F171A824C
:100CB000198242E050E0BE016F5F7F4FC8010E9481
:100CC0004F1742E050E0BE016F5F7F4FC8010E94A6
:100CD0004F1742E050E0BE016F5F7F4FC8010E9496
:100CE0004F175601F6018081882301F16501F60155
:100CF00081912F01882311F08E32B1F446018A18B8
:100D00009B081814190474F48D8641E050E0BE016C
:100D1000635F7F4FC8010E944F17A401B501C8014E
:100D20000E944F175201DECF6201E1CF1D8641E0E4
:100D300050E0BE01635F7F4FC8010E944F17C12C76
:100D4000DD24D394DA82C98242E050E0BE016F5FB5
:100D50007F4FC8010E944F17DA82C98242E050E0FB
:100D6000BE016F5F7F4FC8010E944F17C8010E94EC
:100D70008917892B09F441CFF3E0AF2EB12C230161
:100D800022E0420E511CD4C0F7014281538164819C
:100D90007581808D918DA28DB38D481759076A0793
:100DA0007B0709F008C1848D958DC59709F003C1B3
:100DB00081A192A15DEFC52EDD24DA940C970CF48D
:100DC000ADC04CE050E0BE016F5F7F4FC8010E9494
:100DD0003C138B819C819827892798279A8B898B34
:100DE000F7014681578129813A814217530709F05B
:100DF000E7C097FFE5C08F7092703BEFC32EDD24F4
:100E0000DA94892B09F08AC06F807884762467246D
:100E100076242AEFC22EDD24DA946114710409F4D9
:100E20007DC0D12CC12C8D819E8198278927982740
:100E3000C816D906F8F441E050E0BE01635F7F4F69
:100E4000C8010E943C134D85442331F050E070E00E
:100E500060E0C8010E943C138D858111ECCF44E015
:100E600050E070E060E0C8010E943C13FFEFCF1A31
:100E7000DF0AD9CF912C812C41E050E0BE016D5E9C
:100E80007F4FC8010E943C134B89842F807C09F05E
:100E90006CC0442331F050E070E060E0C8010E9473
:100EA0003C138B898111E8CF42E050E0BE01615FC5
:100EB0007F4FC8010E943C1342E050E0BE01635FD7
:100EC0007F4FC8010E943C1344E050E070E060E0B6
:100ED000C8010E943C1342E050E0BE016F5E7F4FAC
:100EE000C8010E943C138F85988949895A898115C8
:100EF000914009F043C0CD84DE84DC24CD24DC2481
:100F000081E0C816D104D1F54115544009F04AC01A
:100F100044E050E0B201C8010E943C1321E0A21A53
:100F2000B10809F46CCEFFEFCF16DF0609F067CEEB
:100F30000E94BC843B014C01C8010E948513181615
:100F400019060CF421CF0E94BC8466197709880920
:100F50009909693873418105910548F562E370E0AC
:100F600080E090E00E94ED81E7CF41E050E070E04A
:100F700060E0C8010E943C131B8A93CF5427452789
:100F8000542770E060E0C8010E943C13FFEF8F1A05
:100F90009F0A6814790409F06FCF96EFC92EDD24FB
:100FA000DA94BCCFE7EFCE2EDD24DA94B7CFCC2491
:100FB000CA94DC2CB3CF6EEFC62EDD24DA94AECF0C
:100FC0004CEFC42EDD24DA94A9CF8EEFC82EDD2499
:100FD000DA9430CED12CC12C2DCE1F920F920FB6A9
:100FE0000F9211242F933F938F939F93AF93BF93AF
:100FF0008091171390911813A0911913B0911A139F
:101000003091161323E0230F2D3758F50196A11DBB
:10101000B11D209316138093171390931813A09368
:101020001913B0931A1380911B1390911C13A09164
:101030001D13B0911E130196A11DB11D80931B13AA
:1010400090931C13A0931D13B0931E13BF91AF91E7
:101050009F918F913F912F910F900FBE0F901F90F6
:10106000189526E8230F0296A11DB11DD2CF1F921D
:101070000F920FB60F9211240BB60F922F933F933E
:101080004F935F936F937F938F939F93AF93BF9390
:10109000EF93FF9348E251E064E271E090E080E07A
:1010A0000E94A880FF91EF91BF91AF919F918F9186
:1010B0007F916F915F914F913F912F910F900BBE58
:1010C0000F900FBE0F901F9018951F920F920FB6A2
:1010D0000F9211240BB60F922F933F934F935F9370
:1010E0006F937F938F939F93AF93BF93EF93FF93F0
:1010F00048EA50E064EA70E083E090E00E94A88053
:10110000FF91EF91BF91AF919F918F917F916F91DF
:101110005F914F913F912F910F900BBE0F900FBE9B
:101120000F901F9018951F920F920FB60F921124D7
:101130000BB60F922F933F934F935F936F937F93D1
:101140008F939F93AF93BF93EF93FF9348E950E042
:1011500064E970E082E090E00E94A880FF91EF9146
:10116000BF91AF919F918F917F916F915F914F91BF
:101170003F912F910F900BBE0F900FBE0F901F90BD
:1011800018951F920F920FB60F9211240BB60F9263
:101190002F933F934F935F936F937F938F939F937F
:1011A000AF93BF93EF93FF9348E850E064E870E09B
:1011B00081E090E00E94A880FF91EF91BF91AF91F4
:1011C0009F918F917F916F915F914F913F912F915F
:1011D0000F900BBE0F900FBE0F901F90189560934D
:1011E0000E1370930F138093101390931113645D7B
:1011F0007E4F8F4F9F4F60930A1370930B13809312
:101200000C1390930D1382E090E090930913809358
:1012100008130E94BC846093041370930513809399
:101220000613909307130895CF92DF92EF92FF92E7
:101230000F931F930E94BC848B019C01C0900413E8
:10124000D0900513E0900613F090071360910E13F1
:1012500070910F1380911013909111130C191D09A7
:101260002E093F09083E134021053105E0F0DC015D
:10127000CB010196A11DB11D80930E1390930F1306
:10128000A0931013B0931113B701A60148515C4FFE
:101290006F4F7F4F409304135093051360930613D1
:1012A00070930713C7CF1F910F91FF90EF90DF90BE
:1012B000CF900895CF93DF93EC010E9414899E0193
:1012C000220F331F220F331FF901E152FD4F6083BC
:1012D000718382839383CE01880F991FFC01E952A9
:1012E000FD4F408151811416150644F4FC01E15371
:1012F000FD4F408151811416150614F1FC01E9528D
:10130000FD4F41E050E05183408381539D4FFC01EC
:101310005183408321543D4F88E097E0A0E0B0E046
:10132000F90180839183A283B383CE010E941D1AA9
:1013300064EF71E080E090E0DF91CF910C94ED815B
:10134000DF91CF9108954F925F926F927F928F922B
:101350009F92AF92BF92CF92DF92EF92FF920F9344
:101360001F93CF93DF934B015C0180910013909109
:101370000113A0910213B091031388159905AA05D2
:10138000BB0509F4C6C08CE3C82ED12CE12CF12C8E
:10139000C501A70196010E9463B16093D20BCA01F7
:1013A000B901A70196010E9463B16093D30BC501F7
:1013B000B40120E13EE040E050E00E9463B1CA0188
:1013C000B90128E130E040E050E00E9463B1609351
:1013D000D40BC501B40120E831E541E050E00E94A2
:1013E00063B169017A01CA01B9016C5F7F4F8F4F08
:1013F0009F4F27E030E040E050E00E9463B16F5F14
:101400006093D50B412C512C320140E004E610E0F2
:10141000C0E9D1E0242F30E02E54384FF901E370B9
:10142000FF273097F9F4C901B8010E94F1B2892B66
:1014300031F4C901BE010E94F1B2892B99F48EE604
:1014400091E0A0E0B0E0480E591E6A1E7B1ED30159
:10145000C201AA27BB27C816D906EA06FB0638F040
:101460004F5FD8CF8DE691E0A0E0B0E0ECCF4093A5
:10147000D80BC90164E670E00E94F1B2EC01C90129
:1014800060E971E00E94F1B2309721F42097D9F41D
:101490000097C9F04DE651E060E070E0441A550A4B
:1014A000660A770AC418D508E608F708A5E3B3E08A
:1014B00020E0213069F43097E9F5209711F4009786
:1014C000C9F54DE106C04EE651E060E070E0E6CFC0
:1014D0004C9150E070E060E031E0320FC416D50668
:1014E000E606F70640F0C41AD50AE60AF70A11968E
:1014F000232F3C30F1F62F5F2093D70BC394C0927B
:10150000D60B8092001390920113A0920213B09216
:101510000313DF91CF911F910F91FF90EF90DF9018
:10152000CF90BF90AF909F908F907F906F905F9083
:101530004F9008954CE1CDCF0E9414890E94A38959
:101540008091D80B90E08E54984F08950E94148992
:101550000E94A3898091D70B90E008950E9414897E
:101560000E94A3898091D60B90E008950E9414896F
:101570000E94A3898091D30B90E008950E94148962
:101580000E94A3898091D40B90E008951F920F923E
:101590000FB60F9211240BB60F922F933F934F93D8
:1015A0005F936F937F938F939F93AF93BF93EF93CB
:1015B000FF93809130120E94427620913312309135
:1015C00034122F5F3F4F3093341220933312909197
:1015D0003212953618F096E090932F1290912F12B8
:1015E000943009F46EC0F8F4923031F1933009F47C
:1015F0004CC090913112992319F0811171C02F9A2A
:10160000FF91EF91BF91AF919F918F917F916F91DA
:101610005F914F913F912F910F900BBE0F900FBE96
:101620000F901F901895953009F457C0963009F720
:1016300091E09093FF124FC08111DBCF20913312C4
:10164000309134122436310528F41092341210925D
:101650003312CFCF1092FF1210923212E091321259
:1016600091E09E0F90933212F0E02091331230916E
:101670003412EE0FFF1FEB5CFD4E3183208310927E
:1016800034121092331293E019C0813009F0B1CFB7
:10169000E091321291E09E0F90933212F0E020918F
:1016A000331230913412EE0FFF1FEB5CFD4E31838D
:1016B0002083109234121092331294E090932F12E0
:1016C00098CF882359F22091331230913412253665
:1016D000310508F48ECF95E0F1CF81118ACFB5CFD7
:1016E0002F988ECFCF93DF9391E09093EB118823C7
:1016F000B9F0C091B800D091BA008091BC008A7B4B
:101700008093BC0060E084E10E947A8060E085E123
:101710000E947A800E946281D093BA00C093B80080
:10172000DF91CF9108958F929F92AF92BF92CF9207
:10173000DF92EF92FF920F931F93CF93DF93D0919D
:10174000860CD13208F0D7C0182FC091850C0E94AA
:10175000C8816B017C0180917D0C81116BC082E09E
:1017600080937D0C10937C0C8FEF80937B0C1092F8
:101770007A0CD093790CA5E9B5E1E9E5FCE080E0CD
:10178000D81391C01092580C8091580CCC0FC82BD4
:10179000C093580C8091570C813009F088C010928A
:1017A000570C0E94C8816B017C018091580C80937A
:1017B000BB0080917F0C9091800CA091810CB09126
:1017C000820C892B8A2B8B2BA1F00E94C88100915F
:1017D0007F0C1091800C2091810C3091820C6C193F
:1017E0007D098E099F09061717072807390708F48E
:1017F00042C08091BC0083FDD8CF85EC8093BC00B3
:101800000E94C8816B017C0180917D0C823009F4BB
:1018100050C080917B0C8F3F09F46FC080917B0C8E
:10182000803209F46CC080917B0C803309F469C06C
:1018300084E026C080917F0C9091800CA091810C57
:10184000B091820C892B8A2B8B2B09F484CF0E94B8
:10185000C88180907F0C9090800CA090810CB090FB
:10186000820C6C197D098E099F0986169706A806B9
:10187000B90608F070CF80917E0C0E94728B85E0D3
:101880001092840C1092860C1092830CDF91CF91F1
:101890001F910F91FF90EF90DF90CF90BF90AF908E
:1018A0009F908F9008959D9191938F5F69CF85EE62
:1018B000A5CF80917F0C9091800CA091810CB0916C
:1018C000820C892B8A2B8B2B09F49ECF0E94C88116
:1018D00000917F0C1091800C2091810C3091820C32
:1018E0006C197D098E099F09061717072807390704
:1018F00008F08ACFC0CF81E0C3CF80E0C1CF82E0C3
:10190000BFCF83E0BDCFFC01248131E03093830C55
:101910002093850C1092840C1092860C8385682B82
:1019200082EC9DE00E94E87681E00C94938B0F930B
:101930001F93CF938C01C62F0E94838C6C2F646001
:10194000C8010E94838C6C2F6B7FC8010E94838C1E
:1019500083EC90E00197F1F7CF911F910F910895DB
:101960000F931F93CF938C01C62F607F61600E94FD
:10197000978C80E1C89FB00111246160C8010E946A
:10198000978C81E090E0CF911F910F910895CF93B4
:10199000C82F682F607F84ED91E10E94978C80E1D1
:1019A000C89FB001112484ED91E1CF910C94978CE4
:1019B000CF93DF9300D000D01F921F92CDB7DEB738
:1019C00098E0EBE2F3E0DE01119601900D929A951A
:1019D000E1F79091DD11961708F46FEF70E0660F54
:1019E000771F21E030E02C0F3D1F620F731FFB01BA
:1019F0009081890F806828960FB6F894DEBF0FBEDD
:101A0000CDBFDF91CF910C94C78C85ED8093BC0046
:101A100080917F0C9091800CA091810CB091820CF0
:101A20000796A11DB11D23E0B695A79597958795BB
:101A30002A95D1F72091BC0024FD03C010927D0CA3
:101A4000089540917F0C5091800C6091810C7091B1
:101A5000820C452B462B472B69F30097A105B10556
:101A600041F025E32A95F1F700000197A109B1099A
:101A7000E1CF80917E0C0C94728B1F920F920FB667
:101A80000F9211240BB60F922F933F934F935F93B6
:101A90006F937F938F939F93AF93BF93EF93FF9336
:101AA0008091B900887F803609F44DC008F040C0AD
:101AB000883209F4A9C028F5803109F49DC0C8F422
:101AC000882309F4FBC0883009F496C0FF91EF9198
:101AD000BF91AF919F918F917F916F915F914F9146
:101AE0003F912F910F900BBE0F900FBE0F901F9044
:101AF0001895883109F488C0803241F780937B0CB7
:101B000014C0803409F49DC040F48033B9F38833A5
:101B1000E9F680937B0C85ECB0C0803509F485C074
:101B2000883509F496C0883489F60E94058DCECF99
:101B3000883909F48CC038F5883729F050F4883694
:101B400011F0803719F683E080937D0C10922E12ED
:101B500057C0883809F47BC0803919F0803809F003
:101B6000B5CF80912E12803208F071C0E0912E1214
:101B700081E08E0F80932E128091BB00F0E0E25F37
:101B8000FD4E80833DC0803B39F0E0F4803A09F49B
:101B900079C0883A09F09ACF84E080937D0C109246
:101BA0000D1210920C12E0912713F0912813199541
:101BB00080910C1281110FC081E080930C12109261
:101BC000EC1109C0803C09F4A6CF883C09F4A3CFEE
:101BD000883B09F07BCFE0910D1281E08E0F80935E
:101BE0000D12F0E0E451FE4E80818093BB00909195
:101BF0000D1280910C1229C08091580C8093BB006B
:101C000085EC8093BC0062CF90917A0C8091790C26
